:100000000C94D6250C9407260C9407260C940726EE
:100010000C9407260C9407260C9407260C940726AC
:100020000C9407260C9407260C9407260C9407269C
:100030000C9407260C9407260C9407260C9407268C
:100040000C9407260C9481750C9407260C940726B3
:100050000C9407260C9407260C9406A50C9492C2C7
:100060000C9407260C94A7460C9407260C9407269C
:100070000C9407260C9407260C9407260C9407264C
:100080000C9407260C9407260C9407260C9407263C
:100090000C9407260C9407260C9407260C9407262C
:1000A0000C9407260C9407260C9407260C9407261C
:1000B0000C9407260C9407260C9407260C9407260C
:1000C0000C9407260C9407260C9407260C940726FC
:1000D0000C9407260C9407260C9407260C940726EC
:1000E0000C940726A6AB07AA3DAAE2AB3DAA3DAAFF
:1000F0003DAA3DAA3DAA3DAA3DAA3DAA3DAA3DAAC8
:100100003DAA3DAA3DAA3DAA3DAA3DAA3DAA3DAAB7
:100110003DAA3DAA3DAA3DAA3DAA3DAA3DAA3DAAA7
:10012000DCAB3DAA3DAA3DAA3DAA3DAA3DAA3DAAF7
:100130003DAAB5AB3DAA3DAA3DAA3DAA3DAA3DAA0E
:100140003DAA3DAA3DAA3DAAF9AB3AAA0FC112C1E8
:1001500001C105C10BC149C116C11AC120C124C1C9
:1001600028C12EC132C136C149C13CC140C144C1C0
:10017000AEC1B3C1B8C1C2C1CCC145C2D6C1DEC1D6
:10018000E6C1F0C1FAC104C213C21DC245C227C2F2
:1001900031C23BC2084AD73B3BCE016E84BCBFFD97
:1001A000C12F3D6C74319ABD56833DDA3D00C77F47
:1001B00011BED9E4BB4C3E916BAAAABE00000080E0
:1001C0003F05A84CCDB2D44EB93836A9020C50B96F
:1001D000918688083CA6AAAA2ABE000000803F009B
:1001E0004E414E494E495459494E46CDCCCC3D0A1C
:1001F000D7233C17B7D13877CC2B329595E6241FFF
:10020000B14F0A000020410000C84200401C4620B7
:10021000BCBE4CCA1B0E5AAEC59D7400407A10F38A
:100220005A00A0724E18090010A5D4E80000E87624
:1002300048170000E40B54020000CA9A3B0000007B
:10024000E1F505000080969800000040420F000094
:1002500000A08601000000102700000000E8030055
:100260000000006400000000000A0000000000011F
:1002700000000000002C76D888DC674F0823DFC11F
:10028000DFAE59E1B1B796E5E3E453C63AE65199DA
:100290007696E8E6C28426EB898C9B62ED407C6F03
:1002A000FCEFBC9C9F40F2BAA56FA5F490055A2ABA
:1002B000F75C936B6CF9676DC11BFCE0E40D47FEC6
:1002C000F520E6B500D0ED902E03009435770500BB
:1002D00080841E080000204E0A000000C80C333342
:1002E00033330F986E12831141EF8D2114893BE651
:1002F0005516CFFEE6DB18D1844B381BF77C1D90DA
:100300001DA4BBE424203284725E228100C9F12442
:10031000ECA1E53D27434F4D4D554E4943415449CE
:100320004F4E0044525952554E004552524F52536F
:1003300000494E464F004543484F0047322F473350
:100340002062616420706172616D65746572730A08
:1003500000536C6565702E2E2E0043522D313020D7
:1003600056322072656164792E00526573756D692D
:100370006E67207072696E7400436C69636B2074E1
:100380006F20726573756D652E2E2E004E6F206D79
:100390006F76652E00456E642066696C65206C6919
:1003A00073740A00426567696E2066696C65206C2B
:1003B0006973740A005446207072696E74696E67BE
:1003C000206279746520004E6F742054462070724C
:1003D000696E74696E670A0046696C652064656CB5
:1003E000657465643A0044656C6574696F6E206677
:1003F00061696C65642C2046696C653A20006F70F9
:10040000656E206661696C65642C2046696C653A8E
:1004100020002569730025696D2025697300256911
:10042000682025696D202569730025696420256988
:10043000682025696D202569730025697920256963
:1004400064202569682025696D2025697300507234
:10045000696E742074696D653A200050726F74651E
:10046000637465642050696E0A004578747275641F
:1004700065722025730043522D3130205632207290
:10048000656164792E00360331032A0323031503C3
:100490006F66660044454255473A004B494C4C450F
:1004A000442E20004D3131332053006F6B004352F6
:1004B0002D3130205632204F66662E004361703A4F
:1004C000454D455247454E43595F50415253455261
:1004D0003A300A004361703A434153455F4C494703
:1004E00048545F4252494748544E4553533A300AA4
:1004F000004361703A544F47474C455F4C49474869
:1005000054533A300A004361703A534F46545741AE
:1005100052455F504F5745523A300A004361703A96
:100520004C4556454C494E475F444154413A300A88
:10053000004361703A5A5F50524F42453A300A00C8
:100540004361703A4155544F4C4556454C3A300A38
:10055000004361703A5052494E545F4A4F423A311B
:100560000A004361703A50524F47524553533A3054
:100570000A004361703A4155544F5245504F52540E
:100580005F54454D503A310A004361703A45455039
:10059000524F4D3A310A004649524D574152455F3C
:1005A0004E414D453A4D61726C696E2043726561F2
:1005B0006C69747920334420534F555243455F434F
:1005C0004F44455F55524C3A68747470733A2F2FFC
:1005D0006769746875622E636F6D2F4D61726C6907
:1005E0006E4669726D776172652F4D61726C696ECE
:1005F0002050524F544F434F4C5F56455253494F32
:100600004E3A312E30204D414348494E455F5459B2
:1006100050453A43522D31302056322045585452DD
:10062000554445525F434F554E543A312055554934
:10063000443A63656465326132662D343161322D2E
:10064000343734382D396231322D633535633632E3
:100650006633363766660A002F2F20004D31343559
:1006600020533C696E6465783E206F7574206F6618
:100670002072616E67652028302D31290A0053658C
:100680007474696E672054726176656C204163638F
:10069000656C65726174696F6E3A2000536574749D
:1006A000696E67205265747261637420416363658B
:1006B0006C65726174696F6E3A2000536574746979
:1006C0006E67205072696E7420416363656C657259
:1006D0006174696F6E3A200053657474696E6720A7
:1006E0005072696E7420616E642054726176656C1C
:1006F00020416363656C65726174696F6E3A2000B6
:10070000205A00205900580020204D61783A2000DE
:10071000205A00205900580020204D696E3A2000D0
:100720004F6E20004F666600536F667420656E64DE
:1007300073746F70733A2000000136372603FF3C54
:100740003D380EFF2E303E12FFFF0C0809FFFFFF61
:100750001A1C18FFFF08440AFF43FFFFFFFFFFFFBB
:1007600020643A0020693A0020703A0020643A0080
:1007700020693A0020703A0043290A0061626C65E2
:100780006420286D696E2074656D702000436F6C65
:1007900064206578747275646573206172652000E9
:1007A0004F666673657473206170706C6965640070
:1007B0004572723A20546F6F206661722100546F47
:1007C0006F206661722066726F6D20726566657259
:1007D000656E636520706F696E740A004E6F2063EA
:1007E000617365206C696768740A00416374697697
:1007F000652045787472756465723A2000556E6B99
:100800006E6F776E20636F6D6D616E643A202200AB
:100810004B494C4C45442E200053544F50504544B6
:100820002E20005072696E7465722073746F707040
:1008300065642064756520746F206572726F7273D1
:100840002E2046697820746865206572726F722068
:10085000616E6420757365204D39393920746F20BD
:10086000726573746172742E202854656D706572A0
:1008700061747572652069732072657365742E20CA
:1008800053657420697420616674657220726573A3
:1008900074617274696E67290A004E6F204C696E2C
:1008A00065204E756D626572207769746820636893
:1008B00065636B73756D2C204C617374204C696E8D
:1008C000653A20004E6F20436865636B73756D2039
:1008D00077697468206C696E65206E756D626572EB
:1008E0002C204C617374204C696E653A200063685B
:1008F00065636B73756D206D69736D617463682CCE
:10090000204C617374204C696E653A20004C696E0E
:1009100065204E756D626572206973206E6F74205C
:100920004C617374204C696E65204E756D62657202
:100930002B312C204C617374204C696E653A200079
:100940004D313130004D3331004D3834205820596D
:10095000205A2045005446207265616420657272F9
:100960006F720A00446F6E65207072696E74696EF2
:10097000672066696C650A0020496E76616C69645F
:1009800020657874727564657220000000000000B4
:100990000000000000000000009B4300009B43009B
:1009A00000CD434D36303020486F74656E6420743E
:1009B0006F6F20636F6C6420746F206368616E6773
:1009C000652066696C616D656E740A000000000048
:1009D0000000000000000000000000000000000017
:1009E0000000000000000000000000000000000007
:1009F00000000000000000000000000000000000F7
:100A000000000000000000000000000000000000E6
:100A100000000000000000000000000000000000D6
:100A200000000000000000000000000000000000C6
:100A300000000000000000000000000000000000B6
:100A40000000000000000000000000000000008026
:100A5000000008000000000000000000000000800E
:100A600000000800000000000000000000209E9D23
:100A7000E773C800000000000000000000359291FC
:100A800024924800000000000000000000151E91A4
:100A90002493C8000000000000000000001B10911B
:100AA000249200000000000000000000000A1E9DCB
:100AB000E493C800000000000000000000000000F7
:100AC0000000000000000000000000000000000026
:100AD0000000000000000000000000000000000016
:100AE0000000000000000000000000000000000006
:100AF00000000000000000000000000000000000F6
:100B000000000000000000000000000000000000E5
:100B100000000000000000000000000000000000D5
:100B200000000000000000000000000000000000C5
:100B300000000000000000000000000000000000B5
:100B400000000000000000000000000000000000A5
:100B50000000000000000000000000000000000095
:100B60000000000000000000000000000000000085
:100B70000000000000000000000000000000000075
:100B80000000000000000000000000000000000065
:100B90000000000000000000000000000000000055
:100BA00000000000000000000000000000000FFD39
:100BB000FFC0FF80C0600FFFF80F000000001FFDA6
:100BC000FFE3FF80C0600FFFF81E000000003C0143
:100BD00080678001C0600E0E1E3C000000007001A6
:100BE00080670001E0600E0E0F78000000006001D9
:100BF000806E0003E0600E0E07F000000000600150
:100C0000BFEFFF8370600E0E03E000000000600184
:100C10009FCFFF8738600E0E01C00000000060010A
:100C20008E0E000718600E0E01C00000000070015B
:100C30008707000E1E600E0E01C0000000003C0180
:100C40008387800C0E600E0E01C0000000001FFDA7
:100C500081C3FF9CFE7FEE0E01C0000000000FFD6F
:100C600080E0FFBDFF7FEE0E01C00000000000002D
:100C70000000000000000000000000000000000074
:100C80000000000000000000000000000000000064
:100C90000000000000000000000000000000000054
:100CA0000000000000000000000000000000000044
:100CB0000000000000000000000000000000000034
:100CC0000000000000000000000000000000000024
:100CD0000000000000000000000000000000000014
:100CE0000000000000000000000000000000000004
:100CF00000000000000000000000000000000000F4
:100D000000000000000000000000000000000000E3
:100D100000000000000000000000000000000000D3
:100D200000000000000000000000000000000000C3
:100D300000000000000000000000000000000000B3
:100D400000000000000000000000000000000000A3
:100D50000000000000000000000000000000000093
:100D60000000000000000000000000000000000083
:100D70000000000000000000000000000000000073
:100D80000000000000000000000000000000000063
:100D90000000000000000000000000000000000053
:100DA0000000000000000000000000000000000043
:100DB0000000000000000000000000000000000033
:100DC00000000000000000000000000025753A252A
:100DD00030327500253032753A2530327500257570
:100DE0006420253032753A25303275005A0059009A
:100DF0005800092000000000000000000000000072
:100E000000003FFFF00000000000000000000000B4
:100E1000000038007000000000000000000000002A
:100E2000000030FC30000000000000000000000066
:100E3000000020FC10000000000000000000000086
:100E400000002078100000000000000000000000FA
:100E500000002030107BC08C2260000000000000E9
:100E600000002C00D08A219222901FE00000104147
:100E700000002E31D082209222103FF00000082086
:100E800080002F7BD083DE9222203FF000000820DC
:100E900080002F7BD082809222403FF000001041E2
:100EA00000002E31D08A409214801FE00000208282
:100EB00000002C00D07221CC08F01FE0000041049B
:100EC000000020301000000000003FF0000041044E
:100ED000000020781000000000003FF00000208299
:100EE000000020FC1000000000003FF00000104156
:100EF000000030FC3000000000000FC000000000C7
:100F00000000380070000000000007800000FFFFB4
:100F1000C0003FFFF0000000000003000000FFFFE2
:100F2000C000000000000000000000000000000001
:100F300000003FFFF0000000000000000000000083
:100F400000003800700000000000000000000000F9
:100F500000003387300000000000000000000000A7
:100F60000000278790000000000000000000000043
:100F700000002F87D00000000000000000000000EB
:100F800000002F87D07BC08C226000000000000092
:100F900000002F03D08A219222901FE00000082039
:100FA000800020301082209222103FF000000410B8
:100FB000400020781083DE9222203FF000000410D1
:100FC000400020781082809222403FF000000820EC
:100FD00080002030108A409214801FE000001041F1
:100FE00000002F03D07221CC08F01FE00000208207
:100FF00000002F87D000000000003FF0000020829A
:1010000000002F87D000000000003FF000001041DA
:10101000000027879000000000003FF0000008203B
:10102000800033873000000000000FC00000000087
:101030000000380070000000000007800000FFFF83
:10104000C0003FFFF0000000000003000000FFFFB1
:10105000C0000000005873746570732F6D6D0058E8
:1010600073746570732F6D6D005873746570732F92
:101070006D6D005973746570732F6D6D00597374C5
:101080006570732F6D6D005973746570732F6D6D7E
:10109000005A73746570732F6D6D005A73746570A8
:1010A000732F6D6D005A73746570732F6D6D0045ED
:1010B00073746570732F6D6D004573746570732F55
:1010C0006D6D004573746570732F6D6D0056656CA2
:1010D0006F636974790056656C6F63697479005643
:1010E000656C6F6369747900416363656C657261F7
:1010F00074696F6E00416363656C65726174696FDA
:101100006E00416363656C65726174696F6E004A5D
:1011100065726B004A65726B004A65726B005374AE
:101120006570732F6D6D0053746570732F6D6D0056
:1011300053746570732F6D6D004520696E206D6D61
:1011400033004520696E206D6D33004520696E20A7
:101150006D6D330046696C2E204469612E0046692E
:101160006C2E204469612E0046696C2E2044696112
:101170002E004F6666004F6E200043616E6E6F74E6
:1011800020656E746572207375626469723A20001E
:10119000022E2E0041626F7574205072696E746564
:1011A000720041626F7574205072696E74657200CE
:1011B00041626F7574205072696E74657200777742
:1011C000772E637265616C69747933642E636E0087
:1011D0007777772E6378737733642E636F6D00773C
:1011E00077772E637265616C69747933642E636EF0
:1011F00000457874727564657273203100457874A7
:101200007275646572732031004578747275646517
:101210007273203100426175643A203131353230C9
:101220003000426175643A2031313532303000424D
:101230006175643A20313135323030004372656176
:101240006C6974792056322E350043522D3130208E
:10125000563200312E312E362E3000437265616CCD
:1012600069747920334400202F002042403A002046
:10127000403A0048656174696E6720646F6E652E40
:101280000020573A004578747275646572202573A2
:101290000043522D31302056322072656164792E20
:1012A0000042656420646F6E652E0020573A00424C
:1012B00065642048656174696E672E00205A3A00A3
:1012C00020593A0020436F756E7420583A0020452B
:1012D0003A00205A3A0020593A00583A004B64200C
:1012E0000023646566696E65202044454641554C7F
:1012F000545F004B69200023646566696E65202099
:1013000044454641554C545F004B702000236465B2
:1013100066696E65202044454641554C545F005037
:101320004944204175746F74756E652066696E69F5
:1013300073686564212050757420746865206C6141
:101340007374204B702C204B6920616E64204B64B9
:1013500020636F6E7374616E74732066726F6D209C
:1013600062656C6F7720696E746F20436F6E66697B
:101370006775726174696F6E2E680A005049442067
:101380004175746F74756E65206661696C65642162
:101390002074696D656F75740A0050494420417569
:1013A000746F74756E65206661696C656421205484
:1013B000656D706572617475726520746F6F2068F9
:1013C0006967680A00204B643A2000204B693A2084
:1013D00000204B703A20000A20436C6173736963EC
:1013E00020504944200A002054753A2000204B75B3
:1013F0003A2000206D61783A2000206D696E3A2015
:101400000020643A200020626961733A2000566D22
:101410006178205800566D6178205800566D6178CB
:10142000205800566D6178205900566D617820591A
:1014300000566D6178205900566D6178205A00562B
:101440006D6178205A00566D6178205A00566D61A2
:1014500078204500566D6178204500566D617820F2
:101460004500566D696E00566D696E00566D696E69
:10147000005654726176206D696E00565472617622
:10148000206D696E005654726176206D696E004160
:101490006363656C00416363656C00416363656C05
:1014A00000412D7265747261637400412D72657420
:1014B0007261637400412D726574726163740041DE
:1014C0002D74726176656C00412D74726176656C65
:1014D00000412D74726176656C00416D6178205811
:1014E00000416D6178205800416D617820580041BD
:1014F0006D6178205900416D6178205900416D611E
:1015000078205900416D6178205A00416D61782042
:101510005A00416D6178205A00416D617820450084
:10152000416D6178204500416D6178204500567815
:101530002D6A65726B0056782D6A65726B0056785D
:101540002D6A65726B0056792D6A65726B0056794B
:101550002D6A65726B0056792D6A65726B00567A3A
:101560002D6A65726B00567A2D6A65726B00567A29
:101570002D6A65726B0056652D6A65726B00566543
:101580002D6A65726B0056652D6A65726B00577225
:101590006974696E6720746F2066696C653A200013
:1015A0006F70656E206661696C65642C2046696C9D
:1015B000653A20006F70656E206661696C65642C09
:1015C0002046696C653A200046696C652073656C3D
:1015D00065637465640A002053697A653A200046A1
:1015E000696C65206F70656E65643A20006F706588
:1015F0006E206661696C65642C2046696C653A20D2
:10160000002066696C653A20004E6F77200022202A
:10161000706F73002220706172656E743A220053FD
:101620005542524F5554494E452043414C4C20742D
:1016300061726765743A22004B494C4C45442E2038
:1016400000747279696E6720746F2063616C6C201E
:101650007375622D67636F64652066696C657320BE
:101660007769746820746F6F206D616E79206C6586
:1016700076656C732E204D4158206C6576656C2024
:1016800069733A0043616E6E6F74206F70656E20EF
:10169000737562646972200054462063617264202D
:1016A0006F6B0A006F70656E526F6F7420666169B0
:1016B0006C65640A00766F6C756D652E696E697471
:1016C000206661696C65640A004572726F723A0047
:1016D000544620696E6974206661696C0A00617500
:1016E000746F25692E67004D3234004D323320254A
:1016F000730024F4D43050C38E20C2A24017828BD2
:101700007011127A910D816CD90AA861E108C7584D
:101710006607615143061E4B5D05C145A7041A418A
:101720001104093D9803713931034036DB026533FA
:101730009102D4305402802E1D02632CEE01752AD2
:10174000C501B028A001102781018F2564012B2439
:101750004B01E0223401AC211F018D200D01801FBF
:10176000FC00841EED00971DDF00B81CD200E61BB4
:10177000C600201BBC00641AB200B219A8000A19E6
:10178000A0006A189900D117910040178B00B51678
:10179000840031167E00B31579003A157300C71422
:1017A0006F0058146A00EE13660088136300251357
:1017B0005E00C7125B006C12570015125400C11175
:1017C000510070114F0021114B00D61049008D10AF
:1017D00047004610440002104200C00F4000800F36
:1017E0003E00420F3C00060F3B00CB0E3800930E2C
:1017F00037005C0E3500270E3400F30D3200C10DAA
:101800003100900D3000600D2E00320D2D00050DC1
:101810002C00D90C2B00AE0C2900850C29005C0C87
:101820002700350C27000E0C2600E80B2400C40B03
:101830002400A00B23007D0B23005A0B2100390B41
:101840002100180B2000F80A1F00D90A1E00BB0A4D
:101850001E009D0A1D00800A1D00630A1C00470A25
:101860001B002C0A1B00110A1A00F7091A00DD09D7
:101870001900C4091900AB091900920917007B0966
:101880001800630917004C091600360916002009D4
:1018900016000A091500F5081500E0081400CC0828
:1018A0001400B8081400A4081400900813007D0860
:1018B00012006B0813005808120046081200340882
:1018C0001100230811001208110001081100F0078F
:1018D0001000E0071000D0071000C0071000B0078C
:1018E0000F00A107100091070E0083070F00740777
:1018F0000F0065070E0057070E0049070E003B0753
:101900000D002E070E0020070D0013070D0006071F
:101910000D00F9060C00ED060D00E0060C00D406E3
:101920000C00C8060C00BC060C00B0060C00A40697
:101930000B0099060C008D060B0082060B00770643
:101940000B006C060B0061060A0057060B004C06E4
:101950000A0042060A0038060A002E060A0024067B
:101960000A001A060A001006090007060A00FD050B
:101970000900F4050900EB050900E2050900D90595
:101980000900D0050900C7050900BE050900B50515
:101990000800AD050800A50509009C050800940590
:1019A00008008C050800840508007C050800740503
:1019B00008006C050700650508005D050700560571
:1019C00008004E05070047050700400508003805D8
:1019D0000700310507002A050700230507001C053D
:1019E0000600160507000F0507000805060002059A
:1019F0000700FB040600F5040700EE040600E804F7
:101A00000600E2040700DB040600D5040600CF044C
:101A10000600C9040600C3040600BD040600B7049E
:101A20000600B1040500AC040600A6040600A004EC
:101A300005009B04060095040500900406008A0436
:101A4000050085040500800406007A04050075047D
:101A50000500700405006B040500660405006104C0
:101A600005005C04050057040500520405004D0400
:101A7000050048040500430405003E0404003A0440
:101A8000050035040500300404002C04050027047B
:101A90000400230405001E0404001A0404001604B4
:101AA0000500110404000D040400090405000404E9
:101AB000040000040400FC030400F8030400F40321
:101AC0000400F0030400EC030400E8030400E40352
:101AD0000400E0030400DC030400D8030400D40382
:101AE0000400D0030400CC030400C8030300C503B2
:101AF000030024F404D9201BC40C5C0E9804C40910
:101B00005F0265077101F405F900FB04B3004804A6
:101B10008700C10369005803550003034500BE0256
:101B20003A008402310053022A00290225000402EF
:101B30002000E4011C00C8011900AF011700980142
:101B400014008401130071011000610110005101A3
:101B50000E0043010D0036010B002B010B0020018C
:101B60000B00150109000C01090003010800FB002E
:101B70000800F3000800EB000700E4000600DE00A8
:101B80000600D8000600D2000600CC000500C70001
:101B90000500C2000500BD000400B9000400B50046
:101BA0000400B1000400AD000400A9000400A50079
:101BB0000300A20003009F0004009B0003009800A4
:101BC00003009500020093000300900003008D00C5
:101BD00002008B00030088000200860002008400DF
:101BE0000300810002007F0002007D0002007B00F4
:101BF0000200790002007700010076000200740004
:101C0000020072000100710002006F0002006D000E
:101C100001006C0002006A00010069000200670018
:101C2000010066000100650001006400020062001E
:101C3000010061000100600001005F0002005D0022
:101C400001005C0001005B0001005A000100590026
:101C50000100580001005700010056000100550026
:101C60000100540001005300000053000100520025
:101C7000010051000100500001004F0001004E0022
:101C800000004E0001004D0001004C0001004B001F
:101C900000004B0001004A0001004900010048001B
:101CA0000000480001004700010046000000460017
:101CB0000100450000004500010044000100430010
:101CC000000043000100420000004200010041000A
:101CD000000041000100400001003F0000003F0003
:101CE00001003E0000003E0001003D0000003D00FC
:101CF00001003C0000003C0000003C0001003B00F3
:101D000000003B0001003A0000003A0001003900E9
:101D100000003900010038000000380000003800E1
:101D200001003700000037000100360000003600D7
:101D300000003600010035000000350000003500CD
:101D400001003400000034000000340001003300C2
:101D500000003300000033000100320000003200B8
:101D600000003200010031000000310000003100AD
:101D700001003000000030000000300001002F00A2
:101D800000002F0000002F0000002F0001002E0097
:101D900000002E0000002E0001002D0000002D008C
:101DA00000002D0000002D0001002C0000002C0080
:101DB00000002C0000002C0001002B0000002B0074
:101DC00000002B0000002B0001002A0000002A0068
:101DD00000002A0000002A0001002900000029005C
:101DE000000029000000290000002900010028004F
:101DF0000000280000002800000028000000280043
:101E00000100270000002700000027000000270035
:101E10000000270001002600000026000000260028
:101E2000000026000000260001002500000025001B
:101E3000000025000000250000002500000025000E
:101E40000100240000002400000024000000240001
:101E500000002400010023000000230000002300F4
:101E600000002300000023000000230000002300E6
:101E700001002200000022000000220000002200D9
:101E800000002200000022000100210000002100CB
:101E900000002100000021000000210000002100BE
:101EA00000002100010020000000200000002000B0
:101EB00000002000000020000000200000002000A2
:101EC0000000200001001F0000001F0000001F0094
:101ED00000001F0000001F0000001F0000001F0086
:101EE00001001E0000001E0000001E0000001E0079
:101EF00000004D383420582059205A204500626592
:101F0000640A002C2073797374656D2073746F708C
:101F100070656421204865617465725F49443A20A8
:101F20000048656174696E67206661696C6564006C
:101F300048656174696E67206661696C6564004814
:101F4000656174696E67206661696C6564004865E7
:101F50006174696E67206661696C65640020440085
:101F600020490020204D33303420500020440020F0
:101F7000490020204D333031205000504944207317
:101F8000657474696E67733A0A0020460020420047
:101F900020480020204D3134352053004D617465B8
:101FA0007269616C2068656174757020706172611E
:101FB0006D65746572733A0A00205A00205900203A
:101FC000204D323036205800486F6D65206F6666B0
:101FD0007365743A0A00204500205A0020590020F9
:101FE000580020420020540020204D32303520532C
:101FF00000416476616E6365643A20533C6D696E9E
:102000005F66656564726174653E20543C6D696EFF
:102010005F74726176656C5F666565647261746534
:102020003E20423C6D696E5F7365676D656E745FDF
:1020300074696D655F6D733E20583C6D61785F78A3
:10204000795F6A65726B3E205A3C6D61785F7A5F9A
:102050006A65726B3E20453C6D61785F655F6A65BD
:10206000726B3E0A0020540020520020204D323076
:1020700034205000416363656C65726174696F6EF2
:102080002028756E6974732F7332293A20503C7082
:1020900072696E745F616363656C3E20523C726569
:1020A00074726163745F616363656C3E20543C7459
:1020B000726176656C5F616363656C3E0A00204502
:1020C00000205A0020590020204D32303120580085
:1020D0004D6178696D756D20416363656C657261F2
:1020E00074696F6E2028756E6974732F7332293A84
:1020F0000A00204500205A0020590020204D32308F
:10210000332058004D6178696D756D206665656492
:1021100072617465732028756E6974732F73293A20
:102120000A00204500205A0020590020204D393255
:1021300020580053746570732070657220756E6945
:10214000743A0A0020204D3230302044300A0020FA
:10215000204D3230302044002044697361626C6548
:10216000640A0046696C616D656E742073657474F1
:10217000696E67733A0020204D3134392043203B8B
:1021800020556E69747320696E2043656C736975A0
:10219000730A002020473231202020203B20556E3A
:1021A00069747320696E206D6D0A007A5F6D696EC7
:1021B0003A2000795F6D696E3A2000785F6D696E34
:1021C0003A20005265706F7274696E6720656E64A4
:1021D00073746F70207374617475730A0000002249
:1021E00000250028002B002E0031003400020100E1
:1021F00000050108010B0100002000230026002932
:10220000002C002F0032000001000003010601092C
:102210000105050505070508080808020202020A6B
:102220000A08080404040401010101010101010379
:1022300003030303030303040707070C0C0C0C0C34
:102240000C0C0C0202020206060606060606060B27
:102250000B0B0B0B0B0B0B0102102020080810209E
:102260004010204080020102010804020101020422
:1022700008102040808040201008040201800402E1
:102280000180402010080402010804020101020438
:102290000810204080010204081020408000000A3D
:1022A0000B02090C0D0E08070304010000000000DA
:1022B000000000000000000000000000000000001E
:1022C00000000000000000000012111000000000DB
:1022D00000000000000000000000000000000000FE
:1022E0000000002020506C616E6E6572427566665B
:1022F000657242797465733A2000204672656520E4
:102300004D656D6F72793A2000436F6D70696C6531
:10231000643A2044656320203520323031390A0088
:10232000207C20417574686F723A2043522D313001
:102330002056320A00323031392D31322D303500FD
:10234000204C61737420557064617465643A200098
:10235000312E312E362E300A004D61726C696E00BE
:1023600020536F6674776172652052657365740AD5
:1023700000205761746368646F67205265736574E9
:102380000A002042726F776E206F75742052657359
:1023900065740A002045787465726E616C20526520
:1023A0007365740A00506F77657255700A00737414
:1023B0006172740A006572726F7220777269746953
:1023C0006E6720746F2066696C650A00456E6473E1
:1023D000746F707320256320256320256320256397
:1023E00000205A3A0020593A0020583A00656E649D
:1023F00073746F7073206869743A2000446F6E655F
:1024000020736176696E672066696C652E0A004DDF
:10241000323900290A002062797465733B206372A7
:1024200063200053657474696E67732053746F7210
:102430006564202800202863616C63756C61746595
:102440006429210A0020213D2000454550524F4D6E
:1024500020435243206D69736D61746368202D20A1
:102460002873746F726564292000290A002062793C
:102470007465733B2063726320002073746F726510
:10248000642073657474696E677320726574726911
:1024900065766564202800204D61726C696E3D563A
:1024A0003431290A0028454550524F4D3D004545DD
:1024B00050524F4D2076657273696F6E206D69734F
:1024C0006D61746368200048617264636F64656461
:1024D0002044656661756C742053657474696E6719
:1024E00073204C6F616465640A00F4010000F4011C
:1024F000000064000000E80300000000FA43000050
:10250000FA430000A0400000C8410000A0420000C3
:10251000A0420000C843EC11BF4346696C616D6581
:102520006E7400E0E10046696C616D656E74004C8C
:102530006F61642073657474696E6773004C6F61BA
:1025400064206D656D6F7279004C6F6164207365F6
:102550007474696E677300496E697469616C697A35
:102560006520454550524F4D00496E697469616C54
:10257000697A6520454550524F4D00496E6974692E
:10258000616C697A6520454550524F4D00456E6734
:102590006C69736800456E676C69736800456E67A7
:1025A0006C697368004368696E65736500436869A8
:1025B0006E657365004368696E657365005072658A
:1025C0006865617420504C4120636F6E66005072E4
:1025D000656865617420504C4120BEBF0050726533
:1025E0006865617420504C4120636F6E66005072C4
:1025F00065686561742041425320636F6E660050C8
:102600007265686561742041425320BEBF005072FC
:1026100065686561742041425320636F6E660054A3
:10262000656D706572617475726500C9D20054651C
:102630006D70657261747572650053746F72652098
:1026400073657474696E67730053746F7265206D7F
:10265000656D6F72790053746F7265207365747461
:10266000696E67730048656174696E6720666169A9
:102670006C65640048656174696E67206661696CA9
:1026800065640048656174696E67206661696C65A0
:1026900064004D696E696D756D2054656D702069BB
:1026A000732020313730004D696E696D756D20548F
:1026B000656D702069732020313730004D696E6977
:1026C0006D756D2054656D70206973202031373031
:1026D000004261636B004261636B004261636B00A7
:1026E000524553554D45204F5054494F4E533A0093
:1026F000524553554D45204F5054494F4E533A0083
:10270000524553554D45204F5054494F4E533A0072
:10271000526573756D65207072696E7400526573D1
:10272000756D65207072696E7400526573756D65A4
:10273000207072696E740045787472756465206DDE
:102740006F72650045787472756465206D6F72658F
:102750000045787472756465206D6F726500507203
:1027600065686561742041425320456E6400507273
:1027700065686561742041425320456E6400507263
:1027800065686561742041425320456E6400507253
:10279000656865617420414253204265640050724F
:1027A00065686561742041425320C4C7005072655A
:1027B00068656174204142532042656400473238A5
:1027C000004175746F20686F6D6500BBBCBD004132
:1027D00075746F20686F6D65004D34323800536535
:1027E0007420686F6D65206F66667365747300BED4
:1027F000BFBBBCBDC0C10053657420686F6D652050
:102800006F6666736574730044697361626C6520FA
:10281000737465707065727300B5B6B7B8B9BA00F5
:1028200044697361626C652073746570706572735E
:10283000004368616E67652066696C616D656E74E2
:10284000004368616E67652066696C616D656E74D2
:10285000004368616E67652066696C616D656E74C2
:1028600000436F6F6C646F776E00C8C900436F6F71
:102870006C646F776E005072656865617420504CAF
:102880004100C3C420504C410050726568656174BA
:1028900020504C410050726568656174204142537C
:1028A00000C3C420414253005072656865617420C2
:1028B000414253004D3834004D6F76652061786990
:1028C0007300C1B2CE004D6F7665206178697300E8
:1028D0004D6F76652031306D6D00C1B22031306DA5
:1028E0006D004D6F76652031306D6D004D6F7665F2
:1028F00020316D6D00C1B220316D6D004D6F766578
:1029000020316D6D004D6F766520302E316D6D007C
:10291000C1B220302E316D6D004D6F766520302EA6
:10292000316D6D0070012C0190012701B001220171
:10293000C0011D01F00118011002130130020E0147
:102940006002090190020401C002FF000003FA00C6
:102950004003F5008003F000D003EB002004E60004
:102960007004E100E004DC004005D700C005D2009F
:102970004006CD00D006C8008007C3003008BE0066
:10298000F008B900C009B400B00AAF00B00BAA004B
:10299000D00CA500000EA000500F9B00C0109600A8
:1029A0005012910000148C00C0158700B0178200EF
:1029B000B0197D00D01B7800001E730040206E000F
:1029C00090226900F024640040275F0090295A009B
:1029D000E02B5500102E500020304B0010324600E6
:1029E000E033410090353C0010373700703832003A
:1029F000A0392D00B03A2800A03B2300603C1E0007
:102A0000103D1900903D1400103E0F00703E0A006A
:102A1000C03E0500003F0000403FFBFF803FF6FF47
:102A2000C03FF1FF544845524D414C2052554E4154
:102A300057415900546865726D616C2052756E6122
:102A4000776179004572723A204D494E54454D5098
:102A500020424544004572723A204D494E54454D3E
:102A600050004D494E54454D50207472696767655A
:102A7000726564004572723A204D415854454D507C
:102A800020424544004572723A204D415854454D0C
:102A900050004D415854454D502074726967676528
:102AA000726564004D61696E00AEAFB0004D616942
:102AB0006E004D6F7665205800C1B22058004D6FF2
:102AC00076652058004D6F7665205900C1B22059B7
:102AD000004D6F76652059004D6F7665205A00C114
:102AE000B2205A004D6F7665205A00457874727591
:102AF00064657200CCADBA00457874727564657215
:102B0000004E6F7A7A6C6500D3D4004E6F7A7A6C7F
:102B1000650042656400C4C7004265640046616E9A
:102B200020737065656400D5D6D1D20046616E20F1
:102B3000737065656400436F6E74726F6C00D8D9F2
:102B400000436F6E74726F6C004D6F74696F6E002E
:102B5000DFB2004D6F74696F6E0050726570617204
:102B60006500A4A5005072657061726500526573BE
:102B7000756D65207072696E7400F4F5CAF30052C9
:102B80006573756D65207072696E740053746F7033
:102B9000207072696E7400F2F6CAF30053746F709D
:102BA000207072696E74005052494E542050415545
:102BB000534544005052494E5420504155534544CA
:102BC000005052494E542050415553454400202056
:102BD0004E6F7A7A6C653A200020204E6F7A7A6CBC
:102BE000653A200020204E6F7A7A6C653A2000000A
:102BF000060900FE000000000001090008FE0000B8
:102C000005080806000040F0C88888987810050874
:102C100008060000C0F88888888888F80505050639
:102C200000012030F830200508080600002070F868
:102C300020202020E00509090600FF2070A8A8B880
:102C4000888870200509090600FFE080C0B0A82828
:102C50003028280509090600FFF8A8888888888890
:102C6000A8F8050A0A0600FE205050505088A8A86F
:102C7000887003030306000340A040436172642090
:102C8000696E73657274656400A8A9AAAB0043619C
:102C9000726420696E736572746564004361726466
:102CA0002072656D6F76656400A8A9ACAD004361C4
:102CB00072642072656D6F766564004D6F76696E23
:102CC000672E2E2E004572723A204368616E67654A
:102CD0002046696C616D656E74005072696E742077
:102CE000706175736564004572723A204368616E65
:102CF00067652046696C616D656E74007C3C3E5E64
:102D00002B3D3F2F5B5D3B2C2A225C00506C6561A4
:102D10007365207265736574005052494E54455274
:102D20002048414C544544005072696E74657220CD
:102D300068616C7465642E206B696C6C2829206353
:102D4000616C6C6564210A0062696E004D31313737
:102D500020494E56414C494420444154412E00479D
:102D60003932205A2573204525730062696E0000B0
:102D700000000000000000000000000000484200C9
:102D800000484200008040000000005761726E69F8
:102D90006E673A20486F6D696E672042756D7020CE
:102DA00044697669736F72203C20310A0002020484
:102DB0000000A0400000A0400000004000009B4335
:102DC00000009B430000CD43FFFFFF000C0B00FE03
:102DD000070192032120FFFF0AFF07FF0000000602
:102DE000000A0107070602008080808080008003BF
:102DF0000202060105A0A00507070600005050F8D2
:102E000050F850500507070600002078A07028F001
:102E100020050707060000C0C810204098180507C5
:102E2000070600006090A040A89068020303060116
:102E300004C04080030707060100204080808040D6
:102E40002003070706010080402020204080050560
:102E50000506000120A870A8200505050600012030
:102E600020F820200203030602FFC0408005010174
:102E7000060003F8020202060200C0C005050506AE
:102E800000010810204080050707060000708898A0
:102E9000A8C8887003070706010040C040404040B2
:102EA000E0050707060000708808708080F80507B5
:102EB00007060000F81020100808F00507070600B4
:102EC0000010305090F81010050707060000F88039
:102ED000F008088870050707060000708080F088F9
:102EE0008870050707060000F8081020202020053C
:102EF0000707060000708888708888700507070635
:102F0000000070888878080870020505060200C075
:102F1000C000C0C00206060602FFC0C000C040805C
:102F2000040707060000102040804020100503031E
:102F3000060002F800F80407070600008040201091
:102F40002040800507070600007088081020002038
:102F500005070706000070880868A8A8700507071D
:102F6000060000708888F888888805070706000032
:102F7000F08888F08888F0050707060000708880D0
:102F800080808870050707060000F0888888888898
:102F9000F0050707060000F88080F08080F805073C
:102FA00007060000F88080F0808080050707060093
:102FB00000708880B8888870050707060000888838
:102FC00088F8888888010707060200808080808052
:102FD000808005070706000038101010109060056B
:102FE00007070600008890A0C0A090880507070684
:102FF0000000808080808080F80507070600008838
:10300000D8A8888888880507070600008888C8A887
:103010009888880507070600007088888888887067
:10302000050707060000F08888F080808005070704
:1030300006000070888888A89068050707060000C9
:10304000F08888F0A0908805070706000078808047
:10305000700808F0050707060000F820202020204F
:10306000200507070600008888888888887005077B
:103070000706000088888888885020050707060012
:10308000008888888888A850050707060000888877
:10309000502050888805070706000088888850203F
:1030A0002020050707060000F80810204080F803DC
:1030B0000707060000E08080808080E005050506A7
:1030C00000018040201008030707060000E02020D0
:1030D000202020E00503030600042050880501019C
:1030E000060000F8020202060205804005050506FA
:1030F000000070087888780507070600008080B017
:10310000C88888F005050506000070808088700575
:1031100007070600000808689888887805050506EE
:1031200000007088F880700507070600003048E04E
:10313000404040400506060600FF70888878087009
:103140000507070600008080B0C888888801070747
:10315000060200800080808080800308080601FF4E
:10316000200020202020A0400407070601008080C6
:1031700090A0C0A090030707060100C04040404057
:1031800040E0050505060000D0A8A8A8A80505058B
:10319000060000B0C888888805050506000070880C
:1031A0008888700506060600FFF08888F080800594
:1031B00006060600FF7888887808080505050600D9
:1031C00000B0C8808080050505060000708070088A
:1031D000F00407070600004040E04040403005058D
:1031E000050600008888889868050505060000889F
:1031F000888850200505050600008888A8A8500585
:10320000050506000088502050880506060600FFC8
:10321000888888780870050505060000F8102040A9
:10322000F8030707060100204040804040200107C6
:1032300007060200808080808080800307070601E7
:103240000080404020404080050202060003689054
:1032500000000006000A0000000C000A0000000C3C
:10326000000A0000000C000A0000000C000A000028
:10327000000C000A0000000C000A0000000C000A0C
:103280000000000C000A0000000C000A0000000C06
:10329000000A0000000C000A0000000C000A0000F8
:1032A000000C000A0000000C000A0000000C000ADC
:1032B0000000000C000A0000000C000A0000000CD6
:1032C000000A0000000C000A0000000C000A0000C8
:1032D000000C000A0000000C000A0000000C000AAC
:1032E0000000000C000A0000000C000A0000000CA6
:1032F000000A0000000C000A0000000C000A000098
:10330000000C000A0B0B160C00FFFFE0020002008D
:1033100004000D0014802440C420040004000400B4
:103320000B0B160C00FFF9008A00ABE0AC40AA4082
:10333000AA40AA40AA80210052808C600B0B160C78
:1033400000FF240024003F80440084000400FFE0CC
:103350000A0011002080C0600B0B160C00FF240037
:1033600024003FC044000400FFE0090009001120D0
:10337000212040E00B0B160C00FF20003DE0512007
:1033800091201120FF201120292025E045208000D8
:103390000B0B160C00FF20807FC00840FFE01100DF
:1033A00020805F4080203F8000007FC00B0B160C08
:1033B00000FF224047E09480E4802FE04480F480C6
:1033C00007E03480C48007E00B0B160C00FF04807C
:1033D0008FE0490019002FC0090009002FC04900E3
:1033E00089000FE00B0B160C00FF10003F8051000E
:1033F0000E003180C0603F8024803F8024803F8069
:103400000B0B160C00FF2280FA4007E0FA808A803E
:103410008A80FA802280B280AAA064E00B0B160C8E
:1034200000FF222047409280EFE0220047C0EC409E
:1034300007C03440C7C004400B0B160C00FF080047
:103440000FC008000800FFE008000E0009800840D7
:10345000080008000A0B160C00FFFF8000800080A7
:1034600080808080FF8080008000804080407FC01E
:103470000B0B160C00FF47C04100EFE04100450078
:103480006960C9204D6049204FE0C8200B0B160C25
:1034900000FF0800040004000A000A000A001100EE
:1034A00011002080404080200B0B160C00FF2240B2
:1034B0002200F7E0220023E03520E5202540288087
:1034C000294072200B0A140C000044404440444040
:1034D0007FC004000400842084208420FFE00B0BC4
:1034E000160C00FF040000007FC00400040004006C
:1034F0007FC0040004000400FFE00B0B160C00FF6B
:10350000FFE0110001C0FE00488025000400FFE03C
:1035100015002480C4600B0B160C00FF11007FC047
:1035200044407FC044407FC00400FFE0040004002A
:103530000400090B160C00FF1000FF8080808080C3
:10354000FF8080808080FF8080808080FF800B0BE8
:10355000160C00FF7100010003E0F920212041203A
:1035600051208920FA20022004C00B0B160C00FF0A
:103570007FC01100110011001100FFE011001100C7
:103580002100210041000B0B160C00FF210022003E
:10359000F44057E0502057C094405440244057C056
:1035A00094400B0B160C00FF11000A007FC00400B2
:1035B0000400FFE004000A0011002080C0600A0B34
:1035C000160C00FF5FC0004084408440BF40844030
:1035D0008C409440A4408C4081C00B0B160C00FF23
:1035E000240027C024002400FFE0000014402480B1
:1035F00047000C0070000B0B160C00FF24800480A9
:103600000FC0E48024803FE0248024802880500084
:103610008FE00B0B160C00FF08000800FF8088806D
:103620008880FF8088808880FFA0882007E00B0BBF
:10363000160C00FF27802480F480248074806C8026
:10364000A480248024A028A030600A0B160C00FF60
:10365000FFC0804080409E40924092409E4080400B
:103660008040FFC080400B0B160C00FF7FC0440061
:103670005FC050405FC050405FC042004A8052402F
:10368000A6200B0B160C00FF040007E004007FC00F
:103690004040404040407FC00000524089200B0B1A
:1036A000160C00FF4780248004800480E86020001E
:1036B0002FC024402280310026C00B0B160C00FFC7
:1036C0007FC04A407FC00400FFE004003F802080AC
:1036D00024802480FFE00B0B160C00FF22004FE03B
:1036E00048204FE0C8004FE04AA05AA06FE04AA02F
:1036F00048600B0B160C00FFF3C024402A80F10039
:10370000228065E07220A540208023002C000B0B56
:10371000160C00FF0400FFE080200000FFE0040022
:10372000240027C0240054008FE00B0B160C00FF70
:1037300073E01080510023E0FA202AA022A022A0EA
:103740002080214062200B0B160C00FF2200F78026
:1037500022803680E2A025A024606820000052402C
:1037600089200B0B160C00FF73C0420042007BE067
:103770004A404A407A404A404240444088400B0B0D
:10378000160C00FF0800FFE008001FC030405FC0BB
:1037900090401FC01040104010C00B0B160C00FFD3
:1037A00002007FE0420042005FC0420047004A80C2
:1037B0005240622082000B0B160C00FFF3C09640B3
:1037C0009180A660A10097C091009500E7E081007C
:1037D00081000B0B160C00FF0F8088804F80088043
:1037E0008F8040001FC03540554095403FE00B0B97
:1037F000160C00FF27E02080F88020802080388091
:10380000E08020802080208061800B0B160C00FF60
:103810001FE0910057C0144017C0944057C01100DA
:103820005540992023000B0B160C00FF208027E049
:10383000F240218022403420E240224022402240B7
:1038400064400B0B160C00FF410041004FE0E920E3
:10385000492049206FE0C92049204920CFE00B0BC7
:10386000160C00FF2100F1004FE0A920F9202FE005
:103870003920E92029202FE028200B0B160C00FF0F
:103880008FE049200920CBA049204FE048204BA0E1
:103890004AA06BA050E00B0B160C00FF7FC0040089
:1038A0004440244024800400FFE00400040004009D
:1038B00004000B0B160C00FF820042001FE0C20048
:1038C0005FC052405FC047004A805240BFE00B0BD0
:1038D000160C00FF04007FE048807FE048804F80A6
:1038E00040005FC04840478098600B0B160C00FFFB
:1038F0000100EFE0A100A440AFE0A440AFE0A920A8
:10390000E92002800C600B0B160C00FF14C0F6A01F
:10391000BC60A780A880BFE0A920EFE009200FE0ED
:1039200009200B0B160C00FF7F80408042806280D4
:1039300054804880488054A062A0406080200B0BD7
:10394000160C00FF04007FE040207FE040007DE097
:1039500054204CA0546064A08D600B0B160C00FF2B
:1039600082005FE0040008409FE040200A800A8057
:103970004AA092A022600B0B160C00FF41004FE002
:10398000E820428044406820C7C041004100410017
:10399000CFE00B0B160C00FF50207D209120FF2064
:1039A00011207D205520552054205C2010E00B0B69
:1039B000160C00FF3F8020803F802080FFE0480001
:1039C0007BC0494079404880FB600B0B160C00FF20
:1039D0000400040004002480244044404420842047
:1039E000040004001C000B0B160C00FF0400040074
:1039F0000400FFE004000A000A001100110020800A
:103A0000C060090A140A0000888049000800FF808D
:103A1000008000807F8000800080FF800B0B160CF0
:103A200000FF21001200FFE0000078804A807A80C9
:103A30004A807A80488059800B0B160C00FF27C003
:103A400000000000EFE02100220024402FE02020B1
:103A500050008FE00B0B160C00FF20802700F900B0
:103A600021C077002100F9E027007120A92020E083
:103A70000B0B160C00FF10401040FDE0104038C04A
:103A80003540524094401040104010C00B0B160CB3
:103A900000FF0040F8400BE0084088405240514091
:103AA00021405040484089C00A0B160C00FF84009A
:103AB00084408480F5008600840084009400A44043
:103AC000C44083C00B0B160C00FF11207D001100B9
:103AD000FFE02900FD4049407C8008A0FD600A20ED
:103AE0000B0B160C00FF17C02440244067C0A10038
:103AF0002FE0210023802540292021000B0B160CEC
:103B000000FF0800FFE0100027C020806100AFE048
:103B100021002100210023000B0B160C00FF2400C4
:103B20002FE0B400A480A4A0AAC02A802880294045
:103B3000324024200B0B160C00FF7FE080003FC0BA
:103B400020403FC010001FC010402880470038E0D0
:103B50000B0B160C00FF7FE04000400040004000CF
:103B60004000400040004000400080000B0B160C5D
:103B700000FFFFE004007FC044407FC044407FC09E
:103B8000440024001800E7E00B0B160C00FF11E0C6
:103B9000FD00450029E0FD4011407D4011405540A9
:103BA000924034400B0B160C00FF21005FE04000F8
:103BB000CFC040004FC040004FC048404FC04840B9
:103BC0000B0B160C00FF04007FC040407FC040403C
:103BD0007FC040407FC004405220BFA00B0B160C9A
:103BE00000FF7FC044407FC044407FC004001B00F2
:103BF000E0E01100110061000B0B160C00FFFFE06C
:103C0000040008007FE049204F2049204F20492030
:103C100049207FE00B0B160C00FFFDE05640794079
:103C2000388055409220FFE0040027C02400FFE0C8
:103C30000B0B160C00FFFB8052007BE01240FA4099
:103C400014403F8020803F8020803F800B0B160C6B
:103C500000FF1FE0200027C06440A7C020002FE025
:103C6000282027C0210023000B0B160C00FFF3E0D7
:103C700082208220FA20822082208A20B220C2E084
:103C8000020002000B0B160C00FF248046A095C01A
:103C9000E48027E04480F5C006A03480C48007E0BB
:103CA0000B0B160C00FF27C0410087E0E0202280AC
:103CB0004580F2800FE03080C14002200B0B160CD3
:103CC00000FF02000200220023C022002200220086
:103CD000220022002200FFE0090B160C00FF080062
:103CE0000800FF80888088808880FF8088808880A6
:103CF0008880FF800B0B160C00FF210053A04100B1
:103D0000F7E0510053C0564053C05A4053C04240A0
:103D10000B0B160C00FF7FC0040004000400FFE042
:103D20000A000A0012002220422081E00B0B160C30
:103D300000FF110021002FE06100A38023802540B7
:103D400025402920210021000B0B160C00FFF7E075
:103D50009420F42097E09480F48097E09480F4A07D
:103D6000966004200B0B160C00FF7BE0948004008F
:103D70007FC00400FFE00100FFE021001100070008
:103D80000B0B160C00FF210047C091002FE0608054
:103D9000AFE0208024802280208023800B0B160C33
:103DA00000FF27C02440F7C02EE02AA03EE0E1003B
:103DB0002FE02380254069200B0B160C00FF140018
:103DC00027E02A006200A3C02200220023E0220094
:103DD0002200220000060900FE070192032120FFB5
:103DE000FF08FF07FF0000000600000107070602AA
:103DF0000080808080800080030202060105A0A070
:103E00000507070600005050F850F8505005070706
:103E10000600002078A07028F020050707060000A3
:103E2000C0C810204098180507070600006090A041
:103E300040A89068020303060104C04080030707FE
:103E40000601002040808080402003070706010013
:103E50008040202020408005050506000120A87034
:103E6000A8200505050600012020F82020020303F4
:103E70000602FFC04080050101060003F8020202AD
:103E8000060200C0C005050506000108102040809C
:103E90000507070600007088888888887003070770
:103EA00006010040C040404040E005070706000012
:103EB000708808708080F8050707060000F8102059
:103EC000100808F005070706000010305090F810A1
:103ED00010050707060000F880F00808887005073D
:103EE00007060000708080F08888700507070600CC
:103EF00000F8081020202020050707060000708821
:103F00008870888870050707060000708888780820
:103F10000870020505060200C0C000C0C002060607
:103F20000602FFC0C000C040800407070600001062
:103F3000204080402010050303060002F800F8042A
:103F40000707060100804020102040800507070673
:103F50000000708808102000200507070600007088
:103F6000880868A8A870050707060000708888F808
:103F7000888888050707060000F08888F08888F0A0
:103F80000507070600007088808080887005070795
:103F9000060000F08888888888F00507070600007A
:103FA000F88080F08080F8050707060000F8808020
:103FB000F0808080050707060000708880B8888838
:103FC00070050707060000888888F8888888010738
:103FD0000706020080808080808080050707060039
:103FE0000038101010109060050707060000889038
:103FF000A0C0A09088050707060000808080808010
:1040000080F805070706000088D8A88888888805F2
:1040100007070600008888C8A8988888050707064B
:10402000000070888888888870050707060000F0FF
:104030008888F080808005070706000070888888DF
:10404000A89068050707060000F08888F0A090880F
:10405000050707060000788080700808F00507074C
:10406000060000F820202020202005070706000079
:1040700088888888888870050707060000888888EF
:10408000888850200507070600008888888888A847
:1040900050050707060000888850205088880507CB
:1040A00007060000888888502020200507070600A2
:1040B00000F80810204080F8030707060100E080A0
:1040C00080808080E0050505060001804020100802
:1040D000030707060100E02020202020E00503035D
:1040E000060004205088050101060000F8020202C3
:1040F00006020580400505050600007008788878EE
:104100000507070600008080B0C88888F00505050F
:104110000600007080808870050707060000080808
:1041200068988888780505050600007088F8807012
:104130000507070600003048E040404040050606FD
:104140000600FF7088887808700507070600008061
:1041500080B0C88888880107070602008000808038
:104160008080800308080601FF200020202020A076
:1041700040040707060000808090A0C0A0900307BD
:1041800007060100C04040404040E005050506002C
:1041900000D0A8A8A8A8050505060000B0C8888812
:1041A00088050505060000708888887005060606E3
:1041B00000FFF08888F080800506060600FF7888FA
:1041C00088780808050505060000B0C880808005CD
:1041D000050506000070807008F00407070600005F
:1041E0004040E040404030050505060000888888D2
:1041F0009868050505060000888888502005050593
:104200000600008888A8A85005050506000088500B
:104210002050880506060600FF8888887808700503
:104220000505060000F8102040F803070706010006
:104230002040408040402001070706020080808027
:1042400080808080030707060100804040204040B6
:1042500080050202060002689000000006000000CF
:10426000000006000000000006000000000006003C
:104270000000000006000000000006000000000032
:10428000060000000000060000000000060000001C
:10429000000006000000000006000000000006000C
:1042A0000000000006000000000006000000000002
:1042B00006000000000006000000000006000000EC
:1042C00000000600000000000600000000000600DC
:1042D00000000000060000000000060000000000D2
:1042E00006000000000006000000000006000000BC
:1042F00000000600000000000600000000000600AC
:1043000000000000060000000000060000000000A1
:10431000060000000000060000000000060000008B
:104320000000060000010707060200800080808070
:1043300080800507070600002070A8A0A87020054F
:104340000707060000304040E04050A8050505067C
:10435000000088705070880507070600008850200C
:10436000F820F82001070706020080808000808086
:104370008005080806000030482050502090600357
:104380000101060107A0050707060000F888B8B874
:10439000B888F8050707060001700878887800F8E3
:1043A0000505050600012850A05028050303060056
:1043B00001F8080802020206020640800507070607
:1043C0000000F888A88898A8F8050101060006F8FA
:1043D00004040406000360909060050707060000CF
:1043E0002020F8202000F804050506000360902036
:1043F00040F0030505060003E020E020E002020291
:1044000006020640800508080600FF88888888980C
:10441000E880800507070600007898987818181833
:10442000020202060202C0C00202020602FF40802F
:1044300003050506000340C04040E00507070600ED
:1044400001708888887000F8050505060001A050F5
:104450002850A00507070600008890A858B808084B
:104460000507070600008890B84898203805080816
:10447000060000C040C048D83808080507070600F5
:1044800000200020408088700508080600004020B9
:10449000007088F888880508080600001020007061
:1044A00088F888880508080600002050007088F801
:1044B00088880508080600006890007088F88888D9
:1044C0000508080600005000708888F888880508EC
:1044D000080600002050207088F888880507070625
:1044E00000003860A0B8E0A0B80508080600FF701A
:1044F0008880808870206005080806000040200041
:10450000F880F080F8050808060000081000F88020
:10451000F080F8050808060000205000F880F080C0
:10452000F80507070600005000F880F080F803083F
:1045300008060100804000E0404040E00308080613
:104540000100204000E0404040E003080806010070
:1045500040A000E0404040E0030707060100A00043
:10456000E0404040E0050707060000704848E84882
:10457000487005080806000068900088C8A8988858
:1045800005080806000040207088888888700508A3
:1045900008060000102070888888887005080806C2
:1045A0000000205000708888887005080806000008
:1045B0006890007088888870050808060000500020
:1045C000708888888870050505060001885020508D
:1045D000880508080600FF1070A8A8A8A870400564
:1045E0000808060000402088888888887005080828
:1045F0000600001020888888888870050808060052
:10460000002050008888888870050808060000503F
:1046100000888888888870050808060000102088AF
:1046200050202020200509090600FFC0407048489E
:10463000704040E00408080601FF609090A0909050
:10464000E08005080806000040200070087888789F
:104650000508080600001020007008788878050812
:1046600008060000205000700878887805080806C1
:104670000000689000700878887805070706000039
:10468000500070087888780508080600002050203F
:104690007008788878050606060000D02878A0A85B
:1046A000500506060600FF70808870206005080827
:1046B0000600004020007088F88070050808060099
:1046C000001020007088F88070050808060000209F
:1046D00050007088F88070050707060000500070D1
:1046E00088F8807003080806010080400040C04040
:1046F00040E003080806010020400040C04040E0C0
:1047000003080806010040A00040C04040E0030745
:1047100007060100A00040C04040E0050707060072
:1047200000A040A010788870050808060000689076
:1047300000B0C8888888050808060000402000707E
:104740008888887005080806000010200070888896
:10475000887005080806000020500070888888705E
:1047600005080806000068900070888888700507B2
:10477000070600005000708888887005050506004F
:10478000012000F800200507070600FF1070A8A808
:10479000A870400508080600004020008888889816
:1047A00068050808060000102000888888986805B9
:1047B00008080600002050008888889868050707C8
:1047C000060000500088888898680509090600FFDF
:1047D000102000888888F808700407070601FFC0C9
:1047E0004060506040E00508080600FF50008888DF
:1047F0008878087000002100240027002A002D007E
:104800003000330001010000040107010A01507269
:10481000696E74207061757365640047302046339B
:104820003030302058302059300000473932204590
:104830002573004730205A2573004D3130392053FD
:104840002569004D31343020532569004D31303613
:104850002053323535004730205A2573004732380F
:10486000205830205930004D31303920532569000F
:104870004D31393020532569005072696E742061C2
:10488000626F7274656400506F7765722D4C6F7340
:1048900073205265636F766572793F00A4A5F4F5C5
:1048A000CAF3203F00506F7765722D4C6F737320F1
:1048B0005265636F766572793F00496E666F20734B
:1048C000637265656E00ECEDEEEF00496E666F2079
:1048D00073637265656E0054756E6500CFF00054A9
:1048E000756E65004C616E6775616765004C616E41
:1048F0006775616765004C616E677561676500503B
:1049000061757365207072696E7400F1F2CAF3000C
:104910005061757365207072696E74005072696EB3
:10492000742066726F6D20544600AFB000507269FB
:104930006E742066726F6D205446004E6F20544690
:10494000206361726400F9A8004E6F205446206312
:104950006172640020746F6F206C6F6E67206578E1
:1049600074727573696F6E2070726576656E7465AA
:10497000640A0020636F6C642065787472757369D3
:104980006F6E2070726576656E7465640A00656E80
:104990007175657565696E672022006563686F3A99
:1049A000002E0A006F70656E206661696C65642C6C
:1049B0002046696C653A200057726974696E6720F9
:1049C000746F2066696C653A20004D3630302042A5
:1049D0003000537065656400D1D200537065656422
:1049E00000466C6F7700CCADD1D200466C6F77007B
:1049F0004261627973746570205A00426162797312
:104A0000746570205A004261627973746570205A2F
:104A1000005072656865617420504C4120456E6499
:104A2000005072656865617420504C4120456E6489
:104A3000005072656865617420504C4120456E6479
:104A4000005072656865617420504C412042656475
:104A5000005072656865617420504C4120C4C700E5
:104A60005072656865617420504C41204265640055
:104A70002E0A0046696C652862696E292064656C9F
:104A8000657465640044656C6574696F6E2862695D
:104A90006E29206661696C6564004572726F7220D0
:104AA00077726974696E6720746F20454550524F64
:104AB0004D210A00526573656E643A20006F6B00E9
:104AC00020746F6F206C6F6E6720657874727573D9
:104AD000696F6E2070726576656E7465640A002079
:104AE000636F6C6420657874727573696F6E207083
:104AF000726576656E7465640A00627573793A2032
:104B000070617573656420666F7220696E7075746C
:104B10000A00627573793A20706175736564206666
:104B20006F7220757365720A00627573793A20702E
:104B3000726F63657373696E670A004B494C4C452D
:104B4000442E20004B494C4C2063617573656420F2
:104B50006279204B494C4C20627574746F6E2F70D3
:104B6000696E0A004B494C4C45442E20004B494C81
:104B70004C2063617573656420627920746F6F20C7
:104B80006D75636820696E61637469766520746908
:104B90006D65202D2063757272656E7420636F6D74
:104BA0006D616E643A200000ABF701F611241FBE60
:104BB000CFEFD1E2DEBFCDBF00E00CBF15E0A0E03B
:104BC000B2E0E6E5F3E102E00BBF02C007900D9210
:104BD000A636B107D9F72AE1A6E6B5E001C01D92D5
:104BE000A832B207E1F715E2C5EDD5E200E006C054
:104BF00021970109802FFE010F940D09C43DD107B3
:104C000080E00807A9F70E9479EF0D949A090C94A7
:104C100000002F923F924F925F926F927F928F92FD
:104C20009F92AF92BF92CF92DF92EF92FF920F933B
:104C30001F93CF93DF93CDB7DEB7C056D1090FB620
:104C4000F894DEBF0FBECDBF0091C10F20E6029FDA
:104C5000800111240F5B114F8091CF1580FF1AC086
:104C6000EBE9F9E484917F013FEFE31AF30A811144
:104C700002C0780104C00E944442F701F3CFD7017B
:104C80008D917D01882319F00E944442F8CF8AE07B
:104C90000E94444281E090E09093F7198093F619C6
:104CA00010929105109290058FE3809394051092D5
:104CB00093051092920584E0E0E8F5E0DF011D9293
:104CC0008A95E9F7F80180810F5F1F4F8032D1F399
:104CD0008E34C9F4818190ED980F9A3020F08D3296
:104CE00011F08B3281F4DF0112969D012F5F3F4F4F
:104CF0008C9180538A3010F4D901F7CFFD011196C1
:104D000080818032D9F3F093FF19E093FE197F017F
:104D1000BFEFEB1AFB0A10816AE270E0C7010F9443
:104D20006209009731F0FC01319780818032E1F314
:104D300011821D3431F1143521F1173411F1EBE9F1
:104D4000F9E484918F010F5F1F4F882321F00E94A7
:104D50004442F801F6CF6091FE197091FF198DEF72
:104D600097E00E9466EC82E20E9444428AE00E9440
:104D700044421092F7191092F6190E9483EB0C949A
:104D8000033DC701FC01208101962032D9F3205355
:104D90002A30A8F61093940580E090E06AE03196FE
:104DA000DF0111972C91022E000C330B2053310997
:104DB000689FA001699F500D1124C901840F951FA0
:104DC000208120532A3058F39093930580939205C5
:104DD000DF0131962C912032D9F31D34A9F48E31A4
:104DE0009105D1F03CF487319105B1F08C319105FA
:104DF00059F412C0853791053CF08737910564F06E
:104E0000803AE3E09E0741F00091FE1960E070E017
:104E1000EE24E394F12C43C0B0939105A093900548
:104E20007FC0213209F445C03FEBB32EB20E49E1F9
:104E3000A42EAB1408F45FC0AF01FA0130814F5FBC
:104E40005F4F3032D1F340ED430F4A3008F047C096
:104E5000AF018B2C912C640123E0D594C7942A9543
:104E6000E1F7960120583A4F69012B2D2770D701A1
:104E700002C0AA0FBB1F2A95E2F79D01D6013C9103
:104E8000232B2C9341155105A1F1401BD401AA59A4
:104E9000BA4F4C93208121542A3190F5DF01FD0156
:104EA00031962C912111BDCF70939105609390059F
:104EB00037C01D3409F0B8CF8032910509F0B4CF66
:104EC000F0939105E093900563E270E0CF010F94B9
:104ED0006209009709F4A9C6DC011C9221C043EDC8
:104EE000430F423008F4B4CF3B3211F00C948A3CAB
:104EF000AFCF40E0CBCF6115710561F6BD01CACFE0
:104F0000DF01AD014F5F5F4F2C9120532A3010F429
:104F1000DA01F7CFFD01119620812032D9F3BECFFF
:104F2000809194058D3409F480C6843511F40C9475
:104F30004E3C873409F003CF2090920530909305C2
:104F4000B4E02B16310409F40DC54CF437FC11CF35
:104F500080910602F2E02F16310404F517C02AE50D
:104F60002216310409F4F9C534F44CE12416310455
:104F700009F43DC5FECE5BE52516310409F4F0C504
:104F80008CE52816310409F4EFC5F3CE882309F423
:104F9000F0CE0E94C6410E94A8EAEBCE882309F415
:104FA000E8CE0E94C64182E50E94BA41882309F4F6
:104FB0003CC10E9458414B015C0120E030E0A90156
:104FC0000E9484FF882309F45CC120914E1830911F
:104FD0004F1840915018509151182DA73EA74FA738
:104FE00058AB8091521890915318A0915418B091D9
:104FF000551889AB9AABABABBCAB20914912309141
:105000004A1240914B1250914C1229AF3AAF4BAF1C
:105010005CAF80914D1290914E12A0914F12B091C1
:1050200050128DAB9EABAFABB8AF6DA57EA58FA573
:1050300098A90E9484FF81110DC02DA93EA94FA9F6
:1050400058AD69A97AA98BA99CA90E9484FF8823DD
:1050500009F417C111E092E02916310409F010E0BB
:1050600020E030E0A901C501B4010E9484FF881F3F
:105070008827881F181759F020E030E040E85FEBE0
:1050800029962CAF3DAF4EAF5FAF29970AC080E0A5
:1050900090E0A0E8BFE329968CAF9DAFAEAFBFAF65
:1050A00029972DA53EA54FA558A969AD7AAD8BAD21
:1050B0009CAD0F941D0625966CAF7DAF8EAF9FAF54
:1050C000259729A93AA94BA95CA96DA97EA98FA901
:1050D00098AD0F941D066B017C0125962CAD3DAD5E
:1050E0004EAD5FAD2597CA01B9010E94E9FF2B01C2
:1050F0003C01A7019601C701B6010E94E9FF9B018F
:10510000AC01C301B2010F941E060F948A082196C8
:105110006CAF7DAF8EAF9FAF219720E030E040E0D5
:105120005FE30E94E9FF2B013C01A5019401C50149
:10513000B4010E94E9FF4B015C01A3019201C3018C
:10514000B2010E94E9FF9B01AC01C501B4010F94BB
:105150001D060F948A0829962CAD3DAD4EAD5FAD6E
:1051600029970E94E9FF4B015C01C701B6019058E5
:1051700021962CAD3DAD4EAD5FAD21970F94FA0653
:10518000A50194010E94E9FF6B017C0129AD3AADB4
:105190004BAD5CAD6DA57EA58FA598A90F941E069D
:1051A00020E030E040E05FE30E94E9FF9B01AC01BA
:1051B000C701B6010F941E062DA53EA54FA558A9FF
:1051C0000F941D066B017C012DA93EA94FA958AD76
:1051D00069A97AA98BA99CA90F941E0620E030E04A
:1051E00040E05FE30E94E9FF2B013C0121962CADDA
:1051F0003DAD4EAD5FAD219725966CAD7DAD8EADCD
:105200009FAD25970F94FA06A50194010E94E9FF2E
:105210009B01AC01C301B2010F941E0629A93AA952
:105220004BA95CA90F941D0614C089E40E94BA41E1
:10523000882329F00E9458416B017C0103C0C12CD6
:10524000D12C76018AE40E94BA418823E9F00E94B9
:10525000584169AF7AAF8BAF9CAF20E030E0A90135
:10526000C701B6010E9484FF81111BC020E030E01D
:10527000A90169AD7AAD8BAD9CAD0E9484FF81110F
:1052800010C0E9ECF6E15BC320E030E0A901C70102
:10529000B6010E9484FF8823A1F319AE1AAE1BAE9B
:1052A0001CAEA701960150582DA73EA74FA758AB9B
:1052B00089AD9AADABADBCADB05889AB9AABABABD9
:1052C000BCABCA01B9010E94E9FF4B015C0129A9ED
:1052D0003AA94BA95CA9CA01B9010E94E9FF9B0147
:1052E000AC01C501B4010F941E060F948A0865969F
:1052F0006CAF7DAF8EAF9FAF659720914E18309108
:105300004F1840915018509151182DAB3EAB4FABF8
:1053100058AFA70196016DA97EA98FA998AD0F94EA
:105320001E0629966CAF7DAF8EAF9FAF29978091F7
:10533000521890915318A0915418B0915518219675
:105340008CAF9DAFAEAFBFAF219729AD3AAD4BAD9E
:105350005CADBC01CD010F941E0669966CAF7DAFAC
:105360008EAF9FAF69972091491230914A124091B8
:105370004B1250914C122D962CAF3DAF4EAF5FAFFC
:105380002D9729962CAD3DAD4EAD5FAD29972D964D
:105390006CAD7DAD8EAD9FAD2D970F941D066B014D
:1053A0007C0180914D1290914E12A0914F12B091BC
:1053B000501261968CAF9DAFAEAFBFAF619769964B
:1053C0002CAD3DAD4EAD5FAD6997BC01CD010F94E5
:1053D0001D064B015C0120915618309157184091E1
:1053E0005818509159186D962CAF3DAF4EAF5FAF26
:1053F0006D97609151127091521280915312909159
:1054000054120F941D0625966CAF7DAF8EAF9FAFE3
:105410002597A70196016DA57EA58FA598A90E9445
:10542000E9FF2B013C01A501940169A97AA98BA987
:105430009CA90E94E9FF9B01AC01C301B2010F943A
:105440001E062B013C01A50194016DA57EA58FA52B
:1054500098A90E94E9FF4B015C01A701960169A987
:105460007AA98BA99CA90E94E9FF9B01AC01C50107
:10547000B4010F941D06A30192010F9491066B01D4
:105480007C0120E030E0A9010E9484FF87FF0AC070
:105490002BED3FE049EC50E4C701B6010F941E0626
:1054A0006B017C0132E02316310451F42BED3FE017
:1054B00049EC50E4C701B6010F941D066B017C0155
:1054C00020E030E0A901C701B6010E9484FF8111EC
:1054D00026C02D962CAD3DAD4EAD5FAD2D976DA97F
:1054E0007EA98FA998AD0E9484FF811118C0619692
:1054F0002CAD3DAD4EAD5FAD619721966CAD7DADF0
:105500008EAD9FAD21970E9484FF811108C01BEDD5
:10551000C12E1FE0D12E19ECE12E10E4F12EA701CF
:10552000960165966CAD7DAD8EAD9FAD65970E9481
:10553000E9FF9B01AC010E94E9FF4B015C0125964C
:105540002CAD3DAD4EAD5FAD2597CA01B9010E94AE
:10555000E9FF9B01AC01C501B4010F941E060F9435
:105560008A084B015C012FE632E143E85AE30E94CE
:1055700084FF87FDDEC1C501B4010F9493070F942A
:1055800067077EAF6DAF672B21F421E030E03EAFBF
:105590002DAF40905A1850905B1860905C18709036
:1055A0005D18ADACBEACB50180E090E00E9488FF14
:1055B0004B015C019B01AC01C701B6010F94FA06D7
:1055C0006DAB7EAB8FAB98AFA501940125966CAD0A
:1055D0007DAD8EAD9FAD25970F94FA0665966CAFA5
:1055E0007DAF8EAF9FAF6597A30192016091551279
:1055F0007091561280915712909158120F941D0677
:10560000A50194010F94FA06A1966CAF7DAF8EAF01
:105610009FAFA1972DA93EA94FA958ADCA01B901C5
:105620000E94E9FF20E030E040E05FE30E94E9FFF4
:105630009B01AC0160E070E080E89FE30F941D06E1
:1056400025966CAF7DAF8EAF9FAF25976D962CAD35
:105650003DAD4EAD5FAD6D9729873A874B875C872F
:105660004D865E866F86788A6091700270917102B5
:10567000072E000C880B990B0E948AFF20910D02C7
:1056800030910E0240910F02509110020E94E9FFEA
:105690002AE037ED43E25CE30E94E9FF2D966CAF10
:1056A0007DAF8EAF9FAF2D970E9486C29B01AC014C
:1056B00028533F4F4F4F5F4F61962CAF3DAF4EAFDA
:1056C0005FAF61974DA45EA46FA478A822242394B1
:1056D000312CB9E1DB2EADACBEACA214B30409F49D
:1056E00014C10E94D9710E9486C2DC01CB0161966F
:1056F0002CAD3DAD4EAD5FAD6197821B930BA40BFE
:10570000B50BB7FD11C00E9486C29B01AC012853A6
:105710003F4F4F4F5F4F61962CAF3DAF4EAF5FAFE6
:10572000619780E00E94F6E7DA94DD2009F441C039
:1057300029A93AA94BA95CA925966CAD7DAD8EAD82
:105740009FAD25970E94E9FF4B015C019201A301E7
:105750006DA97EA98FA998AD0E94E9FFA5019401CA
:105760000F941E067B018C019201A30125966CAD5E
:105770007DAD8EAD9FAD25970E94E9FF4B015C0189
:1057800029A93AA94BA95CA96DA97EA98FA998ADB1
:105790000E94E9FF9B01AC01C501B4010F941D06F5
:1057A0002B013C01C701D80189AB9AABABABBCABB9
:1057B0004DC0B10180E090E00E9488FF2DA93EA974
:1057C0004FA958AD0E94E9FF4B015C010F94F70609
:1057D0006B017C01C501B4010F9480084B015C0191
:1057E000A70196016DA57EA58FA598A90E94E9FF46
:1057F0002B013C0129AD3AAD4BAD5CADC501B40107
:105800000E94E9FFA30192010F941E062B013C01A7
:10581000A50194016DA57EA58FA598A90E94E9FF19
:105820004B015C0129AD3AAD4BAD5CADC701B60192
:105830000E94E9FF9B01AC01C501B4010F941D0654
:1058400069AB7AAB8BAB9CABF9E1DF2E9201A30184
:1058500029966CAD7DAD8EAD9FAD29970F941E0638
:1058600069837A838B839C8329A93AA94BA95CA974
:1058700069966CAD7DAD8EAD9FAD69970F941E0698
:105880006D837E838F83988765962CAD3DAD4EAD3D
:105890005FAD659769857A858B859C850F941E061B
:1058A00069877A878B879C87A1962CAD3DAD4EADDD
:1058B0005FADA1976D857E858F8598890F941E06B3
:1058C0006D877E878F87988B80911D02882321F0BA
:1058D000CE0101960E94DFBBC09018062D96ECAC5D
:1058E000FDAC0EAD1FAD2D979E01235F3F4FAE0166
:1058F000475F5F4FBE016B5F7F4FCE0101960E94F5
:10590000CECA3FEF231A330AE6CEC09018062D9672
:10591000ECACFDAC0EAD1FAD2D9725E532E141E5B8
:1059200052E16DE472E189E492E10E94CECA0E94E4
:10593000873F0E9439421DCA0E944442F801849167
:105940008F010F5F1F4F8111F7CFEBE3F3E08491DD
:105950008F010F5F1F4F882309F40BCA0E94444236
:10596000F801F5CF80E50E94BA41882329F00E9412
:1059700018416B017C0103C0C12CD12C760183E559
:105980000E94BA41882361F00E94584120E030E033
:105990004AE754E40E94E9FF0F9467076B017C011A
:1059A0000E94767580912B02811105C060E081E52F
:1059B00093E00E943FC70E94394280911D0E909152
:1059C0001E0EA0911F0EB091200EC80ED91EEA1E09
:1059D000FB1E0E9486C2DC01CB018C199D09AE0919
:1059E000BF09B7FFC6C980E00E94F6E7F2CF0E9468
:1059F000767580910D0290910E02A0910F02B091E8
:105A0000100280938C0590938D05A0938E05B09322
:105A10008F05809170029091710290938B05809315
:105A20008A0584E690E090937102809370020E9450
:105A3000394281E08093090E88E50E948B41E82E6F
:105A400089E50E948B41082F8AE50E948B41F82E40
:105A5000E11005C0011105C011E0182705C00111B2
:105A600002C010E001C0182F0E947D3F111105C037
:105A7000E11003C0002309F444C020E030E040EA14
:105A800050E46091391270913A1280913B129091DA
:105A90003C120F941E066093511270935212809321
:105AA00053129093541220915618309157184091E8
:105AB0005818509159180F94440818167CF41982FC
:105AC0001A821B821C829E012F5F3F4F41E552E1EB
:105AD00062E578E18EE498E10E948E3E111105C0E6
:105AE000E11003C0011107C00CC080E090E00E94EB
:105AF00071BC1123B9F381E090E00E9471BC1111D7
:105B000002C0FF2021F082E090E00E9471BC0E9460
:105B1000B1408091C40F8093090E80918C059091C3
:105B20008D05A0918E05B0918F0580930D02909305
:105B30000E02A0930F02B093100280918A059091FB
:105B40008B0590937102809370020E94394283E02A
:105B500080932A020E94CC580CC91092890509C969
:105B600081E08093890505C985E40E94BA41B82E79
:105B7000811102C00E94767567E9862E62E0962E3A
:105B80007EE4C72E78E1D72EEDE3EE2EE2E1FE2E85
:105B900000E010E0A12C33243394D4018D914D0109
:105BA0000E94BA41882359F1F601408051806280F9
:105BB00073800E945841D6016D937D938D939C9381
:105BC00013970330E1F0023011F430920C0EA30170
:105BD00092010F941D069B01AC01F7016081718158
:105BE000828193810F941E06D7016D937D938D93CF
:105BF0009C931397C8010E94AA3FAA24A3940F5F05
:105C00001F4FB4E0CB0ED11CE4E0EE0EF11C0430CB
:105C1000110519F6AA2019F00E94B14003C0B11075
:105C20000E9430E00E94CC58A4C8809192059091C7
:105C300093058237910509F4A9C70CF0D5C08B34C0
:105C4000910509F424C50CF05DC08831910509F473
:105C500081C2BCF58231910509F4CAC6D4F497FD1E
:105C600088C8823091050CF494C1419709F081C82D
:105C700060E08CE893E00E943FC75F988A989FB7E6
:105C8000F894809108018E7F809308019FBF12983D
:105C900070C88531910509F444C234F4449709F081
:105CA00068C8E4EAF3E0FDC18631910509F43FC21A
:105CB000479709F05EC88091900590919105FC018D
:105CC00040C28C31910509F4AEC25CF48A31910571
:105CD00009F44DC20CF06AC210921F130E9416E024
:105CE00048C88F31910509F4DBC324F44E9709F4B9
:105CF000A4C23FC88032910509F488C38A9709F489
:105D000085C437C88836910509F4CDC40CF044C069
:105D10008235910509F463C634F58D34910509F493
:105D2000BEC40CF4B8C48135910509F022C80E94A4
:105D30005AA80E9476750E9498EA1092EC1510926B
:105D4000EB150E94AEE0109239101092381068EEF8
:105D500073E080E090E00E9423C660E08EEA94E069
:105D60000E943FC706C88435910509F441C60CF46A
:105D70003AC68535910509F46EC68C35910511F04A
:105D80000C94B92627E9C22E22E0D22E3EE5E32E5E
:105D900038E1F32E10E07AC68D36910509F4EAC594
:105DA0009CF48A36910509F4E9C50CF49DC58B363F
:105DB000910509F402C68C36910511F00C94B926B0
:105DC000109229020C94B9268F36910509F4CAC4A1
:105DD0000CF4B5C48037910509F437C581379105B6
:105DE00009F437C50C94B9268C3D910511F40C9437
:105DF0004B390CF056C08B39910509F492C51CF54E
:105E00008737910509F497C774F48537910509F42C
:105E100052C70CF059C78337910511F00C94B9267D
:105E2000E7E9F5E0BCC68937910509F48FC70CF4A2
:105E300086C78C38910509F439C58139910509F473
:105E40008BC70C94B9268B3C910511F40C949F37A9
:105E500094F4883C910509F4FAC7893C910511F442
:105E60000C947B378E3B910511F00C94B9260E945F
:105E70005C5E0C94B9268D3C910511F40C94283885
:105E800014F40C94BC378E3C910511F40C949538A5
:105E9000833D910511F00C94B926EBE9F9E40C94DB
:105EA000B3388039F1E09F0711F40C94283B8CF54E
:105EB0008D3231E0930711F40C94C93994F4823E89
:105EC000910511F40C9474398C3251E0950711F45A
:105ED0000C94A1398D3D910511F00C94B9260C94C8
:105EE00059398F32A1E09A0711F40C94243B14F431
:105EF0000C94D33A8033E1E09E0711F40C945D3AA0
:105F00008336914011F00C94B926E9ECF6E10C943B
:105F1000293C863F21E0920711F40C94123CFCF4DA
:105F20008C3A41E0940711F40C942C3B4CF48A39E0
:105F3000914011F00C94B9260E9473580C94B92624
:105F4000843FB1E09B0711F40C940E3C853F9140D7
:105F500011F00C94B9260E94E0840C94B92688357F
:105F6000F2E09F0711F40C94233C3CF4873F9140EE
:105F700011F40C94163C0C94B926803A43E0940733
:105F800009F481C2873E934011F40C943C3C0C947C
:105F9000B926A0909005B090910580E50E94BA4185
:105FA000882359F00E9418416B017C0111E0672B96
:105FB000682B692B31F410E004C010E0C12CD12C07
:105FC000760183E50E94BA418823F1F00E9458418E
:105FD00020E030E04AE754E40E94E9FF0F946707AD
:105FE0006B017C01111112C0672B682B692B71F4B6
:105FF000A114B10459F0D5018C91882339F061E0E6
:10600000C5010E945DC707C0112391F360E089E7D5
:1060100093E00E943FC783E090E09093F71980934C
:10602000F61981E0809337100E9476750E943942FC
:10603000C114D104E104F104E1F080911D0E9091AE
:106040001E0EA0911F0EB091200EC80ED91EEA1E82
:10605000FB1E0E9486C2DC01CB018C199D09AE0992
:10606000BF09B7FF1AC08091371081110C94943C7E
:1060700014C080913710882321F080E00E94F6E759
:10608000F8CF80911F1360E0882319F08AE693E02F
:1060900002C08AE593E00E943FC7109237100C942B
:1060A000B92684918F010F5F1F4F882321F00E9432
:1060B0004442F801F6CF1092C4151092C31580E542
:1060C00093E10E94C9B68BE1E0E5F3E1DE011596AC
:1060D00001900D928A95E1F780914E1390914F13A4
:1060E0009C838B838FE992E09A83898340E050E020
:1060F000BE016F5F7F4F89E095E00E94826DCE0107
:1061000001960E9454BDE5E9F3E084918F010F5F91
:106110001F4F882311F40C94B9260E944442F801C1
:10612000F4CF0E94046C0E945CBD0C94B9261092BE
:106130001F13109220130C94B926203209F41082F8
:10614000319620812111F9CF40E061E00E948B6FF0
:106150000C94B9260E94AEE080912013882319F098
:1061600081E080931F130E946EE00C94B926809109
:106170002013882311F40C94B92683E50E94BA41B8
:10618000882311F40C94B9260E942841AB01BC016C
:106190004093BA155093BB156093BC157093BD1511
:1061A0008AEE94E10E9451E50C94B9268091201367
:1061B000811103C0E7ECF3E02AC0E5EBF3E0849142
:1061C0008F010F5F1F4F882321F00E944442F80186
:1061D000F6CF6091BA157091BB158091BC15909166
:1061E000BD154AE00E944B428FE20E9444426091FA
:1061F000B6157091B7158091B8159091B9154AE010
:106200000E944B428AE00E9444420C94B926849139
:106210008F010F5F1F4F882311F40C94B9260E9441
:106220004442F801F4CF40E060E080919005909105
:1062300091050E948B6F0C94B926809120138823BE
:1062400011F40C94B9268AEE94E10E941FE58AEEBF
:1062500094E10E946CB510921E1310921D13E090F1
:106260009005F090910580912013882311F40C94EF
:10627000B92610921F138091ED14882321F08AEE25
:1062800094E10E946CB5FE0131966F01CF010E942E
:10629000C3E28CE493E190936C1380936B13D7016A
:1062A0008C918F3209F060C06FE270E0C7010F94EB
:1062B00062098C010F5F1F4F09F45CC06FE270E050
:1062C000C8010F9462095C01009709F454C00817D3
:1062D000190708F050C04C01801A910AA401B801B6
:1062E000CE0180960F948B09E0E2F0E0EC0FFD1FE9
:1062F000E80DF91D10828E01005E1F4FF80181919B
:106300008F01882319F00E944442F8CF8AE00E944E
:10631000444260916B1370916C136115710511F01B
:106320006C5F7F4F21E0AE01405E5F4FCE0105966E
:106330000E94FABA811112C0BE01605E7F4F8EEFDB
:1063400093E00E9466EC8EE20E9444428AE00E9442
:106350004442C6010E9454BD0C94B926D0926C13DD
:10636000C0926B138501A6CF8DE693E190936C13D9
:1063700080936B13870180916B1390916C1300973E
:1063800009F00496B8010E9475E7811103C0E6EE9A
:10639000F3E021C0E8EDF3E084917F012FEFE21AF2
:1063A000F20A882321F00E944442F701F5CFD80178
:1063B0008D918D01882319F00E944442F8CF8AE024
:1063C0000E9444421092BA151092BB151092BC154F
:1063D0001092BD1516C084917F01BFEFEB1AFB0A26
:1063E000882321F00E944442F701F5CFF801819102
:1063F0008F01882319F00E944442F8CF8EE20E9458
:106400004442C6010E9454BD0C94B92680911F13CA
:1064100081110E947675E0909005F090910580E5DD
:106420000E948B41182F882319F00E944941182F90
:1064300080912013882311F40C94B926412F61E038
:10644000C7010E948B6F83E50E94BA41882381F0C7
:106450000E942841AB01BC014093BA155093BB1573
:106460006093BC157093BD158AEE94E10E9451E5CE
:1064700080912013882319F081E080931F1311115C
:106480000C94B92670CE809190059091910521E0F1
:1064900020931E1340E060E00E948B6F0C94B9269D
:1064A0000E944C6D7B018C0120E831E541E050E019
:1064B0000F94C005C9016DE671E00F94E6084B0129
:1064C0005C01C801B70120E13EE040E050E00F94DC
:1064D000C005CA01B90128E130E040E050E00F9466
:1064E000C005762E672EC62ED72E5CE3252E312CC6
:1064F000412C512CC801B701A20191010F94C00594
:10650000F62EE72ECA01B901A20191010F94C00530
:10651000CB018E010F5F1F4F8114910499F0EF9210
:10652000FF927F936F936F927F92BF92AF929F92F1
:106530008F928AE394E09F938F931F930F930E940F
:106540001EFF13C0A114B104B1F0EF92FF927F932C
:106550006F936F927F92BF92AF928AE294E09F9383
:106560008F931F930F930E941EFF0FB6F894DEBF08
:106570000FBECDBF30C0CD2879F0EF92FF927F9350
:106580006F936F927F928EE194E09F938F931F930E
:106590000F930E941EFFE9CF892B69F0EF92FF92C3
:1065A0007F936F9386E194E09F938F931F930F9354
:1065B0000E941EFFDACFEF92FF9282E194E09F9358
:1065C0008F931F930F930E941EFF0F900F900F90B9
:1065D0000F900F900F9060E0C8010E945DC7EBE93B
:1065E000F9E484917F01BFEFEB1AFB0A882321F0C5
:1065F0000E944442F701F5CFB8018EE494E00E9476
:1066000066EC8AE00E9444420C94B92683E50E941D
:10661000BA41882311F40C94B9260E943841E82E1F
:1066200080E50E94BA41882311F40C94B9260E9497
:106630002841162FC62ED72ED7FE02C00C94B9269D
:10664000E8E3F7E080E697E02491121303C0E9EC59
:10665000F6E109C031968E179F07B1F70C94993C6B
:106660000E944442F80184918F010F5F1F4F8111F6
:10667000F7CFEBE5F4E084918F010F5F1F4F882384
:1066800011F40C94B9260E944442F801F4CF0E9400
:106690006EE00C94B9260E9416E00C94B9260E9474
:1066A0009ED80C94B92688E690E00E94B6428111EB
:1066B0000C94B9268091CF1583FF02C00C94B926A3
:1066C00083E50E94BA418823B1F10E9458410F949A
:1066D0006207CB010E94C5C60E94584120E030E00D
:1066E0004AEA52E40E9484FF18163CF00E949ED8A9
:1066F00060E086E794E00E943FC70E9458412091E5
:106700005F123091601240916112509162120F94A9
:106710004408181684F48DE093E09F938F938AE6E3
:1067200094E09F938F931F920E94B7D80F900F9081
:106730000F900F900F900E9411ED0C94B9268EE4EB
:106740000E94BA41882311F40C94B9260E94284172
:106750006093F2197093F3198093F4199093F519DB
:106760000C94B92683E50E948B41882359F083E578
:106770000E94BA41882319F00E94384101C080E08C
:106780008093CF15EBE9F9E484918F010F5F1F4FE0
:10679000811103C0E4E9F4E004C00E944442F8011E
:1067A000F3CF84918F010F5F1F4F882321F00E9448
:1067B0004442F801F6CF8091CF15811103C0E0E982
:1067C000F4E034C046E8C42E44E0D42EE12CF12C91
:1067D00020E08091CF1590E00E2C02C09595879512
:1067E0000A94E2F780FF17C0BB24B394B20E2223B1
:1067F00019F08CE20E944442F60185919491FC01CB
:1068000084918F010F5F1F4F882321F00E94444223
:10681000F801F6CF2B2DEFEFEE1AFE0AF2E0CF0EC5
:10682000D11C35E0E316F104A1F60AC084918F0172
:106830000F5F1F4F882321F00E944442F801F6CFDA
:106840008AE00E9444420C94B9268BE994E00E94AD
:1068500028C083E50E94BA41811103C0EBE9F9E445
:106860000DC00E943841809382028D3310F40C9445
:10687000B9268CE3809382020C94B92684918F010F
:106880000F5F1F4F882321F00E944442F801F6CF8A
:106890004091820250E060E070E084EA94E00E945F
:1068A00013EC8AE00E9444420C94B9268091CF15E3
:1068B00083FF02C00C94B92683E50E94BA41882365
:1068C00011F40C94B9260E9458410F9462076E3758
:1068D000710514F06DE770E07093EA156093E915A7
:1068E0000E940EA80C94B92689E690E00E94B64258
:1068F000811111C0EBEAF4E084918F010F5F1F4F0B
:10690000882321F00E944442F801F6CF0E948B595F
:106910008AE00E9444421092F7191092F6190C94E2
:10692000033D83E50E94BA41882311F40C94B926F3
:106930000E9438418093FC198D3318F08CE38093CA
:10694000FC190E9486C26B017C012091FC1930E089
:10695000A8EEB3E00F940E06C60ED71EE81EF91E71
:10696000C092F819D092F919E092FA19F092FB1935
:106970000C94B9260E9402600C94B92683E50E940B
:10698000BA41882339F00E9428418B016F3F71057D
:1069900019F010F00FEF10E080E50E94BA4181116C
:1069A00006C01093EC150093EB150C94B9260E94C9
:1069B000384181110C94B926F4CF80E50E94BA4188
:1069C000811106C01092EC151092EB150C94B926AB
:1069D0000E942841672B11F00C94B926F3CF109236
:1069E00088050C94B92681E0809388050C94B9261B
:1069F00083E50E94BA418823A1F00E94584120E01B
:106A000030E04AE754E40E94E9FF0F94670760937F
:106A100083027093840280938502909386020C9483
:106A2000B92688E50E948B4181119CC789E50E94A7
:106A30008B41811197C78AE50E948B41811192C7D2
:106A400085E40E948B4181118DC70E9476750E945A
:106A500098EA0C94B92683E50E948B41882311F4AF
:106A60000C94B9260E94584120E030E04AE754E4F3
:106A70000E94E9FF0F9467076093001A7093011A50
:106A80008093021A9093031A0C94B926D6018D9123
:106A90006D010E948B41882309F46DC0133009F009
:106AA00063C00E9458414B015C0120E030E040EAA5
:106AB00051E40E9484FF87FF4EC0A50194016091BC
:106AC0006A1870916B1880916C1890916D180F94E2
:106AD000FA062B013C019B01AC016091B00670915C
:106AE000B1068091B2069091B3060E94E9FF6093CF
:106AF000B0067093B1068093B2069093B306A301DB
:106B0000920160918406709185068091860690912D
:106B100087060E94E9FF6093840670938506809340
:106B200086069093870660911E1A70911F1A8091B5
:106B3000201A9091211A0E9488FFA30192010E94BD
:106B4000E9FF0F94670760931E1A70931F1A8093D2
:106B5000201A9093211A80926A1890926B18A09232
:106B60006C18B0926D1807C00E945841F7016083FD
:106B70007183828393831F5FF4E0EF0EF11C143066
:106B800009F084CF0E945FEE0C94B9260E947675BE
:106B90000E94CC580C94B9260E944442F80184917A
:106BA0008F010F5F1F4F8111F7CFE9E8F5E003C0B8
:106BB0000E944442F80184918F010F5F1F4F8111A1
:106BC000F7CFE2E7F5E003C00E944442F801849168
:106BD0008F010F5F1F4F8111F7CFE2E6F5E003C091
:106BE0000E944442F80184918F010F5F1F4F811171
:106BF000F7CFE1E5F5E003C00E944442F80184913B
:106C00008F010F5F1F4F8111F7CFE0E4F5E003C064
:106C10000E944442F80184918F010F5F1F4F811140
:106C2000F7CFE1E3F5E003C00E944442F80184910C
:106C30008F010F5F1F4F8111F7CFECE1F5E003C02B
:106C40000E944442F80184918F010F5F1F4F811110
:106C5000F7CFE6E0F5E003C00E944442F8018491DA
:106C60008F010F5F1F4F8111F7CFE1EFF4E003C0F9
:106C70000E944442F80184918F010F5F1F4F8111E0
:106C8000F7CFE4EDF4E003C00E944442F8018491A0
:106C90008F010F5F1F4F8111F7CFECEBF4E0849170
:106CA0008F010F5F1F4F882311F40C94B9260E94A7
:106CB0004442F801F4CF60E08091900590919105F5
:106CC0000E945DC70C94B92685E40E948B418823FD
:106CD00081F00E944941882361F0EBE9F9E4849155
:106CE0008F010F5F1F4F882321F00E944442F8015B
:106CF000F6CF81E40E948B41882381F00E944941B4
:106D0000882361F0E8E5F6E084918F010F5F1F4F63
:106D1000882321F00E944442F801F6CF00919005AB
:106D200010919105D8018D918D01882309F488CDAA
:106D30000E944442F7CF0E94F17E0C94B92681E074
:106D40008093090E8093C40F0C94B9261092090EFB
:106D50001092C40F0C94B92683E50E94BA4188238F
:106D600019F00E94284102C060E070E08B011127F9
:106D700002301105DCF0E9ECF6E184918F010F5F40
:106D80001F4F811103C0ECE5F6E004C00E944442AD
:106D9000F801F3CF84918F010F5F1F4F882311F407
:106DA0000C94B9260E944442F801F4CF88E40E9472
:106DB000BA418823A9F00E9428416A3A71053CF043
:106DC0006530B1E07B072CF064E071E002C06AEA54
:106DD00070E0F801EE0FFF1FE753F04F71836083FF
:106DE00086E40E94BA418823A9F00E942841F80154
:106DF000EE0FFF1FE353F04F718360836F3F710508
:106E000019F014F06FEF70E077FF02C060E070E0FF
:106E10007183608382E40E94BA41882311F40C9448
:106E2000B9260E9428416530710534F06F3671052E
:106E30002CF06EE670E002C065E070E0000F111FFC
:106E4000F801EB53F04F718360830C94B92688EC02
:106E500090E00E94B64281110C94B92684E40E940D
:106E60008B41882309F443C00E9458416B017C0187
:106E700011E020E030E0A9010E9484FF811101C0EF
:106E800010E010935E0620E030E0A901C701B601D2
:106E90000E9484FF882359F10091840510E00E942C
:106EA0005841000F111F000F111FF801E65AF94F4A
:106EB000608371838283938320E030E0A901609135
:106EC0005A0670915B0680915C0690915D060E9467
:106ED00084FF81110CC080E090E0A0EEBFE38093BE
:106EE0005A0690935B06A0935C06B0935D060E94E1
:106EF000AFE70C94B926E7E9EE2EE2E0FE2E08E8B3
:106F000016E0F8E9CF2EF6E0DF2EF70181917F0140
:106F10000E948B41882351F00E9458410F946707CB
:106F2000D8016D937D938D939C9313970C5F1F4FA6
:106F3000C016D10651F70E9441ED0C94B92677E9AD
:106F4000E72E72E0F72E08E716E0F70181917F0146
:106F50000E948B41882341F00E945841D8016D93D3
:106F60007D938D939C9313970C5F1F4FB6E0083869
:106F70001B0759F70C94B92683E50E948B4188239F
:106F8000D9F00E945841AB01BC014093A006509338
:106F9000A1066093A2067093A306409398065093AF
:106FA000990660939A0670939B0688ED96E00E947E
:106FB00030EC8AE00E94444280E50E948B418823A5
:106FC00099F00E945841AB01BC014093A006509338
:106FD000A1066093A2067093A3068BEB96E00E9435
:106FE00030EC8AE00E94444282E50E948B41882373
:106FF00099F00E945841AB01BC0140939C0650930C
:107000009D0660939E0670939F068CE996E00E9411
:1070100030EC8AE00E94444284E50E948B41882340
:1070200011F40C94B9260E945841AB01BC01409365
:1070300098065093990660939A0670939B068EE784
:1070400096E00E9430EC8AE00E9444420C94B926FB
:1070500083E50E948B41882351F00E945841609340
:10706000740670937506809376069093770684E590
:107070000E948B41882351F00E9458416093700612
:1070800070937106809372069093730682E40E9457
:107090008B41882351F00E94184160937D127093B8
:1070A0007E1280937F129093801288E50E948B411C
:1070B000882351F00E9458416093A4067093A5065E
:1070C0008093A6069093A70689E50E948B418823AA
:1070D00051F00E9458416093A8067093A9068093CE
:1070E000AA069093AB068AE50E948B41882351F053
:1070F0000E9458416093AC067093AD068093AE0633
:107100009093AF0685E40E948B41882311F40C9480
:10711000B9260E9458416093B0067093B1068093DF
:10712000B2069093B3060C94B92667E9E62E62E0A6
:10713000F62E00E010E0F70181917F010E948B4163
:10714000882331F00E945841AB01BC01C80158D7D7
:107150000F5F1F4F0330110571F70E94B1400E946D
:10716000CC580C94B92684918F010F5F1F4F882350
:1071700021F00E944442F801F6CF83E50E948B4142
:10718000882321F00E94494180931D02E8E2F7E044
:1071900084918F010F5F1F4F882321F00E9444428A
:1071A000F801F6CF80911D02882319F0E0E2F7E0A4
:1071B00002C0E4E2F7E084918F010F5F1F4F81115D
:1071C00003C0E8E1F7E004C00E944442F801F3CFB5
:1071D00084918F010F5F1F4F882321F00E9444424A
:1071E000F801F6CF4091E40F5091E50F6091E60F62
:1071F0007091E70F86E197E00E9430EC4091E80F34
:107200005091E90F6091EA0F7091EB0F83E197E0E5
:107210000E9430EC4091EC0F5091ED0F6091EE0F19
:107220007091EF0F80E197E00E9430ECE8E0F7E02A
:1072300084918F010F5F1F4F882321F00E944442E9
:10724000F801F6CF409111025091120260911302A1
:107250007091140286E097E00E9430EC4091150294
:1072600050911602609117027091180283E097E026
:107270000E9430EC4091190250911A0260911B0259
:1072800070911C0280E097E00E9430EC8AE00E943E
:1072900044420C94B92683E50E94BA41882311F434
:1072A0000C94B926D5D770937102609370020C9438
:1072B000B9268DED90E00E94B64281110C94B9265A
:1072C00083E50E94BA41882311F40C94B9260091F9
:1072D000840510E0BDD7000F111FF801E259FD4FE2
:1072E000718360830C94B92680E50E948B418823CA
:1072F00011F40C94B926ACD7F62EC62ED72E83E502
:107300000E94BA41882319F0A3D78B0102C00FEF66
:107310001FEFC8010196039710F00C94B926D7FE11
:1073200002C00C94B926E8E3F7E080E697E02491E8
:10733000F21611F40C94B92631968E179F07B9F7FF
:1073400039C383E50E94BA41882311F081D702C076
:1073500064E071E079A368A380E50E94BA418823C4
:1073600031F076D76938F3E17F0730F402C068EE78
:1073700073E07A83698304C088E893E19A83898300
:10738000BE01605E7F4FCE0101960E94E2DF0C9449
:10739000B92685E4EFD781110EC080E5BCD78823DC
:1073A00081F086D76093A90D7093AA0D8093AB0DE1
:1073B0009093AC0D06C05CD7882379F3E9ECF6E135
:1073C0006CC089E4A8D7882379F072D72CEA35EC11
:1073D00047E25EE30E94E9FF6093A50D7093A60D5E
:1073E0008093A70D9093A80D84E495D7882379F016
:1073F0005FD72CEA35EC47E25EE30F94FA06609320
:10740000AD0D7093AE0D8093AF0D9093B00DEBE981
:10741000F9E484918F010F5F1F4F882321F00E94B0
:107420004442F801F6CF4091A90D5091AA0D609108
:10743000AB0D7091AC0D88E697E00E9430EC2CEA21
:1074400035EC47E25EE36091A50D7091A60D809149
:10745000A70D9091A80D0F94FA06AB01BC0184E62C
:1074600097E00E9430EC2CEA35EC47E25EE3609155
:10747000AD0D7091AE0D8091AF0D9091B00D0E9449
:10748000E9FFAB01BC0180E697E00E9430EC8AE0A6
:10749000FBD70C94B926F8D7F80184918F010F5FC0
:1074A0001F4F8111F8CF08E113E0D8018D918D01B4
:1074B000882309F4C5C9E8D7F8CF80E52CD78823FD
:1074C00049F0F6D66093A10D7093A20D8093A30DA1
:1074D0009093A40D89E41FD7882379F0E9D62CEA8C
:1074E00035EC47E25EE30E94E9FF60939D0D7093E7
:1074F0009E0D80939F0D9093A00D84E40CD788235C
:1075000079F0D6D62CEA35EC47E25EE30F94FA0622
:107510006093990D70939A0D80939B0D90939C0DA1
:10752000EBE9F9E484918F010F5F1F4F882319F075
:10753000ABD7F801F7CF4091A10D5091A20D60910A
:10754000A30D7091A40D84E797E00E9430EC2CEA23
:1075500035EC47E25EE360919D0D70919E0D809148
:107560009F0D9091A00D0F94FA06AB01BC0180E72E
:1075700097E00E9430EC2CEA35EC47E25EE3609144
:10758000990D70919A0D80919B0D90919C0D0E9488
:10759000E9FFAB01BC018CE697E00E9430EC8AE089
:1075A00073D70C94B92683E5B6D6182F882369F0D3
:1075B0007FD60F946207709328026093270221E020
:1075C000672B09F020E02093631280E5A4D688237E
:1075D00059F02091270230912802232B09F059D627
:1075E000809363120C94B92611110C94B926EBE91F
:1075F000F9E484918F010F5F1F4F882319F044D75E
:10760000F801F7CF80916312882319F061EC73E0E1
:1076100002C069E073E08DE897E00E9466EC60913B
:107620002702709128028CE797E00E944DECE8E772
:10763000F7E084918F010F5F1F4F882311F40C94A2
:10764000B92622D7F801F5CF0E940E5A0C94B9261C
:107650000E9476750C94B926E9E1F6E0FEA7EDA745
:1076600081E3882E82E1982E9EE4A92E98E1B92E1E
:1076700024EEC22E2FE0D22E31E1232E32E0332E23
:107680004FE6E42E4DE2F42E00E010E0ADA5BEA5DD
:107690008D91BEA7ADA7882309F485C0F501408070
:1076A000518062807380D1012D913D914D915C910B
:1076B000F60160817181828193810F941E0620E022
:1076C00030E040E05FE30E94E9FF9B01AC01C301B1
:1076D000B2010F944408181654F4F701859195915E
:1076E000A591B49189AB99AFADABBDAF04C019AA58
:1076F00019AE1DAA1DAED4012D913D914D915C9105
:10770000C301B2010F941D069B01AC0169A979ADBB
:107710008DA99DAD0F941D062B013C0120E030E0AA
:1077200040EA51EC0F94440887FD0AC020E030E0A5
:1077300040EA51E4C301B2010E9484FF18161CF410
:10774000E9ECF6E107C0B301A201C80159D42BC08E
:107750009BD6F80184918F010F5F1F4F8111F8CFE5
:10776000EEEBF7E084918F010F5F1F4F882319F034
:107770008BD6F801F7CF61E080EB97E00E943FC71E
:107780000E944D4A88E290E09A83898388EC90E0D9
:1077900099A388A3BE016F5F7F4FCE0180960E94A0
:1077A000E2DF0C94B9260F5F1F4FB4E08B0E911CE3
:1077B000E4E0AE0EB11CF4E0CF0ED11C24E0220EAA
:1077C000311C34E0E30EF11C0330110509F05ECFEB
:1077D000C8D40E94CC5860E080EA97E00E943FC77E
:1077E00083E992E099A388A304E610E01A83098351
:1077F000BE01605E7F4FCE0101960E94E2DF8AEB00
:1078000092E099A388A31A830983BE01605E7F4F2B
:10781000CE0101960E94E2DF0C94B9260E94DA891B
:107820000C94B9260E94A9830C94B92683E573D5DC
:10783000882311F02ED501C081E091E089270E94B4
:10784000537F0C94B9260E94D0460C94B9261CD6BE
:10785000F80184918F010F5F1F4F8111F8CFECED7C
:10786000F7E084918F010F5F1F4F882311F40C9470
:10787000B9260AD6F801F5CF81E08093060210926E
:107880008A1283E548D5811104C00E94A2EB0C94B2
:10789000B926FFD481110C94B926F7CFF090920548
:1078A000FF2001F1EBE9F9E484918F010F5F1F4F95
:1078B000882319F0E9D5F801F7CF84E5E5D56F2DD8
:1078C00070E080E090E04AE0E6D580E2DDD508E1B6
:1078D00013E0D8018D918D01882311F40C9420348C
:1078E000D3D5F7CF10921806EBE9F9E484918F0114
:1078F0000F5F1F4F882319F0C7D5F801F7CF6091AC
:10790000180670E08BEE97E00E944DEC8AE0BCD543
:107910000C94B9266115710519F4BF016150710904
:1079200040E050E00C94292780E00E94F6E70C9498
:10793000293061E0812F0E944AC16E2D812F0E9463
:107940007A83F12CB701812F0E9486C1B9E0CB1652
:10795000D10411F00C94B926F092EC15E092EB15DD
:107960000C94B9260E94767588E5D5D4882319F041
:107970005F9A10920A0E89E5CED4882319F08A9A6C
:1079800010920B0E8AE5C7D4882351F09FB7F89464
:10799000809108018160809308019FBF10920C0EB6
:1079A00085E4B9D4882311F40C94B9260E94F4E735
:1079B0000C94B9260E94767560E08F2D0E944AC112
:1079C0000F3FEFEF1E0759F48F2D0E94518331E0D6
:1079D00020E0892B09F030E0032F122F05C0013081
:1079E000110571F401E010E08F2D0E945183801782
:1079F000910711F40C94B92680E00E94F6E7F4CFC9
:107A000000E010E0F1CFC05ADF4F0FB6F894DEBFB0
:107A10000FBECDBFDF91CF911F910F91FF90EF90DF
:107A2000DF90CF90BF90AF909F908F907F906F909E
:107A30005F904F903F902F9008959091210EE92FE5
:107A4000F0E0E75EF14F80839F5F943018F49093ED
:107A5000210E02C01092210E8091C20F8F5F809381
:107A6000C20F0895089580E090E008958FB7F894CC
:107A70009091F1192091F019921759F0E92FF0E047
:107A8000E059F64E208130E09F5F9F779093F11987
:107A900002C02FEF3FEF8FBFC90108950F931F93CF
:107AA000CF93DF93EC010E9486C20E811F8128854F
:107AB0003985011511052105310559F52C8522233C
:107AC000A9F13A8521502C8721E0230F2A874D8583
:107AD000241301C01A86FE0124E0329FE00DF11D3F
:107AE000112406851785208931890A831B832C83FD
:107AF0003D83DC01CB01800F911FA11DB11D8E8341
:107B00009F83A887B9878C819D81892B79F0409AC2
:107B10000DC0DC01CB01801B910BA20BB30BB7FD99
:107B200005C040981E821F8218861986DF91CF916A
:107B30001F910F910895CF92EF92FF920F931F9391
:107B4000E0900D02F0900E0200910F0210911002D1
:107B5000C09018062AE538E146E558E162E578E18B
:107B60008EE498E10E94CECA1F910F91FF90EF9092
:107B7000CF900895CF92DF92EF92FF92CF9381E062
:107B800080932902C1E081E090912902992309F4B0
:107B900049C0882309F446C080E00E94F6E760915E
:107BA000220E7091230E6115710581F1072E000CD4
:107BB000880B990B0E948AFF9B01AC0160915F12B8
:107BC0007091601280916112909162120F941D0663
:107BD0006B017C0120E030E0A9010F9444081816E5
:107BE0005CF020E030E040E450ECC701B6010E94B8
:107BF00084FF87FD0DC00AC020E030E040E450E47F
:107C0000C701B6010F944408181614F080E0BCCFE9
:107C1000C0932E1040E050E0BA018AEC97E90E9430
:107C20002A4AB1CFCF91FF90EF90DF90CF90089587
:107C3000CF92DF92EF92FF920F931F93CF93DF9338
:107C400000D01F92CDB7DEB7182F662351F01092E7
:107C50000606109202061092030610920406109275
:107C600005060E9486C2C0900206D0900306E090EE
:107C70000406F09005069B01AC012C193D094E0944
:107C80005F0957FD3EC017FD16C040910606212F23
:107C9000012E000C330B2C5F3F4FE42F042E000C01
:107CA000FF0B2E173F076CF141172CF000E911E094
:107CB00020E030E004C004EC19E020E030E0DC011A
:107CC000CB01800F911FA21FB31F809302069093D8
:107CD0000306A0930406B093050680ED97E09C830D
:107CE0008B838CE291E09A838983BE016D5F7F4F25
:107CF000CE0101960E94E2DF809106068F5F80939D
:107D000006060F900F900F900F90DF91CF911F916B
:107D10000F91FF90EF90DF90CF9008954F925F9278
:107D20006F927F928F929F92AF92BF92CF92DF928B
:107D3000EF92FF920F931F93CF93DF935C014B0160
:107D40008A01E90140900D0250900E0260900F02EE
:107D500070901002FA01208131814281538160913B
:107D600056187091571880915818909159180E9480
:107D700084FF87FF2DC0C880D980EA80FB8020E087
:107D800030E0A901B601C7010E9484FF811108C03B
:107D9000E3E8FDE285919591A591B4916C017D0197
:107DA000C601D70180930D0290930E02A0930F029B
:107DB000B0931002F80180819181A281B3818093F8
:107DC000561890935718A0935818B0935918B3DECB
:107DD000C880D980EA80FB8020E030E0A901C7019B
:107DE000B6010E9484FF811106C0C12CD12C88E409
:107DF000E82E82E4F82EC0920D02D0920E02E0929C
:107E00000F02F0921002F50180819181A281B3816D
:107E100080934E1890934F18A0935018B093511818
:107E2000F40180819181A281B38180935218909353
:107E30005318A0935418B09355187DDEF801208193
:107E40003181428153816091561870915718809109
:107E50005818909159180F94440818169CF5D8801A
:107E6000E980FA80CB8120E030E0A9016D2D7E2DE4
:107E70008F2D9C2F0E9484FF81110AC0E3E8FDE250
:107E800085919591A591B491D82EE92EFA2ECB2FFC
:107E90008D2D9E2DAF2DBC2F80930D0290930E0241
:107EA000A0930F02B0931002F80180819181A2810A
:107EB000B3818093561890935718A0935818B09395
:107EC000591839DE0E94767540920D0250920E02CA
:107ED00060920F0270921002DF91CF911F910F916B
:107EE000FF90EF90DF90CF90BF90AF909F908F90DA
:107EF0007F906F905F904F90089580E1EEE4F8E1FD
:107F0000A9E4B2E101900D928A95E1F7089580E12C
:107F1000E9E4F2E1AEE4B8E101900D928A95E1F76F
:107F20000895CF92EF92FF920F931F93C09018067F
:107F30007B018C0125E532E141E552E16DE472E11E
:107F400089E492E10E94CECA1F910F91FF90EF90B9
:107F5000CF900895CF92DF92EF92FF920F931F93ED
:107F6000CF93DF93EC01CC0FDD1FCC0FDD1FFE01A3
:107F7000E35FF14F20E030E0A901608171818281EF
:107F800093810F941E06FE01E35CFD4E208131813A
:107F9000428153810F941E066B017C01FE01EF5C50
:107FA000FD4E6083718382839383FE01E557F64F14
:107FB00025913591459154918E010C51104F0F949C
:107FC0001E06F8016083718382839383FE01E95664
:107FD000F64F2591359145915491CF5EDD4FC70104
:107FE000B6010F941E06688379838A839B83DF9191
:107FF000CF911F910F91FF90EF90DF90CF90089558
:108000008F929F92AF92BF92EF92FF920F931F9326
:10801000CF93DF938C014A015B01EC01CC0FDD1F94
:10802000CC0FDD1FCE01825B974E7C01C35FD14F29
:10803000288139814A815B81C501B4010F941D06F5
:10804000F70120813181428153810F941E06F7018F
:10805000608371838283938388829982AA82BB82A0
:10806000C801DF91CF911F910F91FF90EF90BF90CA
:10807000AF909F908F906ECFCF93FC0120812B33D8
:10808000A1F02091C20F243080F4C62FBC01809152
:10809000210EF0E68F9FC00111248F5B914F0F944A
:1080A00076098C2FCADC81E001C080E0CF91089571
:1080B000DF92EF92FF920F931F93CF93DF93CDB791
:1080C000DEB76E970FB6F894DEBF0FBECDBF6091DE
:1080D000C2087091C3086115710549F14DE150E086
:1080E000CE0101967C010E94F5FE1E8EF7018F01E4
:1080F0000E191F09D190DD2019F09AE0D912F7CF9F
:10810000F701E00FF11F1082C7010E9449DA8823AE
:1081100071F0DD20A9F00F5F1F4F8091C208909190
:10812000C308080F191F1093C3080093C20881E009
:108130002091C2083091C308232B29F480E003C0AA
:1081400000E010E0F0CF6E960FB6F894DEBF0FBEE1
:10815000CDBFDF91CF911F910F91FF90EF90DF90F6
:1081600008952AE538E146E558E162E578E18EE4D4
:1081700098E10C949CED8F929F92AF92BF92CF9218
:10818000DF92EF92FF920F931F93CF93DF934A01F9
:108190005B017901EC01CC0FDD1FCC0FDD1FCE019F
:1081A000825B974E6C01FC01108211821282138255
:1081B000D8DFF60180829182A282B382C090180635
:1081C00020E030E0A901B801C7010E9484FF8111BD
:1081D0000CC0FE01E558F24D4591559165917491A1
:1081E000342F252F962F872F04C0302F212F9E2D1F
:1081F0008F2DE32EF22E092F182F2AE538E146E5C0
:1082000058E162E578E18EE498E10E94CECA0E94CE
:1082100076751092400EDF91CF911F910F91FF90D4
:10822000EF90DF90CF90BF90AF909F908F90089588
:108230008091950590919605009731F04AE050E0C5
:1082400060E070E00C94CBFD60E070E0CB0108953D
:108250008091950590919605009731F04AE050E0A5
:1082600060E070E00C949EFC60E070E0CB0108954B
:10827000EFDF97FD0AC0ECDF6F3F710581059105C7
:1082800009F02CF4E5DF862F089580E008958FEF44
:1082900008958091950590919605892B31F0E8DF3E
:1082A00091E0811103C090E001C091E0892F089511
:1082B0000F931F93CF93809195059091960500970A
:1082C000F1F0FC018F01C1912C2F2F7D89F0C53475
:1082D00011F0C536B9F7F801108260E070E00E9435
:1082E0004AFBF801C083562F472F382F292F0BC088
:1082F00060E070E0CF911F910F910C944AFB50E029
:1083000040E030E020E0652F742F832F922FCF9133
:108310001F910F91089581548A3150F5482F50E0F4
:10832000FA0193E0F595E7959A95E1F7E058FA4F51
:10833000208130E0877002C0359527958A95E2F755
:10834000822F817020FF15C0FA01EA59FA4F9081FF
:10835000992339F02091FE193091FF19290F311D11
:1083600002C020E030E030939605209395050895F3
:1083700080E00895D0DF882341F081E020919505C9
:1083800030919605232B09F480E00895CF92DF9277
:10839000EF92FF920F931F93CF93DF9387E9E82E1D
:1083A00082E0F82E09E412E1CEE4D8E195E8C92E86
:1083B00095E0D92EF70181917F01ADDF8823D9F0B7
:1083C00077DF9B01AC01F6018081811104C08091AF
:1083D0008905882329F0688179818A819B8103C07E
:1083E00060E070E0CB010F941E06F801608371839A
:1083F0008283938309C088819981AA81BB81F80116
:1084000080839183A283B3830C5F1F4F2496FFEF79
:10841000CF1ADF0A8BE9E81682E0F80659F686E4FF
:10842000A9DF8823B9F044DF20E030E0A9010F94F0
:10843000440818167CF43CDF20E030E040E752E4CA
:108440000F94FA0660930D0270930E0280930F0250
:1084500090931002DF91CF911F910F91FF90EF90B9
:10846000DF90CF900895FC01238121110C946CB50D
:1084700008950E9486C260931D0E70931E0E809315
:108480001F0E9093200E08959091C00095FFFCCF91
:108490008093C60008958F929F92AF92BF92EF9201
:1084A000FF920F931F93CF93DF93CDB7DEB7A097C3
:1084B0000FB6F894DEBF0FBECDBF61157105810503
:1084C000910589F100E0842E912CA12CB12C102F64
:1084D000EE24E394F12CEC0EFD1EE00EF11C07FDE2
:1084E000FA94A50194010F94C005F7016083B901C6
:1084F000CA010F5F611571058105910541F71F3FA5
:1085000021F1E1E0F0E0EC0FFD1FE10FF11D17FD9F
:10851000FA9580818A3010F097E301C090E3890FCB
:10852000B3DF1150ECCF80E3A0960FB6F894DEBF16
:108530000FBECDBFDF91CF911F910F91FF90EF90B4
:10854000BF90AF909F908F909FCFA0960FB6F8945A
:10855000DEBF0FBECDBFDF91CF911F910F91FF9076
:10856000EF90BF90AF909F908F900895EF92FF9201
:108570000F931F93CF93DF937C0184E5FBDED82F0D
:10858000882321F175DEC82F1816E4F4EBE9F9E42D
:1085900084918F010F5F1F4F882319F075DFF80159
:1085A000F7CF8DE471DFB70180E090E04AE073DF40
:1085B0006C2FCC0F770B88E799E00E944DEC8AE096
:1085C00063DF08C080938405D0E004C08091180662
:1085D000809384058D2FDF91CF911F910F91FF9094
:1085E000EF900895CF92DF92EF92FF926B017C01A2
:1085F00097FF0AC08DE248DFF094E094D094C094D5
:10860000C11CD11CE11CF11C4AE0C701B601FF905E
:10861000EF90DF90CF903FCFFF920F931F93CF93B8
:10862000DF93F82E092F162FE9ECF6E18491EF0184
:108630002196882319F028DFFE01F8CFEF2DF02FC7
:108640008491EF012196882319F01EDFFE01F8CFF7
:108650006091F2197091F3198091F4199091F519C4
:10866000C1DF8AE011DF11110E94A2EB1092FC051C
:108670001092FB05DF91CF911F910F91FF9008950C
:108680002F923F924F925F926F927F928F929F9222
:10869000AF92BF92CF92DF92EF92FF920F931F9310
:1086A000CF93DF931F92CDB7DEB702DD8111CAC22F
:1086B0008091C20F843008F065C0D8D99C0197FD25
:1086C00061C0982F0091FB051091FC058A3019F0CC
:1086D0009D3009F021C11092FD050115110541F3EE
:1086E000F801E556FA4F10821092FC051092FB0536
:1086F0002BE935E08901F90180812F5F3F4F8032FE
:10870000C9F38E3409F072C078016AE270E0C801E2
:108710000F9462096C01E114F10409F4ADC060E446
:1087200079E0C8010E9404FF5C01892B09F061C057
:108730004AE050E060E070E0C70101960E949EFCB4
:1087400060939705709398058093990590939A0587
:108750004090F2195090F3196090F4197090F51947
:10876000FFEF4F1A5F0A6F0A7F0A641575058605C9
:10877000970509F449C0AB2809F046C061E08DE0D7
:1087800099E04ADF80911F13882309F45BC280912E
:10879000C20F811102C01092010680913810909191
:1087A0003910181619060CF0E4C00091FE0510915E
:1087B000FF0520E6209FC001219F900D11248F5AB4
:1087C0009F4E0E9449DA882309F43CC20F5F1F4F75
:1087D0001093FF050093FE05809138109091391099
:1087E000019790933910809338102CC2E12CF12C12
:1087F0008CCF6EE470E0C80104960F946209009774
:1088000009F496CF7C0194CFC114D10401F180E02A
:10881000F12CF801E80FF11D90819A3219F08F5F69
:10882000F926F7CF4AE050E060E070E0C60101961B
:108830000E949EFCCF2CD12CE12CF12C6C157D05D7
:108840008E059F0541F061E08EEE98E09ACF61E0E1
:1088500084EC98E096CF8091970590919805A0912F
:108860009905B0919A058093F2199093F319A0930A
:10887000F419B093F51906C0892B21F060E08AE95C
:1088800098E07FCF80910602811122C067E470E0FA
:10889000C8010F9462090097D9F04AE050E060E007
:1088A00070E001960E949EFC6430710588F4E3E25A
:1088B000F8E084917F012FEFE21AF20A882319F081
:1088C000E3DDF701F6CF60E089E198E00E943FC761
:1088D00069E273E0C8010F946D09892B21F41092AD
:1088E0002902109237106EE273E0C8010F946D09EF
:1088F000892B21F480E198E00E9428C063E373E0B3
:10890000C8010F946D09892B11F40E94735861E01E
:108910008BE995E0B1DBCCCE0F3511050CF0C8CE5C
:108920009C3599F4A3D897FDC3CE2091FD05211164
:10893000BFCE98012F5F3F4F3093FC052093FB057E
:10894000F801E556FA4F8083B3CE9B3319F481E0EA
:108950008093FD058091FD058111AACEC801019685
:108960009093FC058093FB05F801E556FA4F2083B0
:108970009FCEEE24E3944091BA155091BB156091BF
:10898000BC157091BD158091B6159091B715A09149
:10899000B815B091B915481759076A077B0708F44D
:1089A000E12C00E010E09924939480E6882E99E46D
:1089B000A92E99E0B92E25E4622E29E0722E80912D
:1089C000C20F843008F03EC1E1103CC18091010625
:1089D000811138C18091F2149091F314A091F41494
:1089E000B091F5148093BA159093BB15A093BC1564
:1089F000B093BD1541E050E0BE016F5F7F4F8AEE3E
:108A000094E10E94EDB7019719F4898190E002C0CA
:108A10008FEF9FEFF82E2090BA153090BB15409045
:108A2000BC155090BD154091B6155091B715609189
:108A3000B8157091B915EE24E39424163506460650
:108A4000570608F4E12C2416350646065706B0F4FE
:108A5000019609F4AAC0FAE0FF1609F4C3C02DE09C
:108A6000F21609F4BFC083E2F81619F09AE3F9127E
:108A7000CFC0809100068111CBC0AFC0E4E6F9E021
:108A800084916F012FEFC21AD20A882319F0FCDCFF
:108A9000F601F6CF0E9476758AEE94E10E946CB5DD
:108AA00080912415882369F1815080932415EDE885
:108AB000E89FC001112441E061E0875D9A4E0E9469
:108AC0008B6FE091241524E0E29FF0011124EB5D0F
:108AD000FA4E40815181628173814093BA1550935F
:108AE000BB156093BC157093BD158AEE94E10E948E
:108AF00051E580912013882309F447C090921F13F9
:108B000044C010921F136AE58DE298E10E9441D89B
:108B10001092F51510923D1840E050E0BA0189E03E
:108B200095E10E9451E549E452E065EF75E189E085
:108B300095E10E94E7E5019669F438E3C32E33E03E
:108B4000D32EF60181916F01882311F09DDCF9CFBE
:108B50008AE09ADC89E095E10E946CB510923910A8
:108B600010923810B092C308A092C208A1DA0E94F5
:108B70009ED80E944C6D6D3371058105910528F0DA
:108B80007092C3086092C20893DA1092C215809165
:108B90002013882319F00E94556B1FC00E94046C9B
:108BA000809120138111F7CF18C0E9ECF6E1849190
:108BB0006F012FEFC21AD20A882319F065DCF60183
:108BC000F6CFE5E5F9E084916F019FEFC91AD90A64
:108BD000882319F059DCF601F6CFE3E2FE1202C059
:108BE00090920106109200060115110509F4E7CED6
:108BF0008091210E889E000D111D1124F801EF5B5C
:108C0000F14F108280E00E941D3D00E010E0D7CEC1
:108C10000F35110508F0D3CEFBE3FF1202C090928E
:108C20000006809100068111CACE8091210EF801C4
:108C3000889EE00DF11D1124EF5BF14FF0820F5F74
:108C40001F4FBDCE0F90DF91CF911F910F91FF90DD
:108C5000EF90DF90CF90BF90AF909F908F907F90DC
:108C60006F905F904F903F902F9008958F929F92BA
:108C7000AF92BF92CF92DF92EF92FF92CF936B01B0
:108C80007C01B42E20E030E0A9010E9484FF87FF20
:108C900006C08DE2F9DBF7FAF094F7F8F094C0E043
:108CA00060E070E080E09FE3CB1541F02DEC3CEC00
:108CB0004CEC5DE30E94E9FFCF5FF6CF9B01AC0176
:108CC000C701B6010F941E066B017C010F94670764
:108CD0004B015C014AE0DFDBCC2379F1C501B40133
:108CE0000E9488FF9B01AC01C701B6010F941D06CD
:108CF0006B017C018EE2C8DB20E030E040E251E411
:108D0000C701B6010E94E9FF4B015C010F946207A5
:108D10006B01770FEE08FF08C701B60163DCC701DE
:108D2000B6010E948AFF9B01AC01C501B4010F94FA
:108D30001D066B017C01C150F9F6CF91FF90EF90B9
:108D4000DF90CF90BF90AF909F908F9008951F922B
:108D50000F920FB60F9211240BB60F922F938F9391
:108D60009F93EF93FF93E091F01981E08E0F8F773F
:108D70009091C6002091F119821731F0F0E0E0598E
:108D8000F64E90838093F019FF91EF919F918F9110
:108D90002F910F900BBE0F900FBE0F901F90189544
:108DA0002F923F924F925F926F927F928F929F92FB
:108DB000AF92BF92CF92DF92EF92FF920F931F93E9
:108DC000CF93DF93CDB7DEB764970FB6F894DEBFCD
:108DD0000FBECDBF85E49FDA882321F069DA6B01ED
:108DE0007C0105C0C12CD12CE12C30ECF32E8AE59E
:108DF000C1DA882321F05CDA2B013C0103C0412C4D
:108E0000512C320188E5B6DA882311F051DA03C01B
:108E100060E070E0CB0169877A878B879C8789E562
:108E2000A9DA882311F044DA03C060E070E0CB01D6
:108E30006D877E878F87988B85E56DDA882321F093
:108E400037DA4B015C0106C0812C912C28ECA22E54
:108E500022ECB22E8CE45FDA882331F029DA698BB8
:108E60007A8B8B8B9C8B04C0198A1A8A1B8A1C8A6A
:108E700082E480DA882319F0EBD9162F01C015E0BF
:108E800020900F13309010138091FD1981119BC217
:108E90008091CF1583FD3CC020E030E0A901C501E1
:108EA000B4010E9484FF811109C020E030E0A901D3
:108EB000C701B6010E9484FF882351F1809163129B
:108EC000811124C02091220E3091230E809127021F
:108ED0009091280228173907CCF4E9ECF6E1849147
:108EE0007F019FEFE91AF90A882319F0CDDAF7011B
:108EF000F6CFE3EAF9E084917F019FEFE91AF90ADE
:108F0000882309F460C2C0DAF701F5CF0E94BA3DA8
:108F100081E08093FD1990911F13992321F0109205
:108F20001F13809307060E9416E081E080932E10A5
:108F300040E050E0BA0180EF98E98CD20E9476754B
:108F400080E1EEE4F8E1A8E0B6E001900D928A95A8
:108F5000E1F720E030E0A901C701B6010E9484FFDB
:108F60008823F1F00E947D3FA70196016091551280
:108F70007091561280915712909158120F941E06BC
:108F80006093551270935612809357129093581213
:108F900060E070E080E792E40E94913F0E94767565
:108FA00020E030E0A901C301B2010F944408181673
:108FB00024F580E090E0A0EAB0E48D839E83AF8347
:108FC000B887A3019201609156187091571880914B
:108FD0005818909159180F941E0669837A838B83D1
:108FE0009C839E012B5F3F4FAE014F5F5F4F62E559
:108FF00078E18EE498E10E948E3E80E090E0A8EC5B
:10900000B2E489839A83AB83BC839E012F5F3F4F79
:1090100046E558E1BE01635F7F4FCE0109960E948D
:109020008E3E20E030E0A901C501B4010E9484FF1A
:10903000882351F181E080932E1040E050E0BA0186
:109040008DE598E907D280E00E94F6E70E947D3F17
:10905000A50194016091551270915612809157129A
:10906000909158120F941E066093551270935612E9
:10907000809357129093581260E070E080E291E480
:109080000E94913F0E94767501E000932E1040E00F
:1090900050E0BA0184EA96E9DDD161E0812F0E94B7
:1090A000183E80E00E94F6E70E94F4E764E670E074
:1090B00080E090E00E9423C60E9486C2DC01CB01C2
:1090C00088539045AF4FBF4F8093B10D9093B20D31
:1090D000A093B30DB093B40D1092210683E090E0FD
:1090E0009093F7198093F6190093371080913710F9
:1090F000882309F44CC060E0812F0E94183E8091C3
:109100002106882309F43FC000932E1040E050E070
:10911000BA0187E397E99ED18091371081112FC062
:109120001092B10D1092B20D1092B30D1092B40DB9
:10913000109221060E947DA80E94BA3D00932E1035
:1091400040E050E0BA0184EA96E984D10E9486C2E8
:10915000DC01CB0188539045AF4FBF4F8093B10DD9
:109160009093B20DA093B30DB093B40D109221065D
:109170000093371061E0812F0E94183E04C081E007
:109180000E94F6E7C9CF81E00E94F6E7AFCF81E009
:1091900090E09093F7198093F6198091FD19882338
:1091A00009F411C1F09021061092B10D1092B20D88
:1091B0001092B30D1092B40D1092210680E00E941F
:1091C0007DA8F1100E94BA3D61E0812F0E94183EF7
:1091D0000E947D3F20E030E0A90169897A898B896E
:1091E0009C890E9484FF882309F446C0FF2049F02F
:1091F00081E080932E1040E050E0BA0184EA96E9C5
:1092000029D183E090E09093F7198093F61981E0DB
:109210008093371080913710882311F0F110D9C056
:1092200081E090E09093F7198093F61980932E10C7
:1092300040E050E0BA0181E196E90CD129893A89F0
:109240004B895C896091551270915612809157122A
:10925000909158120F941E066093551270935612F7
:10926000809357129093581260E070E080EC90E485
:109270000E94913F0E94767511E083E0C82ED12CA8
:10928000EE24E394F12C10932E1040E050E0BA014C
:109290008EE795E9DFD020E030E048E452E46091C9
:1092A00055127091561280915712909158120F9446
:1092B0001E06609355127093561280935712909326
:1092C000581260E070E080E490E40E94913F0E94B8
:1092D0007675D092F719C092F61910923710109344
:1092E0002E101092D70F1092D60F40E050E0BA0126
:1092F00083E899E9AFD08091D60F9091D70F00976E
:1093000021F481E00E94F6E7F6CFF092F719E0929F
:10931000F619019709F4B7CF11E010932E1040E031
:1093200050E0BA018DE095E995D0809114069091B6
:109330001506A0911606B091170680935A189093BF
:109340005B18A0935C18B0935D18809355129093AE
:109350005612A0935712B09358120E9430E080E04A
:1093600090E0A8ECB2E489839A83AB83BC839E012E
:109370002F5F3F4F46E558E16CE076E088E096E0ED
:109380000E948E3E80E090E0A0EAB0E489839A8358
:10939000AB83BC839E012F5F3F4F40E156E062E507
:1093A00078E18EE498E10E948E3E77D080910706A6
:1093B000882339F080912013811110931F1310928C
:1093C00007061092FD192A94232859F40E946EE092
:1093D00008C060E0812F0E94183E81E00E94F6E7FD
:1093E00019CF64960FB6F894DEBF0FBECDBFDF91E4
:1093F000CF911F910F91FF90EF90DF90CF90BF9092
:10940000AF909F908F907F906F905F904F903F9024
:109410002F900895809147068630D8F496E0899F72
:10942000F0011124ED5DF94F20917A0230917B0219
:10943000318320834091D6155091D7156091D8156E
:109440007091D91542835383648375838F5F8093B2
:109450004706089520917A0230917B022817390738
:10946000D9F090937B0280937A024093D615509363
:10947000D7156093D8157093D915855A9B4421F45C
:1094800010922E101092470682E080932A0281E00B
:109490008093D80F10923510089540E050E0BA0143
:1094A00085EA9BE4D7CFE0914706EE2381F0E150B7
:1094B000E093470686E0E89FF0011124ED5DF94F47
:1094C000428153816481758180819181C3CFE5CFD1
:1094D000CF93DF9380912A02882349F06091230281
:1094E0007091240220E041E081E00E9493DF8091AE
:1094F0002206811118C081E080932206C0917A0271
:10950000D0917B0240E050E0BA0188E69AE4A2DF05
:109510000E9476751092220640E050E0BA01CE011A
:10952000DF91CF9197CFDF91CF910895CF92DF92C6
:10953000EF92FF920F931F93CF93DF939C017B01D8
:1095400080E090E0F901E80FF91FE491EE2311F0BB
:109550000196F8CFF701AF014E195F0961916111D2
:10956000FACF04E110E0041B110999270817190725
:109570001CF0DD24D39402C082E0D82E8091921298
:1095800090E06D2D70E06F5F7F4F0F94FA08C62E4C
:10959000C6E0C60F8091C512C81748F04091C712A7
:1095A00050E08C2F90E00B97481759078CF5D0E0CE
:1095B000E114F104B1F18AE30E940CD982E0D812DF
:1095C0000FC0CC0D8091C512C81758F12091C71259
:1095D00030E08C2F90E00B97281739071CF421C03E
:1095E000DD23F9F0802F880F080F000F0093C812B9
:1095F000C093C91280E20E940CD9C701DF91CF91BC
:109600001F910F91FF90EF90DF90CF900C9481AC61
:109610001092C812C093C912C9010E9474ACD1E063
:10962000C7CFDF91CF911F910F91FF90EF90DF9007
:10963000CF9008959CE0899F802D112491E0980F90
:1096400090936E182CE0280F20936F184091C5124C
:1096500050E030E02E5F3F4F24173507CCF0292F24
:1096600030E04091C71250E0241735078CF4662390
:1096700041F08E5F0E947DDF80916F188E5F0E94A7
:109680007DDF80916F181092C8128093C9120895DF
:109690000895FF920F931F93CF93DF931F92CDB73F
:1096A000DEB783E690E00F949B05809364128130CF
:1096B00011F4809359068091CA12811105C081E08E
:1096C0008093CA120E9472D9609193127091941281
:1096D00019829E012F5F3F4F4FE081E992E10E9486
:1096E0000EC380910002882349F1109200028091FC
:1096F000911290E08058910997FD01969595879574
:10970000182F0E94D9D934E0F32E00E420E840E07D
:10971000612F81E992E10E942AC3882339F02CEC61
:1097200039E040E460E0812F0E940BDA0E94B8C665
:10973000F0922F100E94D2D88111E7CF0F90DF91C5
:10974000CF911F910F91FF9008952F923F924F92CA
:109750005F927F928F929F92AF92BF92CF92DF9251
:10976000EF92FF920F931F93CF93DF93CDB7DEB7A6
:109770002A970FB6F894DEBF0FBECDBF10923410FB
:1097800080913610882341F084DF40E050E0BA0138
:1097900085EB98EC5FDE2DC54091D6155091D7151D
:1097A0006091D8157091D915209170023091710295
:1097B000C901840F951F2436310524F4853691059F
:1097C0003CF416C02436310531F08436910584F41A
:1097D00084E690E00DC0473051056105710514F035
:1097E000069706C04A3F5F4F6F4F7F4F6CF4069657
:1097F00090937102809370021092D6151092D71533
:109800001092D8151092D915809170029091710222
:109810008A3091053CF0883E23E092072CF087EED9
:1098200093E002C08AE090E090937102809370020E
:109830000E949DB4182F0E94B8C681E080932F101B
:109840008091C512853108F5112359F08091EB15EF
:109850009091EC15892B29F0B5E2EB2EBFE0FB2EA1
:1098600004C0A5EFEA2EADE0FA2E03E120E841E0C6
:1098700060E081E992E10E942AC3882331F09701D8
:1098800043E161E080E00E940BDA8091C5128D31E6
:1098900008F07DC1883008F041C080912106112375
:1098A000D9F16091220E7091230E072E000C880BC7
:1098B000990B0E948AFF20E030E040E05FE30F94C4
:1098C0001E060F9462079B01643671051CF52A3051
:1098D0003105F4F04CE022E130E0241B310937FF80
:1098E00002C02F5F3F4F359527953195219531095E
:1098F0002A5D2093C81227E02093C912CB010E9451
:10990000EDC50E9481AC82EF9DE00E9474AC06C060
:1099100046E0E1CF42E1DFCF882319F28091C51202
:109920008D31D0F58091C7128531B0F120E030E063
:1099300040E05FE360915F1270916012809161126C
:10994000909162120F941E060F9462079B01643679
:1099500071050CF023C32A3031050CF41DC34CE013
:1099600022E130E0241B310937FF02C02F5F3F4F57
:10997000359527953195219531092A5D2093C81297
:109980002CE12093C912CB010E94EDC50E9481AC4D
:1099900082EF9DE00E9474AC8091C512853108F57C
:1099A0008091C7128131E8F06091220E7091230EF0
:1099B000072E000C880B990B0E948AFF20915F12E2
:1099C0003091601240916112509162120F944408DC
:1099D00018160CF4E5C222E042E061E18EE20E943A
:1099E00038E18091C512883008F03FC08091200690
:1099F000111102C0811139C06091E9157091EA1509
:109A0000072E000C880B990B0E948AFF20E030E0A3
:109A100040E05FE30F941E060F9462076436710501
:109A20002CF46A30710524F446E003C042E101C021
:109A30004CE022E130E0241B310937FF02C02F5FE8
:109A40003F4F35952795319521953109285B209316
:109A5000C81227E02093C912CB010E94EDC50E94D5
:109A600081AC82EF9DE00E9474AC8091C5128D3173
:109A7000D0F58091C7128531B0F120E030E040E0B0
:109A80005FE360911C0670911D0680911E06909107
:109A90001F060F941E060F9462079B016436710522
:109AA0000CF08CC22A3031050CF086C246E022E16F
:109AB00030E0241B310937FF02C02F5F3F4F35953F
:109AC0002795319521953109285B2093C8122CE107
:109AD0002093C912CB010E94EDC50E9481AC82EF98
:109AE0009DE00E9474AC8091C512853130F5809163
:109AF000C712813110F16091E9157091EA15072EB6
:109B0000000C880B990B0E948AFF20911C06309153
:109B10001D0640911E0650911F060F94440818160A
:109B20000CF04EC21092B11222E042E062E18FE4EA
:109B30000E9438E181E08093B1128091C5128C318E
:109B400030F58091C712843110F18091EB1590911E
:109B5000EC15019644E6489F9001499F300D112471
:109B600037FF02C021503F4F832F932F990F990B3E
:109B7000009769F028E62093C8122BE12093C912C0
:109B80000E94EDC50E9481AC85E20E940CD94091F3
:109B90005906642F70E02091C51230E083E390E015
:109BA000861B970B821793075CF02091C71230E059
:109BB0008AE290E0861B970B281739070CF007C242
:109BC000409159062091C51230E084E390E0841B57
:109BD0009109821793072CF08091C712813308F006
:109BE00024C280911F13882309F453C04091590661
:109BF0002091C51230E083E390E0841B9109821725
:109C000093070CF446C08091C712823308F441C018
:109C100002E0041B2091ED14222319F18091B61566
:109C20009091B715A091B815B091B9150097A105FD
:109C3000B10509F402C2BC01CD016D597F4F8F4FB0
:109C40009F4F24E630E040E050E00F94C005609163
:109C5000BA157091BB158091BC159091BD150F94EC
:109C6000C00585E3289FB0011124072E000C880B46
:109C7000990B0E948AFF2AE037ED43E25CE30E94E1
:109C8000E9FF0F946707462F202F62E387E30E94C6
:109C900038E18091C512813308F079C08091C712F4
:109CA000893208F474C00E944C6D4B015C0120E1C4
:109CB0003EE040E050E00F94C005722E032FE22EEC
:109CC000F32E8CE3282E312C412C512CC501B401EC
:109CD000A20191010F94C005CA01B901A20191012D
:109CE0000F94C005CE0101966C0191E8891691E5AB
:109CF000990691E0A906B10408F4A1C17F936F937E
:109D0000C70168E170E00F94E6089F938F93C50147
:109D1000B40120E831E541E050E00F94C0053F93E5
:109D20002F938EED9DE09F938F93DF92CF920E94B1
:109D30001EFF0FB6F894DEBF0FBECDBF8CE380933D
:109D4000C81280E38093C912C6010E9481AC809141
:109D50001D0E90911E0EA0911F0EB091200E892B0A
:109D60008A2B8B2B09F4ADC12091ED14211184C1F4
:109D700088E68093C81283E38093C912822F90E013
:109D80000E94EDC50E9426E185E20E940CD9E09177
:109D90008B12F0918C1284818111CCC060914E188D
:109DA00070914F1880915018909151180F9462073C
:109DB000CB010E946CC5BC0184E596E00F94760946
:109DC00060915218709153188091541890915518C1
:109DD0000F946207CB010E946CC5BC018FE496E032
:109DE0000F9476092CEA35EC47E257E36091561858
:109DF0007091571880915818909159180F941E0619
:109E000020E030E048EC52E40E94E9FF0F94620742
:109E10006B017C0197FD19C090E1C91697E2D90644
:109E2000E104F104E4F0C701B60120E137E240E0CB
:109E300050E00F94E205CA01B9012AE030E040E0A9
:109E400050E00F94E205605D0BC0F094E094D09474
:109E5000C094C11CD11CE11CF11C6DE201C060E288
:109E60006093EE1528EEC21623E0D206E104F10459
:109E700094F0C701B60128EE33E040E050E00F94C3
:109E8000E205CA01B9012AE030E040E050E00F9459
:109E9000E205605D01C060E26093EF15C701B601A5
:109EA00024E630E040E050E00F94E2059AE0892E8D
:109EB000912CA12CB12CCA01B901A50194010F94D8
:109EC000E205605D6093F015C701B601A50194013C
:109ED0000F94E205062F662381F08EE28093F11540
:109EE000CA01B901A50194010F94E205605D609378
:109EF000F215005D0093F31517C0CA01B901A50161
:109F000094010F94E205662339F08EE28093F115F7
:109F1000605D6093F21505C080E28093F215809336
:109F2000F11580E28093F3156EEE75E188E496E01A
:109F30000F9476098091C512883298F48091C712E7
:109F40008D3178F02BE040E86DE180E00E94F4E094
:109F50008091C512873228F48091C7128F3108F0A2
:109F6000B9C08091C512823328F48091C7128B3218
:109F700008F01BC18091C512803408F03AC180916D
:109F8000C712883308F435C11092C8128FE380934A
:109F9000C9120E945ED92DC146E0E2CC42E1E0CC7C
:109FA0001092B11222E042E061E18EE20E9438E1BB
:109FB00081E08093B11215CD4CE079CD42E177CDAF
:109FC00022E042E062E18FE40E9438E1B6CD6AE22D
:109FD000641B27E048E08AE20E9438E1809159063C
:109FE0006CE2681B25E042E082E30E9438E1809148
:109FF000590661E3681B24E04AE08AE20E94F4E02B
:10A00000909159068BE2891B609193127091941282
:10A0100092E39093AD128093AE122DEA32E142E3C7
:10A0200081E992E10E940EC3CBCD24E0241B45E3DD
:10A0300061E386E30E94F4E0D4CD20E012CE94E602
:10A04000E916F10460F47F936F93C70168E170E053
:10A050000F94E6089F938F9384ED9DE006C07F9355
:10A060006F930F937F928CEC9DE09F938F93DF9281
:10A07000CF920E941EFF5DCE8091B6159091B715CC
:10A08000A091B815B091B9150097A105B105B9F027
:10A09000BC01CD016D597F4F8F4F9F4F24E630E0BB
:10A0A00040E050E00F94C0056091BA157091BB1567
:10A0B0008091BC159091BD150F94C00559CE20E03C
:10A0C00057CE88E68093C81283E38093C91280E05C
:10A0D00090E056CE83E08093C81286E28093C91246
:10A0E000112329F080EF9DE00E9474AC0DC0809197
:10A0F0001906811102C08FE305C080910A0E8111FB
:10A10000F1CF80E20E940CD98BE08093C81206E266
:10A110000093C91284E596E00E9481AC8BE28093A3
:10A12000C8120093C912112329F08EEE9DE00E94FF
:10A1300074AC0DC080911A06811102C08FE305C076
:10A1400080910B0E8111F1CF80E20E940CD983E344
:10A150008093C81206E20093C9128FE496E00E9431
:10A1600081AC83E58093C8120093C912112329F0B2
:10A170008CEE9DE00E9474AC0DC080911B06811195
:10A1800002C08FE305C080910C0E8111F1CF80E2F7
:10A190000E940CD98BE58093C81286E28093C91285
:10A1A00088E496E00E9481ACDCCE0E94B8C684E0D0
:10A1B00080932F1083E08093C81212E31093C9128A
:10A1C00086E00E9460AC0E94B8C681E080932F10A8
:10A1D0008CE08093C8121093C91280917002909104
:10A1E00071020E94EDC50E9481AC85E20E940CD9EB
:10A1F000C1CE2A960FB6F894DEBF0FBECDBFDF9159
:10A20000CF911F910F91FF90EF90DF90CF90BF9073
:10A21000AF909F908F907F905F904F903F902F9046
:10A220000895CF93DF9380913610882319F0DF9142
:10A23000CF9139C9109234108091D6159091D715CD
:10A24000A091D815B091D91581309048A105B105DC
:10A2500040F01092D6151092D7151092D815109282
:10A26000D915C091D6158091630618160CF5282FC4
:10A27000082E000C330B255031094C2F0C2E000CEE
:10A28000550B42175307A4F085301CF0CBEFC80FD5
:10A2900001C0C0E08C2F0C2E000C990BAA0BBB0B3D
:10A2A0008093D6159093D715A093D815B093D91550
:10A2B000C093D90FD0E0C11114C080912A02882325
:10A2C000D9F180916412882341F0813019F462EA57
:10A2D00071E105C064E971E102C060EB71E121E068
:10A2E00027C0C13049F480912A02882329F120E057
:10A2F00041E06BE572E11DC0C23049F480912A0251
:10A300008823D1F020E041E063E572E112C0C33060
:10A31000F1F0C43059F580912A02882369F08091C8
:10A320006412882301F18130D9F460ED71E120E0FD
:10A3300041E08D2F0E9493DFDF5FCF5FD53009F0C2
:10A34000BACF88E080936306DF91CF910895809122
:10A350002A02882389F320E041E06AE472E1E9CF30
:10A360006EEB71E1E4CF6FED71E1E1CFC53099F4AF
:10A3700080912A02882301F380916412882341F09E
:10A38000813019F46DEF71E1D2CF61EF71E1CFCF80
:10A3900069E072E1CCCFC63049F480912A0288236B
:10A3A00059F220E041E06CE372E1C3CFC73021F6FF
:10A3B00080912A02882309F4BFCF809164128823F8
:10A3C00041F0813019F462E272E1B1CF65E172E1EE
:10A3D000AECF6FE272E1ABCF3F924F925F926F923E
:10A3E0007F928F929F92AF92BF92CF92DF92EF9225
:10A3F000FF920F931F93CF93DF93109234108091AD
:10A40000D6159091D715A091D815B091D915813056
:10A410009048A105B10540F01092D6151092D715BD
:10A420001092D8151092D915C091D6158091610659
:10A430001816DCF4282F082E000C330B215031099C
:10A440004C2F0C2E000C550B4217530774F0CFEF16
:10A45000C80F8C2F90E0A0E0B0E08093D6159093C9
:10A46000D715A093D815B093D9151092D80F809115
:10A47000D90FC81714F4C093D90F8091D90F082EA3
:10A48000000C990B04962C2F0C2E000C330B82170A
:10A49000930724F48CEF8C0F8093D90F3090D90F51
:10A4A000D0E03CED832E35E0932EA12CB12C46ED6F
:10A4B000442E46E0542E612C712C5FEAC52E57EED7
:10A4C000D52E31101EC080913610811106C08091AA
:10A4D0002A02882309F451C009C0C111F8CF0E9493
:10A4E000534A8091D80F882391F3EFC00E94F3F470
:10A4F000AC0181E0C11180E024E06D2F0E9479C69B
:10A500003CC081E0381239C080913610811105C0FD
:10A5100080912A02811112C030C0C130C9F78091E8
:10A520005E068C2780935E0683E080932A020E9459
:10A53000AFE78091D80F882359F3C7C080915E069A
:10A54000811103C022E731E102C026E731E18091A9
:10A550006412882341F0813019F442E451E105C0CE
:10A5600049E351E102C04BE451E181E0C13009F01F
:10A5700080E001E06D2F0E9489EE80915E068823C5
:10A5800009F49BC092E0391296C080913610811177
:10A5900006C080912A02882309F48DC06AC0C230A7
:10A5A000C1F781E080933410109230101092311076
:10A5B000109232101092331080916412882341F06F
:10A5C000813019F40EE511E105C004E511E102C086
:10A5D00008E611E10E940A4A83E080932A02109360
:10A5E000E5150093E4158AE596E09093E3158093D2
:10A5F000E2158092DE159092DF15A092E015B092E0
:10A60000E1154092DA155092DB156092DC157092DC
:10A61000DD1520E030E04AE754E460915A0670917D
:10A620005B0680915C0690915D060E94E9FF20E048
:10A6300030E84BEB54E40F941D060F9467076093CA
:10A64000D6157093D7158093D8159093D9158FE6AA
:10A6500090EB90937B0280937A02D092E815C0929F
:10A66000E7151092E6158091D80F882309F491CF51
:10A670002CC080916412882361F0813029F42EE58A
:10A68000E22E21E1F22E09C094E5E92E91E1F92EA6
:10A6900004C088E6E82E81E1F82E8AE596E00E9463
:10A6A0005BE19C0181E0C23009F080E000E0A7019D
:10A6B0006D2F0E9489EE83E001C082E0DF5F33945A
:10A6C000D53009F0FECE80936106DF91CF911F91C6
:10A6D0000F91FF90EF90DF90CF90BF90AF909F9041
:10A6E0008F907F906F905F904F903F9008951F9351
:10A6F000CF93DF93109234108091D6159091D71597
:10A70000A091D815B091D91581309048A105B10517
:10A7100040F01092D6151092D7151092D8151092BD
:10A72000D915C091D615809160061816DCF4282F33
:10A73000082E000C330B215031094C2F0C2E000C2D
:10A74000550B4217530774F0CFEFC80F8C2F90E0D2
:10A75000A0E0B0E08093D6159093D715A093D815BC
:10A76000B093D9151092D80F8091D90FC81714F44F
:10A77000C093D90F8091D90F082E000C990B049625
:10A780002C2F0C2E000C330B8217930724F48CEF24
:10A790008C0F8093D90F1091D90FD0E011111BC0ED
:10A7A00080913610811106C080912A02882309F415
:10A7B0007DC009C0C111F8CF0E94534A8091D80FC3
:10A7C000882391F3B5C00E94F3F4AC0181E0C1117C
:10A7D00080E024E068C0113039F580913610811195
:10A7E00006C080912A02882309F460C00BC0C130E2
:10A7F000C1F78DEC91E60E94F2B48091D80F8823C6
:10A8000081F396C080916412882341F0813019F45D
:10A8100046ED50E105C04DEC50E102C04FED50E176
:10A8200081E0C130F1F53EC0123031F58091361033
:10A83000811105C080912A028823C1F10BC0C2306A
:10A84000C9F78CEC96E60E94F2B48091D80F882369
:10A8500089F36EC080916412882341F0813019F42D
:10A8600045EF50E105C048EE50E102C042E051E141
:10A8700081E0C230B1F416C0133089F580913610F2
:10A8800081111CC080912A02882381F0809164127A
:10A89000882311F18130E9F444E151E181E0C330D2
:10A8A00009F080E023E06D2F0E9479C6DF5F1F5F13
:10A8B000D53009F073CFD09360063AC0C33011F79A
:10A8C00081E894E60E94F2B48091D80F8823D1F2F7
:10A8D0002FC04FE051E1E2CF49E151E1DFCF143029
:10A8E00029F780913610811105C080912A028823B2
:10A8F000E9F20BC0C430C9F78CE994E50E94F2B4C8
:10A900008091D80F882389F313C080916412882323
:10A9100041F0813019F447E251E105C04EE151E1C7
:10A9200002C040E351E181E0C43009F0BACFBACFB0
:10A93000DF91CF911F910895CF92DF92FF920F93F5
:10A940001F93CF93DF93109234108091D61590917E
:10A95000D715A091D815B091D91581309048A1058F
:10A96000B10540F01092D6151092D7151092D81557
:10A970001092D915C091D61580915F061816DCF497
:10A98000282F082E000C330B215031094C2F0C2E90
:10A99000000C550B4217530774F0CFEFC80F8C2FE4
:10A9A00090E0A0E0B0E08093D6159093D715A093E7
:10A9B000D815B093D9151092D80F8091D90FC81718
:10A9C00014F4C093D90F8091D90F082E000C990B65
:10A9D00004962C2F0C2E000C330B8217930724F4B3
:10A9E0008CEF8C0F8093D90F1091D90FD0E0FF24FA
:10A9F000F39411111EC080913610811106C0809110
:10AA00002A02882309F4D4C009C0C111F8CF0E94DA
:10AA1000534A8091D80F882391F34DC10E94E4F4EA
:10AA2000AC0181E0C11180E024E06D2F0E9479C665
:10AA3000BFC0113009F04BC080913610811106C0A3
:10AA400080912A02882309F4B3C023C0C130C1F722
:10AA5000C0933410109230101092311010923210B6
:10AA60001092331080916412882341F0813019F4E0
:10AA70008FE590E105C085E590E102C089E690E1AF
:10AA80006EE578E10E94C3F98091D80F8823C1F266
:10AA900012C180916412882361F0813029F4BFE5EE
:10AAA000CB2EB0E1DB2E09C0A5E5CA2EA0E1DA2E3F
:10AAB00004C0F9E6CF2EF0E1DF2E8EE598E10E948A
:10AAC0004CC39C0181E0C13009F06CC06CC01230F5
:10AAD00009F04AC080913610811106C080912A0287
:10AAE000882309F465C023C0C230C1F7F092341046
:10AAF00010923010109231101092321010923310C8
:10AB000080916412882341F0813019F48DE790E13F
:10AB100005C083E790E102C087E890E162E678E152
:10AB20000E94C3F98091D80F8823C1F2C4C08091DC
:10AB30006412882361F0813029F4EDE7CE2EE0E144
:10AB4000DE2E09C073E7C72E70E1D72E04C067E878
:10AB5000C62E60E1D62E82E698E10E944CC39C018D
:10AB600081E0C230F9F41FC0133009F057C0809162
:10AB70003610811125C080912A028823C9F0809166
:10AB80006412882309F445C08130F1F55BE9C52ED4
:10AB900050E1D52E86E698E10E944CC39C0181E0ED
:10ABA000C33009F080E000E0A6016D2F0E9489EE1D
:10ABB000DF5F1F5FD53009F01CCFD0935F067BC0ED
:10ABC000C330C9F6F0923410109230101092311048
:10ABD000109232101092331080916412882341F049
:10ABE000813019F48BE990E105C081E990E102C060
:10ABF00085EA90E166E678E10E94C3F98091D80F7A
:10AC0000882309F4B8CF57C041E9C42E40E1D42EBF
:10AC1000C1CF35EAC32E30E1D32EBCCF143041F67C
:10AC200080913610811106C080912A02882309F490
:10AC3000BFCF23C0C430C1F7F0923410109230104F
:10AC400010923110109232101092331080916412D1
:10AC5000882341F0813019F489EB90E105C08FEA37
:10AC600090E102C083EC90E16AE678E10E94C3F9CA
:10AC70008091D80F8823C1F21EC08091641288236E
:10AC800061F0813029F429EBC22E20E1D22E09C0D7
:10AC90009FEAC92E90E1D92E04C083ECC82E80E132
:10ACA000D82E8AE698E10E944CC39C0181E0C43012
:10ACB00009F078CF78CFDF91CF911F910F91FF905E
:10ACC000DF90CF900895AF92BF92CF92DF92EF9234
:10ACD000FF920F931F93CF93DF93CDB7DEB76F979C
:10ACE0000FB6F894DEBF0FBECDBF80912A0281114E
:10ACF00005C080913610882309F4B9C18DE693E12F
:10AD000090936C1380936B1381E090E09093C41543
:10AD10008093C3151092C6151092C51581E793E173
:10AD20000E94C9B680916B1390916C132BE1FC01CA
:10AD30003496DE01159601900D922A95E1F7FC01FB
:10AD4000828193819C838B838FE992E09A838983AC
:10AD500040E050E0BE016F5F7F4F89E095E00E94C8
:10AD6000826DCE0101960E9454BDC090C515D09051
:10AD7000C615109234108091D6159091D715A091D8
:10AD8000D815B091D91581309048A105B10540F092
:10AD90001092D6151092D7151092D8151092D91579
:10ADA0001091D615809162061816DCF4282F082E13
:10ADB000000C330B21503109412F012E000C550B93
:10ADC0004217530774F01FEF180F812F90E0A0E097
:10ADD000B0E08093D6159093D715A093D815B09373
:10ADE000D9151092D80F8091D90F181714F4109319
:10ADF000D90F8091D90F082E000C990B0496212FA2
:10AE0000012E000C330B8217930724F48CEF810F73
:10AE10008093D90FE090D90FF12CE1101CC08091E4
:10AE20003610811105C080912A028823A1F009C043
:10AE30001111F9CF0E94534A8091D80F882399F3BA
:10AE400016C10E942FF5AC0181E0111180E024E0D1
:10AE50006F2D0E9479C662E273E181E793E10E945F
:10AE600091B5809122138F32C9F121E0E21238C0EE
:10AE700080913610882319F1113009F58091C214A0
:10AE80008823D1F081508093C214EFE18E9FC001DE
:10AE90001124FC01E057FC4E2BE1A1E7B3E1019046
:10AEA0000D922A95E1F7FC01E457FC4E82819381D3
:10AEB0009093701380936F131092D90FA4C0809158
:10AEC0002A02882369F081E0113009F080E020E255
:10AED00040E951E16F2D0E9479C602C001E001C036
:10AEE00002E05601F1E0AF1AB10808F4B9C00E1142
:10AEF000B5C060E070E0C5010E943A6F90912113E7
:10AF000080913610992309F48EC0882309F482C0F9
:10AF1000101380C0CE0101960E94C3E28091741389
:10AF2000882319F00DE613E102C00CE413E1780167
:10AF300084E0E80EF11C21E042E253E1B701CE01CA
:10AF400005960E94FABA811126C0EBE9F9E48491D2
:10AF50008F010F5F1F4F882321F00E944442F801A8
:10AF6000F6CFEAE7F1E184918F010F5F1F4F88234D
:10AF700021F00E944442F801F6CF02E213E1F80109
:10AF800081918F01882319F00E944442F8CF8AE012
:10AF90000E9444422CC08091C2148A30C8F491E0CF
:10AFA000980F9093C214FFE18F9FC0011124DC0120
:10AFB000A057BC4E2BE1F70101900D922A95E1F7C5
:10AFC000F80122813381FC01E457FC4E3383228354
:10AFD0008BE1FE013596A1E7B3E101900D928A95D0
:10AFE000E1F78B819C819093701380936F13CE0156
:10AFF00001960E9454BD1092D6151092D71510924A
:10B00000D8151092D91581E08093D80F83E08093F2
:10B010002A022DC080912A02882301F181E01E11AD
:10B0200080E041E018C0811105C080912A02882388
:10B03000A9F00DC01013F9CF82E293E10E94F96AE2
:10B040000E944D4A8091D80F882379F310C081E087
:10B050001E1180E040E06F2D0E94D3F80F5F42CFB9
:10B06000F394E39425E0F212D8CE009362066F9633
:10B070000FB6F894DEBF0FBECDBFDF91CF911F9109
:10B080000F91FF90EF90DF90CF90BF90AF90089519
:10B09000FF920F931F93CF93DF938C01EB01F42E5C
:10B0A00080E20E9444428FEFF81611F084E501C05F
:10B0B00082E40E9444428AE30E944442F801608193
:10B0C00071818281938142E00E9436464881598194
:10B0D0006A817B8187E692E1DF91CF911F910F9189
:10B0E000FF900C9430EC88E893E19093960D809358
:10B0F000950D80916F008D7F80936F009091EF127E
:10B100008091F012981719F00E9406ECF7CF109278
:10B11000980D1092970D80916F00826080936F0060
:10B120008FB7F89410922A1010922B1010922C10B6
:10B1300010922D108FBF0E94767580E090E00E94E3
:10B1400057756093640670936506809366069093C6
:10B15000670681E090E00E945775609368067093DF
:10B16000690680936A0690936B0682E090E00E94E5
:10B17000577560936C0670936D0680936E0690937E
:10B180006F068CE0E4E6F6E0AEE4B8E101900D92E3
:10B190008A95E1F70C94B1404F925F926F927F9243
:10B1A0008F929F92AF92BF92CF92DF92EF92FF92D7
:10B1B000CF93DF93EAEDF2E18491EF0121968823AA
:10B1C00021F00E944442FE01F7CF60914E18709129
:10B1D0004F18809150189091511842E00E943646C5
:10B1E000E6EDF2E18491EF012196882321F00E949F
:10B1F0004442FE01F7CF609152187091531880912C
:10B2000054189091551842E00E943646E2EDF2E162
:10B210008491EF012196882321F00E944442FE018F
:10B22000F7CF6091561870915718809158189091E7
:10B23000591842E00E943646EEECF2E18491EF01AB
:10B240002196882321F00E944442FE01F7CF6091AD
:10B250005A1870915B1880915C1890915D1842E0CB
:10B260000E9436468FB7F89440903E1850903F1891
:10B270006090401870904118809042189090431848
:10B28000A0904418B0904518C0904618D090471828
:10B29000E0904818F09049188FBFE4ECF2E18491F7
:10B2A000EF012196882321F00E944442FE01F7CF4E
:10B2B000C301B2010E94F242E0ECF2E18491EF019D
:10B2C0002196882321F00E944442FE01F7CFC50158
:10B2D000B4010E94F242ECEBF2E18491EF0121967D
:10B2E000882321F00E944442FE01F7CFC701B60136
:10B2F0000E94F2428AE0DF91CF91FF90EF90DF90C1
:10B30000CF90BF90AF909F908F907F906F905F9005
:10B310004F900C9444420F931F93CF93DF93CDB77C
:10B32000DEB728970FB6F894DEBF0FBECDBF609191
:10B33000220E7091230E072E000C880B990B0E9491
:10B340008AFF6D837E838F83988780915F129091AF
:10B350006012A0916112B091621289839A83AB83CB
:10B36000BC834EEFBE016B5F7F4FCE01019690DE36
:10B370006091E9157091EA15072E000C880B990B66
:10B380000E948AFF6D837E838F83988780911C063D
:10B3900090911D06A0911E06B0911F0689839A8385
:10B3A000AB83BC834FEFBE016B5F7F4FCE01019635
:10B3B0006FDEEFE6F2E184918F010F5F1F4F88236C
:10B3C00021F00E944442F801F6CFE0918405F0E0BC
:10B3D000E85FFF4E608170E080E090E00E94F24202
:10B3E000EAE6F2E184918F010F5F1F4F882321F07D
:10B3F0000E944442F801F6CF6091071070E080E0AF
:10B4000090E00E94F24228960FB6F894DEBF0FBE7D
:10B41000CDBFDF91CF911F910F9108952F923F9251
:10B420004F925F926F927F928F929F92AF92BF9254
:10B43000CF92DF92EF92FF920F931F93CF93DF9300
:10B44000CDB7DEB7E1970FB6F894DEBF0FBECDBF24
:10B4500085E40E94BA41882321F00E9428418B0193
:10B4600002C000E010E083E40E94BA41882329F082
:10B470000E9428417BA76AA704C025E030E03BA7D3
:10B480002AA785E50E948B4189A3882319F00E9491
:10B49000494189A317FD07C0C12CD12CB6E1EB2E81
:10B4A000B3E4FB2E06C0C12CD12CACE8EA2EA2E4FA
:10B4B000FA2E83E50E94BA41882321F00E94584168
:10B4C0006B017C010115110511F4109284050E9495
:10B4D00086C22B013C01C8010196029748F141E662
:10B4E00053E05A834983A981BA818D91BA83A98394
:10B4F000882319F00E944442F6CF8AE0E1960FB605
:10B50000F894DEBF0FBECDBFDF91CF911F910F9199
:10B51000FF90EF90DF90CF90BF90AF909F908F9073
:10B520007F906F905F904F903F902F900C9444428B
:10B53000EAE8F3E0FA83E983A981BA818D91BA83BD
:10B54000A983882319F00E944442F6CF8AE00E9422
:10B5500044420E945AA88FE70F3FBFEF1B0719F420
:10B560008093071002C080930810C701B6010F94A2
:10B570006207072E000C880B990B0E948AFF6D8BC7
:10B580007E8B8F8B988F81E0809329024AA25BA2E9
:10B590006CA27DA24CA65DA66EA67FA6198EE0E4E5
:10B5A000EA8FFCE1FB8F26E42C8F1D8E1E8E1F8EF2
:10B5B00018A2198A1A8A1B8A1C8A1D861E861F8653
:10B5C000188AC12CD12C7601FFE78F2E912CA12C4B
:10B5D000B12C8FE790E0A0E0B0E08D839E83AF8335
:10B5E000B8871EA21FA218A619A691E099871C86EB
:10B5F0001B86212C312C19AA18AA80912902882394
:10B6000009F4CFC10E9486C269837A838B839C83AD
:10B6100080910610882309F4A0C00E9463A9011537
:10B62000110559F420905F1230906012A0916112C0
:10B63000A9ABB0916212B8AB0AC020901C06309042
:10B640001D06E0911E06E9ABF0911F06F8AB9101D3
:10B6500049A958A96D8D7E8D8F8D98A10E9484FF78
:10B6600087FF06C02D8E3E8E29A92F8F38A938A3BB
:10B67000298D3A8D4B8D5C8DB10189A998A90E94C5
:10B6800084FF87FF06C0298E3A8E49A94B8F58A99F
:10B690005C8F8985910149A958A96D897E89882384
:10B6A00009F441C08F89988D0E9484FF87FF55C09F
:10B6B00049815A816B817C81441955096609770952
:10B6C000DB01CA0188589341A109B109B7FD45C002
:10B6D0008D819E81AF81B88588199909AA09BB0916
:10B6E000B595A795979587950F3FEFEF1E0719F42E
:10B6F0008093071002C0809308104EA35FA368A731
:10B7000079A7FD89FD8F2E892E8F3F893F8F488D28
:10B7100048A389819A81AB81BC818AA39BA3ACA3F6
:10B72000BDA319861AC08F89988D0F9444081816E6
:10B73000A4F489819A81AB81BC812AA13BA14CA14F
:10B740005DA1821B930BA40BB50BAC01BD01485846
:10B7500053416109710977FF42C120E030E040EABE
:10B7600051E46D897E898F89988D0F941E06910111
:10B7700049A958A90E9484FF87FF0FC0EAE9F3E1B5
:10B780008491DF011196BA83A983882309F47BC2CF
:10B790000E944442E981FA81F3CF80E398EFAFEF52
:10B7A000BFEF2CA53DA54EA55FA5821B930BA40B57
:10B7B000B50B29813A814B815C81820F931FA41FB5
:10B7C000B51FB7FD0CC0A7DD8AE00E944442898105
:10B7D0009A81AB81BC818CA79DA7AEA7BFA78981A9
:10B7E0009A81AB81BC81880F991FAA1FBB1F2AA118
:10B7F0003BA14CA15DA1821B930BA40BB50B84193B
:10B800009509A609B70981349747AB41B10580F086
:10B81000ECE7F3E18491AF014F5F5F4F5A834983B7
:10B82000882309F430C20E944442E981FA81F2CFB0
:10B830008AA59BA5AB85BC858A179B070CF0AEC07B
:10B84000EFE1F3E184919F012F5F3F4F3A8329831A
:10B85000882329F00E944442E981FA81F3CF0F3F07
:10B860003FEF130729F049E055E05A83498304C0AC
:10B870008DE593E09A83898369817A818DE093E1F4
:10B880000E9466ECB701A60189E093E10E9430ECCA
:10B890008AE00E94444269817A8187EF92E10E94A6
:10B8A00066EC4D855E856F85788983EF92E10E9415
:10B8B00030EC8AE00E94444269817A8181EE92E113
:10B8C0000E9466EC49895A896B897C898DED92E1E9
:10B8D0000E9430EC8AE00E94444299A1992309F425
:10B8E000D2C10F3F1F4F69F5C092A10DD092A20D9A
:10B8F000E092A30DF092A40D2CEA35EC47E25EE352
:10B900006D857E858F8598890E94E9FF60939D0DE6
:10B9100070939E0D80939F0D9093A00D2CEA35ECB3
:10B9200047E25EE369897A898B899C890F94FA06DC
:10B930006093990D70939A0D80939B0D90939C0D3D
:10B94000A2C1C092A90DD092AA0DE092AB0DF092C7
:10B95000AC0D2CEA35EC47E25EE36D857E858F8584
:10B9600098890E94E9FF6093A50D7093A60D8093BE
:10B97000A70D9093A80D2CEA35EC47E25EE36989A8
:10B980007A898B899C890F94FA066093AD0D709328
:10B99000AE0D8093AF0D9093B00D75C10E9452B162
:10B9A0002CCE8091290281116EC1E1960FB6F894D8
:10B9B000DEBF0FBECDBFDF91CF911F910F91FF90E2
:10B9C000EF90DF90CF90BF90AF909F908F907F903F
:10B9D0006F905F904F903F902F900C945AA84B859A
:10B9E0005C85141615060CF024C14EA05FA068A457
:10B9F00079A4480E591E6A1E7B1E2EA13FA148A5A0
:10BA000059A5281B390B4A0B5B0BC501B4010F94D8
:10BA1000B105A30192010F94E2058D809E80AF8055
:10BA2000B884820E931EA41EB51E54E1851691049F
:10BA3000A104B1040CF18CEE88169104A104B104A8
:10BA40003CF490E889169104A104B10434F422C0B6
:10BA50005BEE852E912CA12CB12C8D829E82AF8223
:10BA6000B8862EEF30E040E050E0281939094A0945
:10BA70005B0949015A0112C084E190E0A0E0B0E006
:10BA80008D839E83AF83B88744E1842E912CA12CB3
:10BA9000B12C04C08D829E82AF82B886E6E0F4E1CC
:10BAA0008491DF011196BA87A987882329F00E9423
:10BAB0004442E985FA85F4CF6D817E818F81988536
:10BAC0000E94F242E1E0F4E184919F012F5F3F4F39
:10BAD0003A872987882329F00E944442E985FA851C
:10BAE000F3CFC501B4010E94F242498D5A8D6B8D8E
:10BAF0007C8D8AEF93E10E9430EC4D8D5E8D6F8DD1
:10BB000078A183EF93E10E9430EC4B855C85433054
:10BB100051050CF48EC0C501B4010E948AFF20E0DB
:10BB200030E040E850E40E94E9FF6B017C01298D80
:10BB30003A8D4B8D5C8D6D8D7E8D8F8D98A10F9480
:10BB40001D062BED3FE049E450E40E94E9FF20E0B0
:10BB500030E040E05FE30E94E9FF9B01AC01C701D8
:10BB6000B6010F94FA066B017C01C301B2010E9479
:10BB70008AFF2FE632E143E85AE30E94E9FF2B01F6
:10BB80003C01B701A6018DEE93E10E9430ECB301B8
:10BB9000A20187EE93E10E9430EC2AE939E949E1FC
:10BBA0005FE3C701B6010E94E9FF6B017C019B01C5
:10BBB000AC010F941E06A30192010F94FA066D8743
:10BBC0007E878F87988BA7019601C301B2010E94DF
:10BBD000E9FF20E030E040E05EE30E94E9FF698B8E
:10BBE0007A8B8B8B9C8BE7EDF3E184913F015FEFC8
:10BBF000651A750A882321F00E944442F301F5CFAB
:10BC0000B701A60181ED93E10E9430EC4D855E8580
:10BC10006F8578898BEC93E10E9430EC49895A89D1
:10BC20006B897C8985EC93E10E9430EC8AE00E946C
:10BC300044428D819E81AF81B885880D991DAA1DD2
:10BC4000BB1DB595A795979587950F3FEFEF1E07FD
:10BC500019F48093071002C0809308102B853C854F
:10BC60002F5F3F4F3C872B873D89398F4E894A8F05
:10BC70005F895B8F888D8C8F49805A806B807C8038
:10BC800091E099876ACDE1960FB6F894DEBF0FBEBA
:10BC9000CDBFDF91CF911F910F91FF90EF90DF907B
:10BCA000CF90BF90AF909F908F907F906F905F905C
:10BCB0004F903F902F9008952F923F924F925F9216
:10BCC0006F927F928F929F92AF92BF92CF92DF92AC
:10BCD000EF92FF920F931F93CF93DF93CDB7DEB711
:10BCE0002F970FB6F894DEBF0FBECDBF8091CF1552
:10BCF00083FD6FC160E08FEA92E10E943FC783E558
:10BD00000E94BA418887811106C082E50E94BA412B
:10BD1000882309F45EC10E9458410F9462076E3770
:10BD2000710514F06DE770E07093EA156093E91502
:10BD30000E940EA80E94584120E030E040EA50E402
:10BD40000F944408181614F40E946EE081E080936A
:10BD500029028091180680938405412C512C3201D0
:10BD60001C821D821E821F821B8219862CE32A8759
:10BD70003CE13B8746E44C8710E000E050E8598303
:10BD80008FEB8A83812C912C54016091E91570917D
:10BD9000EA15072E000C880B990B0E948AFF7B0185
:10BDA0008F879D879B01AC01612F702F89819A81BC
:10BDB0000E9484FF882309F449C020911C06309119
:10BDC0001D0640911E0650911F069885B7018F856C
:10BDD00091110EC09D850E9484FF881F8827881FAF
:10BDE0008B831E2D0F2DAF85A983BD85BA832EC0F1
:10BDF0009D850E9484FF87FF22C0809129028823AD
:10BE000009F4E7C060E081EA92E12F960FB6F8945A
:10BE1000DEBF0FBECDBFDF91CF911F910F91FF907D
:10BE2000EF90DF90CF90BF90AF909F908F907F90DA
:10BE30006F905F904F903F902F900C943FC71E2DB6
:10BE40000F2D2F8529833D853A831B820E9486C250
:10BE50006B017C01DC01CB012C813D814E815F8136
:10BE6000821B930BA40BB50BB7FD3BC0D701C601DA
:10BE700088519C4FAF4FBF4F8C839D83AE83BF8350
:10BE80004ADAEBEAF2E18491DF011196BE87AD87D1
:10BE9000882329F00E944442ED85FE85F4CF811469
:10BEA0009104A104B104B9F0D501C401805F984D9B
:10BEB000AF4FBF4FBC01CD016C197D098E099F09A1
:10BEC00028EE33E040E050E00F94C005CA01B9010C
:10BED0000E94F24203C08FE30E9444428AE00E9423
:10BEE000444280E00E94F6E70E94394220901C06FE
:10BEF00030901D06B0911E06BF8720911F062D872A
:10BF000091014B2F5D85612F702F89819A810F944C
:10BF10001D069F7781149104A104B10449F420E027
:10BF200030E040E85FE30E9484FF87FF0BC008C059
:10BF300020E030E040E450E40F944408181614F474
:10BF4000460157013B81332361F1411451046104DF
:10BF5000710441F0D701C60184199509A609B709F2
:10BF6000B7FD1FC091014F855D8569857A858B85F9
:10BF70009C850F941D0620E030E040EC5FE30E94BA
:10BF800084FF87FD3ACF2601370140E6440E4AEE92
:10BF9000541E611C711C29863A865F855B878D85DE
:10BFA0008C8780912902882309F427CF811491047A
:10BFB000A104B10409F4E9CE90E1C91A97E2D90AC3
:10BFC000E108F108C818D908EA08FB08F7FE15CF00
:10BFD000DCCE2F960FB6F894DEBF0FBECDBFDF913B
:10BFE000CF911F910F91FF90EF90DF90CF90BF9076
:10BFF000AF909F908F907F906F905F904F903F9009
:10C000002F9008952F923F924F925F926F927F925E
:10C010008F929F92AF92BF92CF92DF92EF92FF9258
:10C020000F931F93CF93DF93CDB7DEB72F970FB644
:10C03000F894DEBF0FBECDBF8DE690E00E94B64201
:10C04000811192C18091CF1583FD8EC183E50E943D
:10C05000BA418887811106C082E50E94BA418823CF
:10C0600009F482C10E9458410F946207CB010E94DB
:10C07000C5C60E94584120E030E04AEA52E40E94DE
:10C0800084FF181644F00E949ED860E081E992E196
:10C090000E943FC702C00E946EE06091220E709124
:10C0A000230E072E000C880B990B0E948AFF20910B
:10C0B0005F123091601240916112509162120F94A0
:10C0C0004408181684F48DE093E09F938F9385E8DD
:10C0D00092E19F938F931F920E94B7D80F900F9079
:10C0E0000F900F900F900E9411ED81E08093290234
:10C0F000412C512C32011C821D821E821F821B8208
:10C1000019862CE32A873CE13B8746E44C8710E004
:10C1100000E050E859838FEB8A83812C912C5401E5
:10C120006091220E7091230E072E000C880B990B44
:10C130000E948AFF7B018F879D879B01AC01612F45
:10C14000702F89819A810E9484FF882309F449C055
:10C1500020915F12309160124091611250916212F1
:10C160009885B7018F8591110EC09D850E9484FF2F
:10C17000881F8827881F8B831E2D0F2DAF85A983CD
:10C18000BD85BA832EC09D850E9484FF87FF22C093
:10C1900080912902882309F4E7C060E083E792E1F7
:10C1A0002F960FB6F894DEBF0FBECDBFDF91CF91B3
:10C1B0001F910F91FF90EF90DF90CF90BF90AF90C5
:10C1C0009F908F907F906F905F904F903F902F90B7
:10C1D0000C943FC71E2D0F2D2F8529833D853A8353
:10C1E0001B820E9486C26B017C01DC01CB012C8189
:10C1F0003D814E815F81821B930BA40BB50BB7FD74
:10C200003BC0D701C60188519C4FAF4FBF4F8C83B5
:10C210009D83AE83BF837FD8E1E8F2E18491DF01A3
:10C220001196BE87AD87882329F00E944442ED8590
:10C23000FE85F4CF81149104A104B104B9F0D501B5
:10C24000C401805F984DAF4FBF4FBC01CD016C1949
:10C250007D098E099F0928EE33E040E050E00F94FD
:10C26000C005CA01B9010E94F24203C08FE30E94D7
:10C2700044428AE00E94444280E00E94F6E70E9425
:10C28000394220905F1230906012B0916112BF87E6
:10C29000209162122D8791014B2F5D85612F702FA8
:10C2A00089819A810F941D069F7781149104A104BE
:10C2B000B10449F420E030E040E85FE30E9484FFED
:10C2C00087FF0BC008C020E030E040E450E40F944A
:10C2D0004408181614F4460157013B81332361F1D9
:10C2E000411451046104710441F0D701C60184195D
:10C2F0009509A609B709B7FD1FC091014F855D8556
:10C3000069857A858B859C850F941D0620E030E039
:10C3100040EC5FE30E9484FF87FD3ACF260137019E
:10C3200040E6440E4AEE541E611C711C29863A8672
:10C330005F855B878D858C8780912902882309F42E
:10C3400027CF81149104A104B10409F4E9CE90E14E
:10C35000C91A97E2D90AE108F108C818D908EA0809
:10C36000FB08F7FE15CFDCCE2F960FB6F894DEBF94
:10C370000FBECDBFDF91CF911F910F91FF90EF9036
:10C38000DF90CF90BF90AF909F908F907F906F90F5
:10C390005F904F903F902F900895DF92EF92FF9221
:10C3A0000F931F93CF93DF93109234108091D61583
:10C3B0009091D715A091D815B091D915813090489A
:10C3C000A105B10540F01092D6151092D715109224
:10C3D000D8151092D915C091D6158091B4061816AB
:10C3E000DCF4282F082E000C330B215031094C2F80
:10C3F0000C2E000C550B4217530774F0CFEFC80FEB
:10C400008C2F90E0A0E0B0E08093D6159093D715E4
:10C41000A093D815B093D9151092D80F8091D90F49
:10C42000C81714F4C093D90F8091D90F082E000CAF
:10C43000990B04962C2F0C2E000C330B82179307AC
:10C4400024F48CEF8C0F8093D90FD090D90FD0E0CB
:10C45000D1101EC080913610811106C080912A0231
:10C46000882309F4DAC009C0C111F8CF0E94534AE9
:10C470008091D80F882391F33CC20E94E4F4AC0170
:10C4800081E0C11180E024E06D2F0E9479C6C5C013
:10C4900081E0D8125AC080913610811106C0809177
:10C4A0002A02882309F4B9C022C0C130C1F78091A3
:10C4B0006412882341F0813019F485E194E105C0CC
:10C4C0008EE094E102C08CE194E1E12C10ECF12EBD
:10C4D00009E714E420E030E040E85FE368E776E055
:10C4E0000E943EF58091D80F8823C9F202C2809144
:10C4F0006412882341F0813019F485E194E105C08C
:10C500008EE094E102C08CE194E123E02F9327EECA
:10C510002F931F9221E02F9328E736E03F932F932C
:10C520009F938F939F938F93DF9381E0C13009F0A6
:10C5300080E08F930E94F9EE8DB79EB70C960FB6F0
:10C54000F8949EBF0FBE8DBF68C092E0D9125AC04A
:10C5500080913610811106C080912A02882309F447
:10C560005CC022C0C230C1F780916412882341F0C0
:10C57000813019F48AE294E105C083E294E102C0BB
:10C5800081E394E1E12C10ECF12E09E714E420E0C2
:10C5900030E040E85FE36CE776E00E943EF5809192
:10C5A000D80F8823C9F2A5C180916412882341F075
:10C5B000813019F48AE294E105C083E294E102C07B
:10C5C00081E394E123E02F9327EE2F931F9221E044
:10C5D0002F932CE736E03F932F939F938F939F9356
:10C5E0008F93DF9381E0C23009F080E08F930E9447
:10C5F000F9EE8DB79EB70C960FB6F8949EBF0FBE9E
:10C600008DBF0BC093E0D91261C0809136108111AB
:10C610000DC080912A0281112BC0DF5FD394D530E9
:10C6200009F016CF87E08093B40663C1C33089F761
:10C6300080916412882341F0813019F48FE394E1F2
:10C6400005C088E394E102C086E494E1E12C10EC9B
:10C65000F12E09E714E420E030E040E85FE360E811
:10C6600076E00E943EF58091D80F882391F241C177
:10C6700080916412882341F0813019F48FE394E1B2
:10C6800005C088E394E102C086E494E123E02F939F
:10C6900027EE2F931F9221E02F9320E836E03F935F
:10C6A0002F939F938F939F938F93DF9381E0C3305A
:10C6B00009F080E08F930E94F9EE8DB79EB70C963B
:10C6C0000FB6F8949EBF0FBE8DBFA7CF24E0D21245
:10C6D0005AC080913610811106C080912A028823A9
:10C6E00009F49BCF22C0C430C1F780916412882323
:10C6F00041F0813019F484E594E105C08DE494E1C2
:10C7000002C08BE594E1E12C10ECF12E09E714E472
:10C7100020E030E040E85FE364E876E00E943EF528
:10C720008091D80F8823C9F2E4C0809164128823D5
:10C7300041F0813019F484E594E105C08DE494E181
:10C7400002C08BE594E123E02F9327EE2F931F92F5
:10C7500021E02F9324E836E03F932F939F938F930C
:10C760009F938F93DF9381E0C43009F080E08F9333
:10C770000E94F9EE8DB79EB70C960FB6F8949EBF47
:10C780000FBE8DBF4ACF85E0D81258C080913610B9
:10C79000811106C080912A02882309F43ECF21C06E
:10C7A000C530C1F780916412882341F0813019F4BB
:10C7B00087E694E105C082E694E102C08CE694E14C
:10C7C000E12C10ECF12E09E714E420E030E0A9019F
:10C7D00064E776E00E943EF58091D80F8823D1F27D
:10C7E00088C080916412882341F0813019F487E673
:10C7F00094E105C082E694E102C08CE694E123E076
:10C800002F9327EE2F931F921F9224E736E03F933A
:10C810002F939F938F939F938F93DF9381E0C530E6
:10C8200009F080E08F930E94F9EE8DB79EB70C96C9
:10C830000FB6F8949EBF0FBE8DBFEFCE96E0D91213
:10C84000ECCE80913610811106C080912A02882397
:10C8500009F4E3CE21C0C630C1F780916412882369
:10C8600041F0813019F48BE794E105C081E794E150
:10C8700002C085E894E1E12C10ECF12E09E714E404
:10C8800020E030E0A90160E776E00E943EF580916B
:10C89000D80F8823D1F22DC080916412882341F0F3
:10C8A000813019F48BE794E105C081E794E102C07F
:10C8B00085E894E123E02F9327EE2F931F921F9298
:10C8C00020E736E03F932F939F938F939F938F930F
:10C8D000DF9381E0C63009F080E08F930E94F9EE8B
:10C8E0008DB79EB70C960FB6F8949EBF0FBE8DBF46
:10C8F00094CEDF91CF911F910F91FF90EF90DF9039
:10C9000008952F923F924F925F926F927F928F92F3
:10C910009F92AF92BF92DF92EF92FF920F931F937D
:10C92000CF93DF93109234108091D6159091D71544
:10C93000A091D815B091D91581309048A105B105C5
:10C9400040F01092D6151092D7151092D81510926B
:10C95000D915C091D6158091B6061816DCF4282F8B
:10C96000082E000C330B215031094C2F0C2E000CDB
:10C97000550B4217530774F0CFEFC80F8C2F90E080
:10C98000A0E0B0E08093D6159093D715A093D8156A
:10C99000B093D9151092D80F8091D90FC81714F4FD
:10C9A000C093D90F8091D90F082E000C990B0496D3
:10C9B0002C2F0C2E000C330B8217930724F48CEFD2
:10C9C0008C0F8093D90FD090D90FD0E0EAE08E2E53
:10C9D000912CA12CB12CFEEA4F2EF2E85F2E66249A
:10C9E0006394712CA5E82A2EADEA3A2ED1101EC010
:10C9F00080913610811106C080912A02882309F4A3
:10CA0000DAC009C0C111F8CF0E94534A8091D80FF3
:10CA1000882391F3AFC10E94E4F4AC0181E0C1111D
:10CA200080E024E06D2F0E9479C6C5C081E0D81255
:10CA30005AC080913610811106C080912A02882345
:10CA400009F4B9C022C0C130C1F7809164128823B3
:10CA500041F0813019F486E395E105C08EE295E15D
:10CA600002C08EE395E1E12C10E8F12E07E714E413
:10CA700020E030E040E85FE364EA76E00E943EF5C3
:10CA80008091D80F8823C9F275C1809164128823E0
:10CA900041F0813019F486E395E105C08EE295E11D
:10CAA00002C08EE395E123E02F932EED2F931F928A
:10CAB00021E02F9324EA36E03F932F939F938F93A7
:10CAC0009F938F93DF9381E0C13009F080E08F93D3
:10CAD0000E94F9EE8DB79EB70C960FB6F8949EBFE4
:10CAE0000FBE8DBF68C092E0D9125AC08091361037
:10CAF000811106C080912A02882309F45CC022C0FB
:10CB0000C230C1F780916412882341F0813019F45A
:10CB10008EE495E105C086E495E102C086E595E1E5
:10CB2000E12C10E8F12E07E714E420E030E040E8C3
:10CB30005FE368EA76E00E943EF58091D80F882393
:10CB4000C9F218C180916412882341F0813019F430
:10CB50008EE495E105C086E495E102C086E595E1A5
:10CB600023E02F932EED2F931F9221E02F9328EA9D
:10CB700036E03F932F939F938F939F938F93DF93F1
:10CB800081E0C23009F080E08F930E94F9EE8DB70A
:10CB90009EB70C960FB6F8949EBF0FBE8DBF0BC00C
:10CBA00093E0D9128AC08091361081110CC0809117
:10CBB0002A0281115FC0DF5FD394D53009F016CF10
:10CBC000D093B606D7C0C33091F780916412882302
:10CBD00041F0813019F406E615E105C00EE515E1D6
:10CBE00002C00EE615E10E940A4A83E080932A0201
:10CBF0001093E5150093E4158CEA96E09093E31505
:10CC00008093E2158092DE159092DF15A092E015D8
:10CC1000B092E1154092DA155092DB156092DC1566
:10CC20007092DD1520E030E048EC52E46091AC06F3
:10CC30007091AD068091AE069091AF060E94E9FF1B
:10CC400020E030E040E251E40F941D060F946707A6
:10CC50006093D6157093D7158093D8159093D915F6
:10CC600030927B0220927A028091D80F882309F4B7
:10CC70009ECF80C080916412882361F0813029F4B6
:10CC800056E6E52E55E1F52E09C04EE5E42E45E1C8
:10CC9000F42E04C03EE6E32E35E1F32E8CEA96E056
:10CCA0000E9401C49C0181E0C33009F080E000E0F3
:10CCB000A7016D2F0E9489EE7ECF24E0D2127BCF98
:10CCC00080913610811106C080912A02882309F4D0
:10CCD00072CF22C0C430C1F780916412882341F022
:10CCE000813019F48EE795E105C086E795E102C031
:10CCF00086E895E1E12C10E8F12E07E714E420E046
:10CD000030E040E85FE360EB76E00E943EF5809122
:10CD1000D80F8823C9F22EC080916412882341F075
:10CD2000813019F48EE795E105C086E795E102C0F0
:10CD300086E895E123E02F932EED2F931F9221E0BB
:10CD40002F9320EB36E03F932F939F938F939F93E6
:10CD50008F93DF9381E0C43009F080E08F930E94CD
:10CD6000F9EE8DB79EB70C960FB6F8949EBF0FBE26
:10CD70008DBF21CFDF91CF911F910F91FF90EF9049
:10CD8000DF90BF90AF909F908F907F906F905F905B
:10CD90004F903F902F900895CF92DF92EF92FF92A5
:10CDA0000F931F93CF93DF9300D01F92CDB7DEB7C1
:10CDB000109234108091D6159091D715A091D81566
:10CDC000B091D91581309048A105B10540F010927D
:10CDD000D6151092D7151092D8151092D91510911A
:10CDE000D6158091B5061816DCF4282F082E000CF5
:10CDF000330B21503109412F012E000C550B4217E6
:10CE0000530774F01FEF180F812F90E0A0E0B0E0FF
:10CE10008093D6159093D715A093D815B093D915B4
:10CE20001092D80F8091D90F181714F41093D90FBE
:10CE30008091D90F082E000C990B0496212F012EFA
:10CE4000000C330B8217930724F48CEF810F80932F
:10CE5000D90FE090D90FF12CE1101EC0809136104F
:10CE6000811106C080912A02882309F4C8C009C034
:10CE70001111F8CF0E94534A8091D80F882391F363
:10CE800046C20E94E4F4AC0181E0111180E024E08C
:10CE90006F2D0E9479C6B3C081E0E81245C0809131
:10CEA0003610811106C080912A02882309F4A7C098
:10CEB0001DC01130C1F780916412882341F0813088
:10CEC00019F485E994E105C08FE894E102C08BE98B
:10CED00094E120E030E040E251E460EA76E00E9434
:10CEE0005EF98091D80F8823F1F211C2809164120B
:10CEF000882361F0813029F475E9C72E74E1D72EBB
:10CF000009C06FE8C62E64E1D62E04C05BE9C52EC9
:10CF100054E1D52E80EA96E00E9482C49C0181E013
:10CF2000113009F066C066C022E0E21244C0809170
:10CF30003610811106C080912A02882309F45FC04F
:10CF40001DC01230C1F780916412882341F08130F6
:10CF500019F48BEA94E105C081EA94E102C085EB03
:10CF600094E120E030E048EC52E46CE976E00E9485
:10CF70005EF98091D80F8823F1F2C9C180916412C3
:10CF8000882361F0813029F44BEAC42E44E1D42E89
:10CF900009C031EAC32E34E1D32E04C025EBC22EE2
:10CFA00024E1D22E8CE996E00E9482C49C0181E0AB
:10CFB0001230F9F41FC023E0E21252C08091361003
:10CFC000811126C080912A028823C9F080916412C1
:10CFD000882309F440C08130C9F598ECC92E94E14A
:10CFE000D92E88E996E00E9482C49C0181E013302A
:10CFF00009F080E000E0A6016F2D0E9489EEF39415
:10D00000E39485E0F81228CF88E08093B5067FC1CD
:10D010001330C1F680916412882341F0813019F4F5
:10D0200088EC94E105C08FEB94E102C081ED94E1BE
:10D0300020E030E048EC52E468E976E00E945EF9D6
:10D040008091D80F882309F4BDCF61C18FEBC82E22
:10D0500084E1D82EC6CF01EDC02E04E1D02EC1CF81
:10D0600084E0E81252C080913610811105C0809191
:10D070002A02882321F21DC01430C9F7809164125E
:10D08000882341F0813019F481EE94E105C08AEDE6
:10D0900094E102C088EE94E124E630E040E050E004
:10D0A00068E876E00E941AFA8091D80F8823F9F296
:10D0B0002EC180916412882361F0813029F4B1EE91
:10D0C000CB2EB4E1DB2E09C0AAEDCA2EA4E1DA2EE4
:10D0D00004C0F8EECF2EF4E1DF2E60918806709147
:10D0E000890680918A0690918B060E9488FF698349
:10D0F0007A838B839C83CE0101960E9482C49C011B
:10D1000081E0143009F075CF75CF25E0E21253C0ED
:10D1100080913610811106C080912A02882309F47B
:10D120006ECF1DC01530C1F780916412882341F085
:10D13000813019F486EF94E105C08FEE94E102C0CE
:10D140008DEF94E124E630E040E050E06CE876E0DA
:10D150000E941AFA8091D80F8823F1F2D8C08091EA
:10D160006412882361F0813029F4E6EFCE2EE4E1E9
:10D17000DE2E09C07FEEC72E74E1D72E04C06DEFFE
:10D18000C62E64E1D62E60918C0670918D0680913A
:10D190008E0690918F060E9488FF69837A838B8325
:10D1A0009C83CE0101960E9482C49C0181E01530CF
:10D1B00009F01FCF1FCF86E0E81253C080913610D0
:10D1C000811106C080912A02882309F418CF1DC05E
:10D1D0001630C1F780916412882341F0813019F430
:10D1E0008BE095E105C084E095E102C082E195E124
:10D1F0002AE030E040E050E060E976E00E941AFA70
:10D200008091D80F8823F1F282C080916412882324
:10D2100061F0813029F45BE0C52E55E1D52E09C0BF
:10D2200044E0C42E45E1D42E04C032E1C32E35E1E2
:10D23000D32E609190067091910680919206909104
:10D2400093060E9488FF69837A838B839C83CE0137
:10D2500001960E9482C49C0181E0163009F0C9CE7B
:10D26000C9CE27E0E212CBCE80913610811106C0E4
:10D2700080912A02882309F4C2CE1DC01730C1F75D
:10D2800080916412882341F0813019F480E295E1A5
:10D2900005C089E195E102C087E295E124E630E02E
:10D2A00040E050E064E976E00E941AFA8091D80FDD
:10D2B0008823F1F22CC080916412882361F08130C0
:10D2C00029F420E2C22E25E1D22E09C099E1C92E0F
:10D2D00095E1D92E04C087E2C82E85E1D82E609151
:10D2E00094067091950680919606909197060E94FB
:10D2F00088FF69837A838B839C83CE0101960E9489
:10D3000082C49C0181E0173009F073CE73CE0F9078
:10D310000F900F900F90DF91CF911F910F91FF9081
:10D32000EF90DF90CF9008950C9441ED0C945FEE58
:10D3300081E00C94BB9180E00C94BB918F929F9202
:10D34000AF92BF92CF92DF92EF92FF921F93CF9353
:10D35000DF93C82F83EC94E19093C1088093C008B9
:10D360001092DF1482E090E0A0E0B0E08093C81457
:10D370009093C914A093CA14B093CB141092BF0811
:10D380001092BB081092BC081092BD081092BE0803
:10D390008FEF9FEFDC018093B7089093B808A093BC
:10D3A000B908B093BA08CC2379F1C53008F0F8C0B9
:10D3B00040E060E070E0CB010E940DE3882309F4B7
:10D3C000EFC020E1C29FC00111248955994FFC0193
:10D3D000E254FE4F20812F7709F0E2C03C96408155
:10D3E000518162817381443651056105710508F4EC
:10D3F000D7C03497C080D180E280F380C114D104BB
:10D40000E104F10421F4CCC0C12CD12C760140E020
:10D41000C701B6010E940DE3182F882309F4C0C08C
:10D420008091C2069091C3068115924009F0B8C060
:10D43000A091C706AA2309F4B3C06091C5067091F4
:10D44000C6066115710509F4ABC02091C4062223FC
:10D4500009F4A6C0A093DA142093CC1480E030E045
:10D4600041E050E0C82FFA01082E02C0EE0FFF1F66
:10D470000A94E2F72E173F0739F08F5FC83091F713
:10D4800089E08093D5148CC08093D5142091CD066B
:10D490003091CE062115310519F040E050E008C06A
:10D4A0002091DB063091DC064091DD065091DE06CE
:10D4B0002093CD143093CE144093CF145093D014B6
:10D4C00046015701860E971EA11CB11C8092DB14E9
:10D4D0009092DC14A092DD14B092DE14E091C806A4
:10D4E000F091C906F093E114E093E014B0E00F94DA
:10D4F000FE05860E971EA81EB91E8092E214909219
:10D50000E314A092E414B092E51485E0EE0FFF1F3F
:10D510008A95E1F7E150FE4FEF2FFF27E6958E0E3B
:10D520009F1EA11CB11C8092D6149092D714A09279
:10D53000D814B092D9142091CA063091CB06211587
:10D54000310521F0A90160E070E008C04091D706E4
:10D550005091D8066091D9067091DA06D701C601BC
:10D5600088199909AA09BB09840F951FA61FB71F1F
:10D5700004C0B695A79597958795CA95D2F78093DD
:10D58000D1149093D214A093D314B093D414853FA4
:10D590002FE09207A105B10528F48CE08093DF14F9
:10D5A00010E01AC0853F9F4FA105B10510F480E13E
:10D5B00011C08091E3069091E406A091E506B09138
:10D5C000E6068093E2149093E314A093E414B093DE
:10D5D000E51480E28093DF14812FDF91CF911F91BA
:10D5E000FF90EF90DF90CF90BF90AF909F908F9083
:10D5F0000895CF92DF92EF92FF920F931F93CF93F4
:10D60000DF93CDB7DEB7EDB6FEB6DC010D9000209E
:10D61000E9F79D01281B390B2C5F3F4F4DB75EB7D3
:10D62000421B530B0FB6F8945EBF0FBE4DBF0DB734
:10D630001EB70F5F1F4F9F938F938BEE96E19F93C3
:10D640008F931F930F930E941EFF680154E0C50E35
:10D65000D11C0F900F900F900F900F900F90F6012C
:10D660008081882349F0082E000C990B0F941F0924
:10D67000F60181936F01F3CFC8010E9449DA87EE6A
:10D6800096E19093C3088093C2080E9458400FB659
:10D69000F894FEBE0FBEEDBEDF91CF911F910F91AA
:10D6A000FF90EF90DF90CF900895AF92BF92CF920E
:10D6B000DF92EF92FF920F931F93CF93DF93CDB73B
:10D6C000DEB7AA970FB6F894DEBF0FBECDBF80912C
:10D6D0004B138F9380914A138F938EED96E19F9316
:10D6E0008F937E0181E2E80EF11CFF92EF920E947F
:10D6F0001EFF0F900F900F900F900F900F9010E063
:10D70000F70101900020E9F73197EE19FF091E1784
:10D7100084F46701C10ED11C17FDDA94F6018081F3
:10D72000082E000C990B0F941F09F60180831F5FD0
:10D73000E7CF80E593E10E94C9B600E0CE010196F3
:10D740006C0180915313823080F080915813909136
:10D750005913A0915A13B0915B138F719927AA277F
:10D76000BB27892B8A2B8B2BF9F0011103C08FEF7C
:10D770009FEF05C080914A1390914B1301969093AF
:10D780004B1380934A13AA960FB6F894DEBF0FBED0
:10D79000CDBFDF91CF911F910F91FF90EF90DF9060
:10D7A000CF90BF90AF90089540E050E0B60180E583
:10D7B00093E10E94BDE41816C4F6F6010190002022
:10D7C000E9F731971E2F1C19115068F05601A10E70
:10D7D000B11C17FDBA94F501808190E00F941F09E8
:10D7E000F5018083F1CF8A858E3709F4AACF45E011
:10D7F00050E0B701C6010F947D09892B09F0A1CF34
:10D80000C701F7DE01E09DCFCF92DF92EF92FF924A
:10D810001F93CF93DF93109220138091531388238B
:10D8200021F080E593E10E946CB51092C71410922C
:10D83000C41485E38093C3140E9486C2EB01A895AB
:10D8400061E08091C3140E944AC183EC94E10E947C
:10D85000CEB62398229A219A209A289A85E080931E
:10D86000C51482E58CBD1DBC1AE08FEF0E94D3B6B3
:10D870001150D9F720E030E0A90160E083EC94E199
:10D880000E94D8B6182F8093C614813049F00E94A8
:10D8900086C26C1B7D0B613D774060F381E054C014
:10D8A0002AEA31E040E050E068E083EC94E10E9435
:10D8B000D8B682FF03C01093C7140EC014E00E94B4
:10D8C000D8BB8093C6141150D1F78A3A11F082E088
:10D8D0003BC082E08093C7148091C714823021F04E
:10D8E000C12CD12C760105C0C12CD12CE12C80E4B7
:10D8F000F82E20E030E0A90167E383EC94E10E9478
:10D90000D8B6A701960169E283EC94E10E94D8B6EB
:10D910008093C614882349F00E9486C26C1B7D0B3D
:10D92000613D774030F38AE00FC08091C7148230A8
:10D9300011F520E030E0A9016AE383EC94E10E9454
:10D94000D8B6882351F088E08093C41483EC94E126
:10D950000E94CEB6EBE9F9E419C00E94D8BB807CE6
:10D96000803C19F483E08093C7140E94D8BB0E94C6
:10D97000D8BB0E94D8BB83EC94E10E94CEB6109233
:10D98000C51481E0DBDC811131C015C08491EF0149
:10D990002196882321F00E944442FE01F7CFE0ED5A
:10D9A000F6E18491EF012196882309F456C00E9484
:10D9B0004442FE01F6CF80E0C1DC811117C0E9ECE2
:10D9C000F6E18491EF012196882321F00E944442E0
:10D9D000FE01F7CFE5EBF6E18491EF012196882374
:10D9E00009F43BC00E944442FE01F6CF68EC74E1AA
:10D9F00080E593E10E9419B5811116C0E9ECF6E1CA
:10DA00008491EF012196882321F00E944442FE0177
:10DA1000F7CFE4EAF6E18491EF0121968823E9F05B
:10DA20000E944442FE01F7CF81E080932013EBE98E
:10DA3000F9E48491EF012196882321F00E94444269
:10DA4000FE01F7CFE8E9F6E18491EF012196882302
:10DA500021F00E944442FE01F7CF8BE1E0E5F3E1C3
:10DA6000A1E7B3E101900D928A95E1F780914E1301
:10DA700090914F139093701380936F138CE493E104
:10DA800090936C1380936B13DF91CF911F91FF9054
:10DA9000EF90DF90CF9008950F931F9380910F1315
:10DAA00090911013019719F40E9486C208C06091EA
:10DAB000191370911A1380911B1390911C130091EC
:10DAC0001513109116132091171330911813601B22
:10DAD000710B820B930B28EE33E040E050E00F9483
:10DAE000C0058091111390911213A0911313B0915E
:10DAF0001413BC01CD01620F731F841F951F1F916A
:10DB00000F9108952F923F924F925F926F927F9262
:10DB10008F929F92AF92BF92CF92DF92EF92FF923D
:10DB20000F931F93CF93DF93CDB7DEB7C057D109C3
:10DB30000FB6F894DEBF0FBECDBF7C013B014A019A
:10DB40002DB73EB7AF963FAF2EAFAF97AD961FAE96
:10DB5000AD972B0134E0430E511C8E01015A1F4F2B
:10DB600080E490E08C0F9D1F0496E1969FAF8EAFEE
:10DB7000E197F3018781823008F459C18485958546
:10DB8000A685B7858F719927AA27BB27892B8A2B52
:10DB90008B2B09F04CC18FE293E1892B11F010928D
:10DBA0002F134FE253E1BE016F5F7F4FC2010E940E
:10DBB000BDE418160CF03BC18C85982F98719031FC
:10DBC00009F0AEC02091C3153091C4152150310920
:10DBD0002230310508F4A4C02DB63EB6BE016F5FF9
:10DBE0007F4FC8010E94ADE2F7018081882341F098
:10DBF000F70101900020E9F73197EE19FF0902C003
:10DC0000E1E0F0E0D8010D900020E9F7E01BF10B16
:10DC1000EA0FFB1F31962DB73EB72E1B3F0B0FB6F9
:10DC2000F8943EBF0FBE2DBFEDB7FEB731965F0132
:10DC3000882311F0B70102C06DE973E0C5010F94AC
:10DC40007609B801C5010F9457096DE973E0C50164
:10DC50000F945709CE01805C9F4F0E94C3E221E0E0
:10DC6000A801B201E1968EAD9FADE1970E94FABA8C
:10DC700081112CC08091C3159091C415892B31F569
:10DC8000EBE9F9E484916F012FEFC21AD20A8823DD
:10DC900021F00E944442F601F5CFE4E8F6E18491D8
:10DCA0006F013FEFC31AD30A882321F00E94444238
:10DCB000F601F5CF6801F60181916F01882319F013
:10DCC0000E944442F8CF8AE00E9444428BE1FE0168
:10DCD000EC5BFF4FDE01959601900D928A95E1F77E
:10DCE00024968EAD9FAD24979CA38BA32FE932E0A1
:10DCF0003AA329A340E050E0BE016F5D7F4FC5010C
:10DD000001DFCE0181960E9454BDCE01805C9F4F01
:10DD10000E9454BD0FB6F8943EBE0FBE2DBE29CF53
:10DD20002981222309F483C0253E09F422CF2E3213
:10DD300009F41FCF20912F132E3209F41ACF8A70C5
:10DD400009F017CF81E0903109F080E08093211332
:10DD5000903141F08985873409F00BCF8A858E3761
:10DD600009F407CF8091C3159091C41581309105B6
:10DD700021F068F00297A9F1FCCE8091C515909131
:10DD8000C61501969093C6158093C515F2CEBE01B7
:10DD90006F5F7F4F82E293E10E94ADE26701F6017F
:10DDA00081916F01882319F00E944442F8CF82E2EA
:10DDB000C82E83E1D82EF60181916F01882319F0D6
:10DDC0000E944442F8CF80E20E9444426D8D7E8DD5
:10DDD0008F8D98A14AE00E944B428AE00E94444203
:10DDE000C8CEBE016F5F7F4F82E293E10E94ADE239
:10DDF0008114910441F062E273E1C4010F9444097B
:10DE0000892B69F414C0AD96FFADAD978F2F90E0CC
:10DE10002091C5153091C6158217930741F0AD9634
:10DE20002FADAD972F5FAD962FAFAD97A2CEAF962A
:10DE30002EAD3FADAF970FB6F8943EBF0FBE2DBFCE
:10DE4000C059DF4F0FB6F894DEBF0FBECDBFDF91D4
:10DE5000CF911F910F91FF90EF90DF90CF90BF90E7
:10DE6000AF909F908F907F906F905F904F903F907A
:10DE70002F900895EF92FF920F931F93CF93DF930C
:10DE8000CDB7DEB76F970FB6F894DEBF0FBECDBF2C
:10DE90007B010BE613E12DE633E1F80131832083AA
:10DEA00022E030E03093C4152093C3159093C6153B
:10DEB0008093C51581E793E10E94C9B6F80180817E
:10DEC00091812BE1FC013496DE01159601900D92B3
:10DED0002A95E1F7FC01828193819C838B838FE9F2
:10DEE00092E09A838983A701BE016F5F7F4F89E02B
:10DEF00095E008DECE0101960E9454BD6F960FB6E4
:10DF0000F894DEBF0FBECDBFDF91CF911F910F916F
:10DF1000FF90EF9008956F927F929F92AF92BF9281
:10DF2000CF92DF92EF92FF920F931F93CF93DF93E5
:10DF3000CDB7DEB7AC970FB6F894DEBF0FBECDBF3E
:10DF400020912013222309F4C2C1962E7C018091D6
:10DF5000ED14882309F474C0442309F48DC1809121
:10DF60002415882329F1E9ECF6E184918F010F5FF4
:10DF70001F4F882321F00E944442F801F6CFE1E4CC
:10DF8000F6E184918F010F5F1F4F882321F00E94DB
:10DF90004442F801F6CF61E070E080E090E00E943A
:10DFA000F2428AE00E94444288E396E10E9428C03F
:10DFB00089E295E10E9478D7EBE9F9E484918F0139
:10DFC0000F5F1F4F882321F00E944442F801F6CFD3
:10DFD000B7018FE196E10E9466EC609124158DE80F
:10DFE000689FB0011124675D7A4E84E196E10E943A
:10DFF00066EC4091BA155091BB156091BC157091BB
:10E00000BD158EE096E10E9413EC8AE00E94444226
:10E010008091241594E0899FF0011124EB5DFA4E64
:10E020004091BA155091BB156091BC157091BD150A
:10E0300040835183628373838F5F809324150DC067
:10E040001092241582E0D82E19C1B70181E096E123
:10E050000E9466EC8AE00E94444210921F13809155
:10E06000ED14882321F08AEE94E10E946CB5CE0174
:10E0700001966C010E94C3E28CE493E190936C13CF
:10E0800080936B13F70180818F3209F060C08701A4
:10E090000F5F1F4F09F461C06FE270E0C8010F9479
:10E0A00062095C01009709F459C00817190708F0C4
:10E0B00055C03C01601A710AA301B801CE018096D7
:10E0C0000F948B09E0E2F0E0EC0FFD1FE60DF71D69
:10E0D0001082CE0180963C018C01F80181918F0164
:10E0E000882319F00E944442F8CF8AE00E944442FB
:10E0F00060916B1370916C136115710511F06C5F79
:10E100007F4F21E0AE01405E5F4FCE0105960E9439
:10E11000FABA811116C0EDEEF5E184918F010F5F1F
:10E120001F4F882321F00E944442F801F6CFF301EB
:10E1300081913F01882319F00E944442F8CF8EE27A
:10E1400085C0D0926C13C0926B138501A1CF8DE670
:10E1500093E190936C1380936B13870190916B13F1
:10E1600080916C13692F782F992009F459C061159B
:10E17000710511F06C5F7F4F21E0A8018AEE94E1F8
:10E180000E94FABA882309F447C08091FB14909149
:10E19000FC14A091FD14B091FE148093B6159093D9
:10E1A000B715A093B815B093B915B8018FED95E1E7
:10E1B0000E9466EC4091B6155091B7156091B81564
:10E1C0007091B91587ED95E10E9413EC8AE00E94E9
:10E1D00044421092BA151092BB151092BC151092C1
:10E1E000BD15E8ECF5E184917F019FEFE91AF90A8A
:10E1F000882321F00E944442F701F5CFB80180E066
:10E2000090E038DE80912F13882319F08FE293E19C
:10E2100001C0C80160E02AC0B80184EB95E110C0DC
:10E220006115710511F06C5F7F4F26E5A8018AEE3C
:10E2300094E10E94FABA81110CC0B80180EA95E11C
:10E240000E9466EC8EE20E9444428AE00E944442B0
:10E250000FC081E080931D13B7018EE895E10E9405
:10E2600066EC8AE00E94444260E0C8010E945DC7FB
:10E27000C6010E9454BD2BC0DD24D394EBE9F9E420
:10E2800084918F010F5F1F4F882321F00E94444229
:10E29000F801F6CFE9E0F6E184918F010F5F1F4F9F
:10E2A000882321F00E944442F801F6CFE1E0DE1617
:10E2B00019F00FE913E002C005EA13E0F8018191BB
:10E2C0008F01882309F4C1CE0E944442F7CFAC9657
:10E2D0000FB6F894DEBF0FBECDBFDF91CF911F9177
:10E2E0000F91FF90EF90DF90CF90BF90AF909F90F5
:10E2F0007F906F900895DF92EF92FF920F931F939C
:10E30000CF93DF93F82ED62EE72E8A018091060256
:10E31000882309F439C0E9ECF6E18491EF012196F4
:10E32000882321F00E944442FE01F7CFED2DFE2DFF
:10E330008491EF012196882321F00E944442FE013E
:10E34000F7CFE3E0FFE18491EF012196882321F0EC
:10E350000E944442FE01F7CFF7FC0BC06F2DFF0C6B
:10E36000770B880B990B0E94F2428AE00E9444428C
:10E370000BC0EEEFFEE18491EF012196882321F09E
:10E380000E944442FE01F7CF8091DB0D811108C04D
:10E390001092060281E08093DB0DC8010E9428C024
:10E3A000DF91CF911F910F91FF90EF90DF900C9430
:10E3B0005AA84F925F926F927F928F929F92AF92E4
:10E3C000BF92CF92DF92EF92FF920F931F93CF9362
:10E3D000DF93CDB7DEB72C970FB6F894DEBF0FBE34
:10E3E000CDBF80910610811117C02C960FB6F894FE
:10E3F000DEBF0FBECDBFDF91CF911F910F91FF9078
:10E40000EF90DF90CF90BF90AF909F908F907F90D4
:10E410006F905F904F9008950E9463A90E9486C2FA
:10E420002B013C0180912106811117C08091B10D13
:10E430009091B20DA091B30DB091B40D0097A105CC
:10E44000B10559F0A3019201281B390B4A0B5B0B54
:10E4500057FD03C081E0809321066091220E7091E8
:10E46000230E072E000C880B990B0E948AFF209127
:10E470005F1230916012409161125091621214E06B
:10E48000812E912C0CE3A02EB12CC12CD12C7B0120
:10E490008C016DEF7DE08BEF9DE00E94EEA68090F9
:10E4A0005F1290906012A0906112B0906212609121
:10E4B000070E7091080E072E000C880B990B0E9416
:10E4C0008AFF9B01AC01C501B4010F9444081816E2
:10E4D0000CF008C160910B0270910C02072E000C29
:10E4E000880B990B0E948AFF9B01AC01C501B40106
:10E4F0000E9484FF87FFF6C04091220E5091230EA8
:10E500005A83498320ED3CEC4CE45DE36091AD0D12
:10E510007091AE0D8091AF0D9091B00D0E94E9FF0A
:10E520006B017C012091F10D3091F20D4091F30DC2
:10E530005091F40DC501B4010F941D069B01AC016F
:10E54000C701B6010E94E9FF6B017C0123E333E3BD
:10E5500043E75FE36091ED0D7091EE0D8091EF0D5B
:10E560009091F00D0E94E9FF9B01AC01C701B6013B
:10E570000F941E066B017C016093ED0D7093EE0D00
:10E580008093EF0D9093F00D8092F10D9092F20D2B
:10E59000A092F30DB092F40D80912106811115C265
:10E5A000A981BA81BD01BB0F880B990B0E948AFF1C
:10E5B000A50194010F941D064B015C0120E030E0A1
:10E5C00040E251E40F94440818160CF40FC220E006
:10E5D00030E040E251ECC501B4010E9484FF87FDA8
:10E5E000F4C129813A81232B09F4EFC18091EC0D0C
:10E5F00081111BC28091E80D9091E90DA091EA0D67
:10E60000B091EB0D89839A83AB83BC832091A90DD4
:10E610003091AA0D4091AB0D5091AC0DC501B401E4
:10E620000E94E9FF6D837E838F839887A501940103
:10E6300069817A818B819C810F941E0669837A831C
:10E640008B839C836093E80D7093E90D8093EA0DB2
:10E650009093EB0D2091A50D3091A60D4091A70D43
:10E660005091A80D0E94E9FF2D813E814F81588570
:10E670000F941E06A70196010F941D066B017C01E5
:10E6800020E030E04FE753E40F94440820E030E00E
:10E69000A90118160CF4D0C1C701B6010E9484FF6D
:10E6A00087FD07C0C701B6010F946207759567958E
:10E6B0001AC020E030E0A901C501B4010E9484FF26
:10E6C00087FF10C0A501940169817A818B819C81AB
:10E6D0000F941D066093E80D7093E90D8093EA0D89
:10E6E0009093EB0D60E0609308108091F90F90918A
:10E6F000FA0FA091FB0FB091FC0F0097A105B10597
:10E7000009F1A3019201281B390B4A0B5B0B57FD42
:10E7100019C06091FD0F7091FE0F80E090E00E94A3
:10E7200088FF9B01AC0160915F1270916012809133
:10E730006112909162120E9484FF87FD3FC180E0C8
:10E740000E947DA88091FF0F90910010A091011070
:10E75000B09102100097A105B10511F1481A590AAC
:10E760006A0A7B0A77FC1CC0609103107091041048
:10E7700080E090E00E9488FF9B01AC0160911C0644
:10E7800070911D0680911E0690911F060E9484FFC5
:10E7900087FF11C141E25FE160E37FE18FEFABDD15
:10E7A0006091E9157091EA15072E000C880B990B02
:10E7B0000E948AFF20911C0630911D0640911E0682
:10E7C00050911F06E2E08E2E912CF8E7AF2EB12C6F
:10E7D000CC24CA94DC2C7B018C0165EF7DE089EFB1
:10E7E0009DE00E94EEA6809120068111E1C0C090BC
:10E7F0001C06D0901D06E0901E06F0901F0620E03B
:10E8000030E040EA50E4C701B6010F94440887FFA6
:10E8100004C060E060930710E8CD20E030E04AEFEC
:10E8200052E4C701B6010E9484FF181694F3609168
:10E83000E9157091EA15072E000C880B990B0E94C0
:10E840008AFFA70196010F941D064B015C012091E0
:10E85000A10D3091A20D4091A30D5091A40D0E94E5
:10E86000E9FF6D837E838F8398872091E40D30913B
:10E87000E50D4091E60D5091E70DC501B4010F94EF
:10E880001E0669837A838B839C836093E40D709367
:10E89000E50D8093E60D9093E70D20919D0D30914D
:10E8A0009E0D40919F0D5091A00D0E94E9FF698738
:10E8B0007A878B879C8720ED3CEC4CE45DE360918C
:10E8C000990D70919A0D80919B0D90919C0D0E94D5
:10E8D000E9FF2B013C012091E00D3091E10D4091C9
:10E8E000E20D5091E30DC701B6010F941D069B0187
:10E8F000AC01C301B2010E94E9FF2B013C0123E3FB
:10E9000033E343E75FE36091DC0D7091DD0D8091AF
:10E91000DE0D9091DF0D0E94E9FF9B01AC01C30168
:10E92000B2010F941E062B013C016093DC0D709325
:10E93000DD0D8093DE0D9093DF0DC092E00DD0923F
:10E94000E10DE092E20DF092E30D29853A854B85C9
:10E950005C856D817E818F8198850F941E06A30151
:10E9600092010F941D066B017C0120E030E04FE71F
:10E9700053E40F94440820E030E0A90118164CF548
:10E98000C501B4010F944408181684F4A50194013C
:10E9900069817A818B819C810F941D066093E40DBF
:10E9A0007093E50D8093E60D9093E70D6FE732CFFE
:10E9B000109207101ACD0E940EA8F2CE4FE35FE12D
:10E9C0006EE47FE180E097DCBDCE81E08093EC0DCA
:10E9D00089CEC701B6010E9484FF87FD0CC0C70124
:10E9E000B6010F9462077595679514CF81E0809307
:10E9F000EC0D6FE778CE20E030E0A901C501B4014D
:10EA00000E9484FF87FF05CFA501940169817A8167
:10EA10008B819C810F941D066093E40D7093E50D2E
:10EA20008093E60D9093E70DF4CE1092EC0D1982D1
:10EA30001A821B821C82EACDC501B4010F944408DE
:10EA40001816BCF6A501940169817A818B819C819D
:10EA50000F941D066093E80D7093E90D8093EA0D05
:10EA60009093EB0D6FE73FCE880F991F880F991F8A
:10EA7000FC01E25CF74E4081518162817381FC01AF
:10EA8000EC5CF14F4083518362837383E091970D77
:10EA9000F091980D82899389A489B5898093D70DC7
:10EAA0009093D80DA093D90DB093DA0D0895CF931C
:10EAB000DF932FB7F894AC01440F551F440F551F37
:10EAC000FA01E25CF74E60817181828193812FBFF0
:10EAD000EA01CC5DD14F0E948AFF288139814A81A9
:10EAE0005B810E94E9FFDF91CF9108959091EF1231
:10EAF0008091F012981721F080E00E94F6E7F6CF9F
:10EB000008951F920F920FB60F9211240BB60F9219
:10EB1000BF92CF92DF92EF92FF920F931F932F93AA
:10EB20003F934F935F936F937F938F939F93AF9395
:10EB3000BF93EF93FF93CF93DF9300D000D0CDB777
:10EB4000DEB780916E008B7F80936E0080916F00A6
:10EB50008D7F80936F007894C090D30DD090D40DAA
:10EB6000E090D50DF090D60DC114D104E104F1046C
:10EB7000F1F18091090E8823D1F10E945A7E09EBB0
:10EB8000C0160BE0D006E104F10488F018EBC11ABE
:10EB90001BE0D10AE108F108C092D30DD092D40D48
:10EBA000E092D50DF092D60D88EB9BE009C0C6012E
:10EBB0001092D30D1092D40D1092D50D1092D60D47
:10EBC000909389008093880020918800309189007B
:10EBD000809184009091850040962817390708F0AD
:10EBE00065C68091840090918500409611C2209165
:10EBF000950D3091960D3A83298321153105E9F061
:10EC0000215031093A8329833093960D2093950D35
:10EC10001092980D1092970D0E9406EC09811A81AE
:10EC2000012B41F482EF9EE19093C3088093C208C8
:10EC30000E94584088EC90E0EBC10091970D109134
:10EC4000980D0115110509F0E8C19091EF1280911E
:10EC5000F012981761F10091F0122DE4029F8001EB
:10EC60001124F801EC53F74FC0902A10D0902B10CC
:10EC7000E0902C10F0902D10CF01875B9F4FDC01AE
:10EC80004D915D916D917C91D701C601841B950BCF
:10EC9000A60BB70B80932A1090932B10A0932C10E7
:10ECA000B0932D108081886080838F010BC08FB757
:10ECB000F89410922A1010922B1010922C1010928F
:10ECC0002D108FBF1093980D0093970D011511050E
:10ECD00009F49CC1F80152A18091940D418158130F
:10ECE0000AC0242F30E080910502082E000C990BF9
:10ECF0002817390731F05093940D409305020E9474
:10ED0000CCEB1092CF0D1092D00D1092D10D10922D
:10ED1000D20DD801D7960D90BC91A02DBA83A983AE
:10ED2000A134ECE9BE0720F4A132BE4478F004C05F
:10ED300020E43CE93A83298349815A8156954795D5
:10ED4000569547955A83498384E00BC089819A81FF
:10ED50008131A7E29A0740F0969587959A83898337
:10ED600082E08093CE0D0BC081E08093CE0DE981CF
:10ED7000FA81B09720F420E230E03A832983498178
:10ED80005A81405251095A834983411568E0560718
:10ED9000F0F0E52FFF27EE0FFF1FEE0FFF1FCF0153
:10EDA0008E50954EFC01329645915491B981AA2717
:10EDB000B59F9001B49F210D3A1F06942A1F3A1F58
:10EDC0001124FC0185919491821B930B22C08981AF
:10EDD0009A81969587958C7F8E50994EFC0125914E
:10EDE0003491FC0132964591549169817A81677022
:10EDF0007727649FC001659F900D749F900D11242B
:10EE000053E0969587955A95E1F7F901E81BF90BC0
:10EE1000CF018436910590F43BEAE32E33E0F32EE4
:10EE2000D7018D917D01882319F00E944442F8CFCB
:10EE300089819A810E946CD784E690E09093CD0DF1
:10EE40008093CC0D8091CE0D8093CB0DF80103AC57
:10EE5000F4ADE02DFA83E983F093CA0DE093C90D78
:10EE6000E1342CE9F20720F4E132FE4478F004C0EA
:10EE700040E45CE95A83498389819A819695879514
:10EE8000969587959A83898384E00BC0A981BA817E
:10EE9000A131E7E2BE0740F0B695A795BA83A983F2
:10EEA00082E08093CE0D0CC081E08093CE0D29814D
:10EEB0003A812032310520F440E250E05A83498300
:10EEC00089819A8180979A8389838115A8E09A071E
:10EED000F0F0E92FFF27EE0FFF1FEE0FFF1FCF010E
:10EEE0008E50954EFC01329645915491B981AA27D6
:10EEF000B59F9001B49F210D3A1F06942A1F3A1F17
:10EF00001124FC0185919491821B930B22C089816D
:10EF10009A81969587958C7F8E50994EFC0125910C
:10EF20003491FC0132964591549169817A816770E0
:10EF30007727649FC001659F900D749F900D1124E9
:10EF400073E0969587957A95E1F7F901E81BF90B3F
:10EF5000CF018436910590F45BEAE52E53E0F52E5F
:10EF6000D7018D917D01882319F00E944442F8CF8A
:10EF700089819A810E946CD784E690E0AC0160E0C0
:10EF800070E04093C50D5093C60D6093C70D70930C
:10EF9000C80D9093890080938800F8018289938935
:10EFA000A489B589B695A79597958795B095A095AD
:10EFB000909581959F4FAF4FBF4F8093C10D909318
:10EFC000C20DA093C30DB093C40D8093BD0D90935B
:10EFD000BE0DA093BF0DB093C00D8093B90D90935B
:10EFE000BA0DA093BB0DB093BC0D8093B50D90935B
:10EFF000B60DA093B70DB093B80D1092D70D109227
:10F00000D80D1092D90D1092DA0D07C080ED97E05F
:10F01000909389008093880049C48091090E8111E2
:10F0200049D62091CE0D222309F4AFC1E091970D6E
:10F03000F091980D42815381648175818091B50D65
:10F040009091B60DA091B70DB091B80D840F951F9A
:10F05000A61FB71F8093B50D9093B60DA093B70D63
:10F06000B093B80D181619061A061B060CF4889AE8
:10F07000E091970DF091980D4681578160857185DB
:10F080008091B90D9091BA0DA091BB0DB091BC0DBE
:10F09000840F951FA61FB71F8093B90D9093BA0DCB
:10F0A000A093BB0DB093BC0D181619061A061B06CB
:10F0B0000CF48E9AE091970DF091980D428553854E
:10F0C000648575858091BD0D9091BE0DA091BF0D99
:10F0D000B091C00D840F951FA61FB71F8093BD0D63
:10F0E0009093BE0DA093BF0DB093C00D18161906D6
:10F0F0001A061B0644F49FB7F89480910B018860B0
:10F1000080930B019FBFE091970DF091980D46857C
:10F110005785608971898091C10D9091C20DA09130
:10F12000C30DB091C40D840F951FA61FB71F809308
:10F13000C10D9093C20DA093C30DB093C40D1816CA
:10F1400019061A061B060CF4149A8091B50D9091BD
:10F15000B60DA091B70DB091B80D181619061A0684
:10F160001B0684F5E091970DF091980D4289538923
:10F1700064897589841B950BA60BB70B8093B50D1D
:10F180009093B60DA093B70DB093B80D8091010286
:10F1900040913E1850913F1860914018709141186D
:10F1A000082E000C990BAA0BBB0B840F951FA61FF2
:10F1B000B71F80933E1890933F18A0934018B093C8
:10F1C000411888988091B90D9091BA0DA091BB0D0E
:10F1D000B091BC0D181619061A061B0684F5E091AD
:10F1E000970DF091980D4289538964897589841B24
:10F1F000950BA60BB70B8093B90D9093BA0DA09306
:10F20000BB0DB093BC0D8091020240914218509109
:10F2100043186091441870914518082E000C990B02
:10F22000AA0BBB0B840F951FA61FB71F8093421814
:10F2300090934318A0934418B09345188E988091EA
:10F24000BD0D9091BE0DA091BF0DB091C00D1816CF
:10F2500019061A061B06BCF5E091970DF091980D62
:10F260004289538964897589841B950BA60BB70B5A
:10F270008093BD0D9093BE0DA093BF0DB093C00DB4
:10F2800080910302409146185091471860914818A8
:10F2900070914918082E000C990BAA0BBB0B840F18
:10F2A000951FA61FB71F8093461890934718A093E9
:10F2B0004818B09349189FB7F89480910B01877F45
:10F2C00080930B019FBF8091C10D9091C20DA091C1
:10F2D000C30DB091C40D181619061A061B0684F545
:10F2E000E091970DF091980D428953896489758951
:10F2F000841B950BA60BB70B8093C10D9093C20D89
:10F30000A093C30DB093C40D8091040240914A189C
:10F3100050914B1860914C1870914D18082E000CAC
:10F32000990BAA0BBB0B840F951FA61FB71F8093C9
:10F330004A1890934B18A0934C18B0934D181498FA
:10F340008091D70D9091D80DA091D90DB091DA0D83
:10F350000196A11DB11D8093D70D9093D80DA09358
:10F36000D90DB093DA0D2150E091970DF091980DE1
:10F37000428953896489758984179507A607B70759
:10F3800008F451CEBB24B39401C0B12CE091970D89
:10F39000F091980D8091D70D9091D80DA091D90D35
:10F3A000B091DA0D46895789608D718D48175907DC
:10F3B0006A077B0708F416C14091C50D5091C60D30
:10F3C0006091C70D7091C80D068D178D20A131A1D8
:10F3D000AA27419FB12D529FC001629F900D619F4E
:10F3E000800D911D429FB00D811D9A1F519FB00D40
:10F3F000811D9A1F609FB00D811D9A1F509FB10DF6
:10F400008A1F9A1FB6958A1F9A1F349F800D911DDF
:10F41000359F900D112423AD34AD820F931F90932F
:10F42000CA0D8093C90D47A950AD61AD72ADA0E082
:10F43000B0E0481759076A077B0720F45093CA0DBC
:10F440004093C90D0091C90D1091CA0D1A8309830B
:10F4500001342CE9120720F401321E4478F004C074
:10F4600040E45CE95A83498389819A81969587951E
:10F47000969587959A83898384E00BC0A981BA8188
:10F48000A131E7E2BE0740F0B695A795BA83A983FC
:10F4900082E08093CE0D0CC081E08093CE0D098177
:10F4A0001A810032110520F420E230E03A832983EA
:10F4B00009811A81005211091A830983011528E074
:10F4C0001207E8F0E12FFF27EE0FFF1FEE0FFF1FDF
:10F4D000CF018E50954EFC01329625913491AA278A
:10F4E000039FA001029F410D5A1F06944A1F5A1FF5
:10F4F0001124FC0125913491241B350B20C08981F6
:10F500009A81969587958C7F8E50994EFC01259116
:10F510003491FC0132964591549169817A816770EA
:10F520007727649FC001659F900D749F900D1124F3
:10F53000B3E096958795BA95E1F7281B390B2436E9
:10F54000310590F4FBEAEF2EF3E0FF2ED7018D9109
:10F550007D01882319F00E944442F8CF89819A8165
:10F560000E946CD724E630E08091090E882301F1D7
:10F57000C901293BBBE03B07E0F068EB7BE00F945F
:10F58000E608883EE3E09E0718F48854944F02C0D2
:10F5900088EB9BE0A901481B590B60E070E04093A9
:10F5A000D30D5093D40D6093D50D7093D60D01C03B
:10F5B000C90190938900809388008091C50D909136
:10F5C000C60DA091C70DB091C80D820F931FA11D4C
:10F5D000B11D8093C50D9093C60DA093C70DB09338
:10F5E000C80D47C18091D70D9091D80DA091D90D2C
:10F5F000B091DA0D428D538D648D758D4817590782
:10F600006A077B0708F005C10091CF0D1091D00D5E
:10F610002091D10D3091D20D09831A832B833C8325
:10F62000468D578D60A171A1AA27059FB12D169F08
:10F630007001269FF00C259FE00CF11C069FB00D79
:10F64000E11CFA1E159FB00DE11CFA1E249FB00D9F
:10F65000E11CFA1E149FB10DEA1EFA1EB695EA1EB1
:10F66000FA1E709FE00CF11C719FF00C1124809128
:10F67000C90D9091CA0DFF96E816F90680F48E190F
:10F680009F0940815181628173816C01E12CF12CD1
:10F69000C416D506E606F70620F4CA0102C080812A
:10F6A000918181341CE9910728F481322EE492077C
:10F6B00048F002C080E49CE99695879596958795D9
:10F6C00024E007C0813137E2930730F096958795A3
:10F6D00022E02093CE0D08C021E02093CE0D803291
:10F6E000910510F480E290E08C01005211091E8314
:10F6F0000D83011528E01207E8F0E12FFF27EE0F38
:10F70000FF1FEE0FFF1FCF018E50954EFC0132966A
:10F7100025913491AA27039FA001029F410D5A1FF2
:10F7200006944A1F5A1F1124FC0125913491241B71
:10F73000350B20C08D819E81969587958C7F8E504C
:10F74000994EFC0125913491FC01329645915491DA
:10F750006D817E8167707727649FC001659F900DE2
:10F76000749F900D112443E0969587954A95E1F793
:10F77000281B390B2436310590F48BEAE82E83E000
:10F78000F82ED7018D917D01882319F00E94444203
:10F79000F8CF8D819E810E946CD724E630E0809165
:10F7A000090E882301F1C901293BBBE03B07E0F0CA
:10F7B00068EB7BE00F94E608883EE3E09E0718F4D0
:10F7C0008854944F02C088EB9BE0A901481B590B59
:10F7D00060E070E04093D30D5093D40D6093D50D4D
:10F7E0007093D60D01C0C901909389008093880061
:10F7F00089819A81AB81BC81820F931FA11DB11DAC
:10F800008093CF0D9093D00DA093D10DB093D20DD6
:10F8100030C02091CC0D3091CD0D8091090E882300
:10F8200001F1293BFBE03F07E0F0C90168EB7BE019
:10F830000F94E608883E03E0900718F48854944F2C
:10F8400002C088EB9BE0A901481B590B60E070E007
:10F850004093D30D5093D40D6093D50D7093D60D76
:10F860009C0130938900209388008091CB0D809378
:10F87000CE0D209188003091890080918400909174
:10F88000850040962817390748F4809184009091AC
:10F89000850040969093890080938800BB2031F0CA
:10F8A0001092980D1092970D0E9406ECF89480919A
:10F8B0000910882321F080916E008B7F03C0809116
:10F8C0006E00846080936E0080916F0082608093F0
:10F8D0006F0026960FB6F894DEBF0FBECDBFDF9146
:10F8E000CF91FF91EF91BF91AF919F918F917F91B8
:10F8F0006F915F914F913F912F911F910F91FF90C9
:10F90000EF90DF90CF90BF900F900BBE0F900FBE87
:10F910000F901F9018954F925F926F927F928F92E7
:10F920009F92AF92BF92CF92DF92EF92FF920F938E
:10F930001F93CF93DF93CDB7DEB76A970FB6F894D6
:10F94000DEBF0FBECDBF9A8F898F5B018A01DC01BC
:10F95000D7966D917D918D919C91DA970E9488FF49
:10F960006B017C01F50120813181428153810E942C
:10F97000E9FF0F94E4060F94670769877A878B87FE
:10F980009C87D8012D913D914D915C91C701B601A5
:10F990000E94E9FF0F94E4060F9467076D877E8746
:10F9A0008F87988B29853A854B855C85283731056B
:10F9B0004105510540F488E790E0A0E0B0E0898778
:10F9C0009A87AB87BC872D853E854F855889283718
:10F9D00031054105510540F488E790E0A0E0B0E032
:10F9E0008D879E87AF87B88BE98DFA8DED5BFF4FD2
:10F9F00020813181428153812D833E834F835887FB
:10FA0000CA01B9010E948AFF69837A838B839C8330
:10FA100069857A858B859C850E9488FF698B7A8BA6
:10FA20008B8B9C8B20E030E0A90169817A818B81EE
:10FA30009C810E9484FF882339F1A7019601C701A8
:10FA4000B6010E94E9FF4B015C0129893A894B8983
:10FA50005C89CA01B9010E94E9FF9B01AC01C501A3
:10FA6000B4010F941D064B015C0129813A814B8141
:10FA70005C81CA01B9010F941E069B01AC01C5014E
:10FA8000B4010F94FA0603C060E070E0CB010F945C
:10FA9000E4060F9462072B013C016D817E818F810A
:10FAA000988590958095709561957F4F8F4F9F4F6A
:10FAB0000E948AFF4B015C016D857E858F85988948
:10FAC0000E9488FF6D837E838F83988720E030E0DB
:10FAD000A901C501B4010E9484FF882349F12D8149
:10FAE0003E814F815885CA01B9010E94E9FF6D8BA3
:10FAF0007E8B8F8B988FA7019601C701B6010E945C
:10FB0000E9FF9B01AC016D897E898F89988D0F94E7
:10FB10001D066B017C01A5019401C501B4010F9480
:10FB20001E069B01AC01C701B6010F94FA0603C083
:10FB300060E070E0CB010F949307A98DBA8D5296C7
:10FB40008D909D90AD90BC90559775016401C4183F
:10FB5000D508E608F7080F946207C61AD70AE80A1C
:10FB6000F90AF7FE6BC020E030E0A90169817A81D3
:10FB70008B819C810E9484FF882309F447C0C501C2
:10FB8000B4010E9488FF6B017C0129813A814B817D
:10FB90005C81CA01B9010F941E069B01AC01C7012B
:10FBA000B6010E94E9FF6B017C0129893A894B89E2
:10FBB0005C89CA01B9010E94E9FF9B01AC01C70140
:10FBC000B6010F941D066B017C012D813E814F8192
:10FBD0005885CA01B9010E94E9FF9B01AC01C70128
:10FBE000B6010F941E066B017C0120E030E040E876
:10FBF00050E469817A818B819C810E94E9FF9B019D
:10FC0000AC01C701B6010F94FA0603C060E070E0D2
:10FC1000CB010F94E4060F9462072B013C0197FF80
:10FC200003C0412C512C3201481459046A047B044E
:10FC300010F024013501C12CD12C76018FB7F89436
:10FC4000E98DFA8D908193FD1DC0468A578A608E9A
:10FC5000718EC40CD51CE61CF71CC28ED38EE48EAC
:10FC6000F58E29853A854B855C8523AF34AF45AF4A
:10FC700056AFFF962D853E854F8558892083318369
:10FC8000428353838FBF6A960FB6F894DEBF0FBED0
:10FC9000CDBFDF91CF911F910F91FF90EF90DF903B
:10FCA000CF90BF90AF909F908F907F906F905F901C
:10FCB0004F9008950F931F93CF93DF93E091970D8B
:10FCC000F091980D82819381A481B581181619064F
:10FCD0001A061B06E4F48091940D80FF18C09CB1B5
:10FCE0008091020E95FB992790F98E7F892780934A
:10FCF000020E9091010E9170892349F08091400E7F
:10FD000081608093400E80E090E00E943475E09125
:10FD1000970DF091980D86819781A085B185181671
:10FD200019061A061B061CF58091940D81FF1FC051
:10FD3000909103018091020E91FB002700F910E0E1
:10FD400011950195110908270270112708270093C2
:10FD5000020E8091010E8270082349F08091400EBE
:10FD600082608093400E81E090E00E943475E091C3
:10FD7000970DF091980D82859385A485B585181609
:10FD800019061A061B0624F58091940D82FF20C0E7
:10FD900099B18091020E93FB992790F9C92F90E0B9
:10FDA000D92FD195C195D109C827C470DD27C8279F
:10FDB000C093020E8091010E8470C82349F0809197
:10FDC000400E84608093400E82E090E00E94347583
:10FDD0008091020E8093010EDF91CF911F910F91C0
:10FDE0000895CF93DF93E3ECF1E28491EF01219644
:10FDF000882321F00E944442FE01F7CFEBEBF1E2B1
:10FE00008491EF012196882321F00E944442FE0153
:10FE1000F7CF659903C0CFEBD3E002C0C4ECD3E0C9
:10FE20008991882319F00E944442FACF8AE00E9407
:10FE30004442E3EBF1E28491EF012196882321F023
:10FE40000E944442FE01F7CF8091030181FD03C06F
:10FE5000CFEBD3E002C0C4ECD3E08991882319F042
:10FE60000E944442FACF8AE00E944442EBEAF1E267
:10FE70008491EF012196882321F00E944442FE01E3
:10FE8000F7CF4B9903C0CFEBD3E002C0C4ECD3E073
:10FE90008991882319F00E944442FACF8AE0DF91C9
:10FEA000CF910C944442AF92BF92CF92DF92EF92E7
:10FEB000FF920F931F93CF93C82F882319F0E3E984
:10FEC000F1E20CC0EBE9F9E484918F010F5F1F4F61
:10FED0008823A9F30E944442F801F6CF84918F0150
:10FEE0000F5F1F4F882321F00E944442F801F6CF94
:10FEF000CC2319F0E6E7F1E20CC0EBE9F9E48491D8
:10FF00008F010F5F1F4F8823A9F30E944442F8011D
:10FF1000F6CF84918F010F5F1F4F882321F00E943D
:10FF20004442F801F6CF8AE00E944442C1112CC03D
:10FF3000EBE9F9E484918F010F5F1F4F882321F0D3
:10FF40000E944442F801F6CFE3E6F1E284918F018A
:10FF50000F5F1F4F882321F00E944442F801F6CF23
:10FF600080915E06882321F08AE00E9444423AC0D4
:10FF7000E8E5F1E284918F010F5F1F4F882391F133
:10FF80000E944442F801F6CF40915A0650915B0618
:10FF900060915C0670915D068FE491E20E9430EC06
:10FFA0008AE00E94444280915E06811127C0CC23E2
:10FFB00019F0E4E4F1E20CC0EBE9F9E484918F017B
:10FFC0000F5F1F4F8823A9F30E944442F801F6CF28
:10FFD00084918F010F5F1F4F882381F00E9444425C
:10FFE000F801F6CFEBE9F9E484918F010F5F1F4F21
:10FFF000882351F20E944442F801F6CFC11124C077
:020000021000EC
:10000000EBE9F9E484918F010F5F1F4F882321F002
:100010000E944442F801F6CFE3E3F1E284918F01BC
:100020000F5F1F4F882321F00E944442F801F6CF52
:10003000EBE9F9E484918F010F5F1F4F882321F0D2
:100040000E944442F801F6CF40915E1850915F182B
:1000500060916018709161188BE291E20E9430EC1F
:1000600040916218509163186091641870916518FE
:1000700088E291E20E9430EC409166185091671836
:10008000609168187091691885E291E20E9430ECE5
:1000900040916A1850916B1860916C1870916D18AE
:1000A00082E291E20E9430EC8AE00E944442C11157
:1000B00024C0EBE9F9E484918F010F5F1F4F88237F
:1000C00021F00E944442F801F6CFE4E0F1E284918D
:1000D0008F010F5F1F4F882321F00E944442F801D7
:1000E000F6CFEBE9F9E484918F010F5F1F4F88236E
:1000F00021F00E944442F801F6CF409178065091D9
:10010000790660917A0670917B068BEF90E20E94EF
:1001100030EC40917C0650917D0660917E06709196
:100120007F0688EF90E20E9430EC4091800650916B
:100130008106609182067091830685EF90E20E94AD
:1001400030EC40918406509185066091860670914E
:10015000870682EF90E20E9430EC8AE00E944442DF
:10016000C11124C0EBE9F9E484918F010F5F1F4FA7
:10017000882321F00E944442F801F6CFE0EDF0E23E
:1001800084918F010F5F1F4F882321F00E9444420A
:10019000F801F6CFEBE9F9E484918F010F5F1F4F6F
:1001A000882321F00E944442F801F6CF409188064E
:1001B0005091890660918A0670918B0687EC90E2D7
:1001C0000E9413EC40918C0650918D0660918E0632
:1001D00070918F0684EC90E20E9413EC409190069F
:1001E00050919106609192067091930681EC90E295
:1001F0000E9413EC409194065091950660919606EA
:10020000709197068EEB90E20E9413EC8AE00E94B8
:100210004442C11124C0EBE9F9E484918F010F5FDE
:100220001F4F882321F00E944442F801F6CFE4E7F3
:10023000F0E284918F010F5F1F4F882321F00E940D
:100240004442F801F6CFEBE9F9E484918F010F5FA6
:100250001F4F882321F00E944442F801F6CF4091BD
:10026000A0065091A1066091A2067091A3068BE6AC
:1002700090E20E9430EC40919C0650919D06609166
:100280009E0670919F0688E690E20E9430EC4091B5
:1002900098065091990660919A0670919B0685E6A2
:1002A00090E20E9430EC8AE00E944442C11124C0D6
:1002B000EBE9F9E484918F010F5F1F4F882321F050
:1002C0000E944442F801F6CFE1EFFFE184918F01F3
:1002D0000F5F1F4F882321F00E944442F801F6CFA0
:1002E000EBE9F9E484918F010F5F1F4F882321F020
:1002F0000E944442F801F6CF409174065091750671
:10030000609176067091770688EE9FE10E9430EC4E
:10031000409170065091710660917206709173065B
:1003200085EE9FE10E9430EC40917D1250917E124B
:1003300060917F127091801282EE9FE10E9413EC17
:100340004091A4065091A5066091A6067091A7065B
:100350008FED9FE10E9430EC4091A8065091A906D4
:100360006091AA067091AB068CED9FE10E9430EC83
:100370004091AC065091AD066091AE067091AF060B
:1003800089ED9FE10E9430EC4091B0065091B1069A
:100390006091B2067091B30686ED9FE10E9430EC49
:1003A0008AE00E944442C11124C0EBE9F9E484913F
:1003B0008F010F5F1F4F882321F00E944442F801F4
:1003C000F6CFE8ECFFE184918F010F5F1F4F882388
:1003D00021F00E944442F801F6CFEBE9F9E4849160
:1003E0008F010F5F1F4F882321F00E944442F801C4
:1003F000F6CF40910D0E50910E0E60910F0E709140
:10040000100E8FEB9FE10E9430EC4091110E509145
:10041000120E6091130E7091140E8CEB9FE10E94EE
:1004200030EC4091150E5091160E6091170E7091A0
:10043000180E89EB9FE10E9430EC8AE00E94444252
:10044000CC2379F089ECA82E8FE0B82E95ECC92E3C
:100450009FE0D92E2DECE22E2FE0F22E00E010E0EE
:1004600024C0EBE9F9E484918F010F5F1F4F8823CB
:1004700021F00E944442F801F6CFECE9FFE18491BB
:100480008F010F5F1F4F882321F00E944442F80123
:10049000F6CFEBE9F9E484918F010F5F1F4F8823BA
:1004A00089F20E944442F801F6CFB80183E99FE146
:1004B0000E944DECF501619171915F0180E99FE12E
:1004C0000E944DECF601619171916F018DE89FE101
:1004D0000E944DECF701619171917F018AE89FE1E3
:1004E0000E944DEC8AE00E9444420F5F1F4F023091
:1004F0001105D9F6C11124C0EBE9F9E484918F010B
:100500000F5F1F4F882321F00E944442F801F6CF6D
:10051000EBE7FFE184918F010F5F1F4F882321F0EC
:100520000E944442F801F6CFEBE9F9E484918F018F
:100530000F5F1F4F882321F00E944442F801F6CF3D
:100540004091A90D5091AA0D6091AB0D7091AC0D29
:1005500082E79FE10E9430EC2CEA35EC47E25EE353
:100560006091A50D7091A60D8091A70D9091A80D99
:100570000F94FA06AB01BC018FE69FE10E9430ECBC
:100580002CEA35EC47E25EE36091AD0D7091AE0D63
:100590008091AF0D9091B00D0E94E9FFAB01BC01BD
:1005A0008CE69FE10E9430EC8AE00E944442C11137
:1005B0000CC0EBE9F9E484918F010F5F1F4F882392
:1005C00021F00E944442F801F6CF4091A10D5091D4
:1005D000A20D6091A30D7091A40D83E69FE10E948E
:1005E00030EC2CEA35EC47E25EE360919D0D7091B2
:1005F0009E0D80919F0D9091A00D0F94FA06AB0176
:10060000BC0180E69FE10E9430EC2CEA35EC47E229
:100610005EE36091990D70919A0D80919B0D909180
:100620009C0D0E94E9FFAB01BC018DE59FE10E949A
:1006300030EC8AE0CF911F910F91FF90EF90DF9007
:10064000CF90BF90AF900C944442CF92DF92EF9244
:10065000FF920F931F93CF93DF936C017A018B016D
:10066000C0E0D0E0CE15DF0581F0D8016D918D019D
:10067000D601ED91FC910190F081E02DC601199514
:10068000892B11F02196EECF7E01C701DF91CF912A
:100690001F910F91FF90EF90DF90CF9008950F94EE
:1006A0001B09CF93DF93282F30E0F901E356FD4D6E
:1006B0008491F901E95AFD4DD491F901EF5EFD4DA8
:1006C000C491CC2391F081110E94F4C0EC2FF0E092
:1006D000EE0FFF1FE950FE4DA591B491EC91ED2373
:1006E00081E090E021F480E002C080E090E0DF91C2
:1006F000CF9108951F93CF93DF93282F30E0F90116
:10070000E356FD4D8491F901E95AFD4DD491F9016B
:10071000EF5EFD4DC491CC23C1F0162F81110E94D4
:10072000F4C0EC2FF0E0EE0FFF1FE352FE4DA59159
:10073000B4919FB7F894111104C08C91D095D8232F
:1007400002C0EC91DE2BDC939FBFDF91CF911F9114
:100750000895CF93DF932EE538E1C8E7D6E0A8E807
:10076000B6E080E090E0FC01E65FFA4D45915591DE
:1007700065917491F90141935193619371939F0134
:10078000FC01E650FB4D459155916591749149935B
:10079000599369937993FC01E651FB4D459155912D
:1007A000659174914D935D936D937D930496803123
:1007B0009105C9F680E090E0AAEFB3E48093A0062B
:1007C0009093A106A093A206B093A30680939C06E3
:1007D00090939D06A0939E06B0939F0680E090E0C4
:1007E000AAE7B4E48093980690939906A0939A069A
:1007F000B0939B06109274061092750610927606BE
:100800001092770680E29EE4A0E0B0E080937D1233
:1008100090937E12A0937F12B09380121092700674
:1008200010927106109272061092730680E090E0AA
:10083000A0E2B1E48093A4069093A506A093A60637
:10084000B093A7068093A8069093A906A093AA0642
:10085000B093AB068DEC9CECACECBEE38093AC06A5
:100860009093AD06A093AE06B093AF0680E090E003
:10087000A0EAB0E48093B0069093B106A093B206CC
:10088000B093B3068CE0EDE0FEE0DF011D928A95A7
:10089000E9F789EB90E09093CA0F8093C90F80EF3E
:1008A00090E09093CC0F8093CB0F8DE290E09093EB
:1008B000C60F8093C50F86E490E09093C80F809395
:1008C000C70F8FEF90E09093CE0F8093CD0F909352
:1008D000D00F8093CF0F8FE892ECABE9B1E4809317
:1008E000A90D9093AA0DA093AB0DB093AC0D8DEF15
:1008F00090E6A5E8BEE38093A50D9093A60DA09386
:10090000A70DB093A80D81E496E4A5EBB3E4809322
:10091000AD0D9093AE0DA093AF0DB093B00D89E2E5
:100920009CEDA9E4B3E48093A10D9093A20DA09354
:10093000A30DB093A40D80E294ECAFEDBFE38093E0
:100940009D0D90939E0DA0939F0DB093A00D89EEE9
:1009500094E2A6EBB5E48093990D90939A0DA09341
:100960009B0DB0939C0D10925E0680E090E0A0EE8F
:10097000BFE380935A0690935B06A0935C06B09306
:100980005D061092090E1092C40F0E949CE2EBE9E2
:10099000F9E48491EF012196882321F00E944442DA
:1009A000FE01F7CFE7ECF4E28491EF012196882372
:1009B00021F00E944442FE01F7CFDF91CF910895CC
:1009C0002F923F924F925F926F927F928F929F925F
:1009D000AF92BF92CF92DF92EF92FF920F931F934D
:1009E000CF93DF93CDB7DEB7CA55D1090FB6F894D0
:1009F000DEBF0FBECDBFADB6BEB62B961FAE1EAED0
:100A00002B9784E690E02D969FAF8EAF2D979E0199
:100A1000275B3F4F44E050E0BE016F5B7F4FCE014C
:100A2000855B9F4F0E94F9E19E01275B3F4F42E0AB
:100A300050E0BE01635B7F4FCE01855B9F4F0E94FC
:100A4000F9E143E050E0BE016F5B7F4F83EE92E03F
:100A50000F947D09892B09F43AC022968FAD229715
:100A6000863539F08FE322968FAF229723961FAEFB
:100A70002397EBE9F9E484918F010F5F1F4F8111F8
:100A800003C0EEEAF4E204C00E944442F801F3CF4E
:100A900084918F010F5F1F4F882321F00E944442F1
:100AA000F801F6CFBE016F5B7F4F85EA94E20E94AA
:100AB00066ECE7E9F4E284918F010F5F1F4F882312
:100AC00021F00E944442F801F6CF43DE4DC42DB61A
:100AD0003EB621961CAE1DAE1EAE1FAE21972B96C4
:100AE0001FAE1EAE2B979E01275B3F4F41E050E0AB
:100AF000BE016B5A7F4FCE01855B9F4F0E94F9E18B
:100B000080E1E3EBF2E0DE01919601900D928A958F
:100B1000E1F780E1E3ECF2E0DE01519601900D9205
:100B20008A95E1F780E1E3EDF2E0DE0111960190B4
:100B30000D928A95E1F76696CFAC6697D12C23E0AB
:100B4000C20ED11CCC0CDD1CCC0CDD1C8DB79EB7AD
:100B50008C199D090FB6F8949EBF0FBE8DBFEDB7DF
:100B6000FEB731963F012DB73EB72C193D090FB6A0
:100B7000F8943EBF0FBE2DBF0DB71EB70F5F1F4FBE
:100B80008DB79EB78C199D090FB6F8949EBF0FBE06
:100B90008DBFEDB7FEB731967F019E01275B3F4FBA
:100BA000A601B301CE01855B9F4F0E94F9E19E0132
:100BB000275B3F4FA601B801CE01855B9F4F0E9486
:100BC000F9E19E01275B3F4FA601B701CE01855B8E
:100BD0009F4F0E94F9E166968FAD669790E002966E
:100BE00028E8822E26E0922EB701AE014F5F5F4FBC
:100BF00028E736E069963FAF2EAF6997D8017E01AE
:100C000031E1E30EF11C3EE5C32E38E1D32E6B96A5
:100C10007FAE6EAE6B978E010F5D1F4F20E030E010
:100C2000821793072CF06B96EEADFFAD6B9701C06A
:100C3000F8014080518062807380F60141925192A8
:100C4000619271926F018217930734F04D905D901D
:100C50006D907C90139705C0F701408051806280B1
:100C600073806996EEADFFAD6997419251926192A2
:100C700071926996FFAFEEAF69978217930714F0F0
:100C8000FB0101C0FA014080518062807380F40151
:100C900041925192619271924F012F5F3F4F6C5F71
:100CA0007F4F4C5F5F4F1496F4E0EF0EF11C6B9694
:100CB000EEADFFAD6B9734966B96FFAFEEAF6B97D3
:100CC0000C5F1F4F2430310509F0AACF9E01275B2E
:100CD0003F4F44E050E060EA76E0CE01855B9F4FF5
:100CE0000E94F9E19E01275B3F4F44E050E06CE930
:100CF00076E0CE01855B9F4F0E94F9E19E01275B64
:100D00003F4F44E050E068E976E0CE01855B9F4FBD
:100D10000E94F9E19E01275B3F4F44E050E064E709
:100D200076E0CE01855B9F4F0E94F9E19E01275B33
:100D30003F4F44E050E060E776E0CE01855B9F4F97
:100D40000E94F9E19E01275B3F4F44E050E06DE7D0
:100D500072E1CE01855B9F4F0E94F9E19E01275B06
:100D60003F4F40E150E064EA76E0CE01855B9F4F63
:100D70000E94F9E19E01275B3F4F4CE050E06DE09F
:100D80007EE0CE01855B9F4F0E94F9E19E01275BCB
:100D90003F4F44E050E0BE01635C7F4FCE01855B76
:100DA0009F4F0E94F9E19E01275B3F4F41E050E0D9
:100DB000BE016C5A7F4FCE01855B9F4F0E94F9E1C7
:100DC0009E01275B3F4F44E050E0BE01635C7F4FD4
:100DD000CE01855B9F4F0E94F9E19E01275B3F4F4B
:100DE00041E050E0BE016D5A7F4FCE01855B9F4FC1
:100DF0000E94F9E19E01275B3F4F41E050E0BE01B8
:100E00006E5A7F4FCE01855B9F4F0E94F9E1649639
:100E10008FAD64976396EFAC63978E9D700111243C
:100E200000E010E09E01275B3F4F44E050E0BE0130
:100E30000E151F0551F0635C7F4FCE01855B9F4F00
:100E40000E94F9E10F5F1F4FEDCF675C7F4FCE012E
:100E5000855B9F4F0E94F9E11AE011509E01275BCC
:100E60003F4F112359F044E050E0BE01635C7F4FD7
:100E7000CE01855B9F4F0E94F9E1EFCF41E050E04A
:100E8000BE016F5A7F4FCE01855B9F4F0E94F9E1F3
:100E90009E01275B3F4F41E050E0BE01605B7F4F0A
:100EA000CE01855B9F4F0E94F9E19E01275B3F4F7A
:100EB00044E050E0BE016B5C7F4FCE01855B9F4FED
:100EC0000E94F9E19E01275B3F4F44E050E0BE01E4
:100ED0006F5C7F4FCE01855B9F4F0E94F9E1629668
:100EE0008FAD62976196EFAC61978E9D7001112472
:100EF00000E010E09E01275B3F4F0E151F0569F0D3
:100F000044E050E0BE01635C7F4FCE01855B9F4FA4
:100F10000E94F9E10F5F1F4FEDCF41E050E0BE01AD
:100F20006A5A7F4FCE01855B9F4F0E94F9E19E0177
:100F3000275B3F4F44E050E0BE01635C7F4FCE0132
:100F4000855B9F4F0E94F9E19E01275B3F4F41E087
:100F500050E0BE01615B7F4FCE01855B9F4F0E94D9
:100F6000F9E121961CAE1DAE1EAE1FAE21971DE00D
:100F700011509E01275B3F4F44E050E0112349F0A0
:100F8000BE01635C7F4FCE01855B9F4F0E94F9E1FC
:100F9000EFCF69EC7FE0CE01855B9F4F0E94F9E1C6
:100FA0009E01275B3F4F44E050E065EC7FE0CE01BF
:100FB000855B9F4F0E94F9E19E01275B3F4F44E014
:100FC00050E06DEC7FE0CE01855B9F4F0E94F9E120
:100FD00010E09E01275B3F4F44E050E0BE01635CA0
:100FE0007F4FCE01855B9F4F0E94F9E1111110C028
:100FF0002196CCACDDACEEACFFAC219720E030E824
:101000004BE355E4C701B6010E9484FF811102C081
:1010100004E02EC0C092A90DD092AA0DE092AB0DB3
:10102000F092AC0D9E01275B3F4F44E050E065EA33
:101030007DE0CE01855B9F4F0E94F9E19E01275B19
:101040003F4F44E050E06DEA7DE0CE01855B9F4F6D
:101050000E94F9E19E01275B3F4F44E050E0BE0152
:10106000635C7F4FCE01855B9F4F0E94F9E110C00A
:10107000015071F09E01275B3F4F44E050E0BE01FC
:10108000635C7F4FCE01855B9F4F0E94F9E1F0CFFB
:101090001F5F153009F09DCF9E01275B3F4F42E057
:1010A00050E0BE01695B7F4FCE01855B9F4F0E9480
:1010B000F9E19E01275B3F4F44E050E0BE01635CD5
:1010C0007F4FCE01855B9F4F0E94F9E12196CCAC0A
:1010D000DDACEEACFFAC219720E030E84BE355E40B
:1010E000C701B6010E9484FF882301F1C092A10DBF
:1010F000D092A20DE092A30DF092A40D9E01275B69
:101100003F4F44E050E06DE97DE0CE01855B9F4FAD
:101110000E94F9E19E01275B3F4F44E050E069E9FE
:101120007DE0CE01855B9F4F0E94F9E19E01275B28
:101130003F4F42E050E0BE016B5B7F4FCE01855BCD
:101140009F4F0E94F9E19E01275B3F4F41E050E035
:10115000BE016A5A7F4FCE01855B9F4F0E94F9E125
:1011600019E011509E01275B3F4F112359F044E0D5
:1011700050E0BE01635C7F4FCE01855B9F4F0E94B4
:10118000F9E1EFCF41E050E06EE576E0CE01855B1E
:101190009F4F0E94F9E110E09E01275B3F4F44E022
:1011A00050E0BE01635C7F4FCE01855B9F4F0E9484
:1011B000F9E111110EC021968CAD9DADAEADBFAD64
:1011C000219780935A0690935B06A0935C06B09398
:1011D0005D061F5F153001F71BE09E01275B3F4F47
:1011E00042E050E0BE016B5C7F4FCE01855B9F4FBC
:1011F0000E94F9E1115089F79E01275B3F4F44E0BF
:1012000050E0BE01635C7F4FCE01855B9F4F0E9423
:10121000F9E19E01275B3F4F44E050E0BE01635C73
:101220007F4FCE01855B9F4F0E94F9E114E0115082
:1012300071F09E01275B3F4F44E050E0BE016F5CC0
:101240007F4FCE01855B9F4F0E94F9E1F0CF2B9637
:101250002EAD3FAD2B972F968EAD9FAD2F972817B4
:10126000390719F0E9ECF6E13DC00E949CE2EBE998
:10127000F9E484918F010F5F1F4F811103C003EECA
:1012800012E004C00E944442F801F3CFF8018191BA
:101290008F01882319F00E944442F8CF2D966EAD3D
:1012A0007FAD2D97645671098AE794E20E944DEC58
:1012B0002B964EAD5FAD2B9760E070E08DE694E22B
:1012C0000E9413ECEAE6F4E284918F010F5F1F4F56
:1012D000882309F444C00E944442F801F5CF0E94DB
:1012E0004442F80184918F010F5F1F4F8111F7CFA6
:1012F000EAE4F4E284918F010F5F1F4F882321F00D
:101300000E944442F801F6CF2F966EAD7FAD2F9725
:1013100080E090E04AE00E944B42E5E4F4E28491F0
:101320008F010F5F1F4F882321F00E944442F80174
:10133000F6CF2B966EAD7FAD2B9780E090E04AE024
:101340000E944B42E5E3F4E284918F010F5F1F4F4F
:10135000882321F00E944442F801F6CFFAD90FB653
:10136000F8943EBE0FBE2DBE80E00E94537F909148
:10137000C30F81E089270FB6F894BEBE0FBEADBE85
:10138000C65ADF4F0FB6F894DEBF0FBECDBFDF9158
:10139000CF911F910F91FF90EF90DF90CF90BF9072
:1013A000AF909F908F907F906F905F904F903F9005
:1013B0002F9008958F929F92AF92BF92CF92DF921B
:1013C000EF92FF920F931F93CF93DF93CDB7DEB7CA
:1013D000C155D1090FB6F894DEBF0FBECDBF19823B
:1013E0001A821B821C828091CE039091CF03A09120
:1013F000D003B091D1038D839E83AF83B8872196AC
:101400001FAE1EAE219784E690E023969FAF8EAF6D
:1014100023971092C30F9E01215C3F4F44E050E0A0
:10142000BE016B5F7F4FCE018F5B9F4F0E9431E209
:1014300023968EAD9FAD2397029623969FAF8EAFD6
:10144000239721961FAE1EAE219781E02A968FAF7B
:101450002A979E01215C3F4F41E050E0BE01675B4F
:101460007F4FCE018F5B9F4F0E9431E29E01215C36
:101470003F4F40E150E06EE578E1CE018F5B9F4F3A
:101480000E9431E29E01215C3F4F40E150E068E75D
:1014900076E0CE018F5B9F4F0E9431E29E01215C7E
:1014A0003F4F40E150E068E876E0CE018F5B9F4F10
:1014B0000E9431E29E01215C3F4F44E050E060EA2F
:1014C00076E0CE018F5B9F4F0E9431E29E01215C4E
:1014D0003F4F44E050E06CE976E0CE018F5B9F4FD8
:1014E0000E9431E29E01215C3F4F44E050E068E9F8
:1014F00076E0CE018F5B9F4F0E9431E29E01215C1E
:101500003F4F44E050E064E776E0CE018F5B9F4FB1
:101510000E9431E29E01215C3F4F44E050E060E7D1
:1015200076E0CE018F5B9F4F0E9431E29E01215CED
:101530003F4F44E050E06DE772E1CE018F5B9F4F7B
:101540000E9431E29E01215C3F4F40E150E064EA9D
:1015500076E0CE018F5B9F4F0E9431E29E01215CBD
:101560003F4F4CE050E06DE07EE0CE018F5B9F4F3F
:101570000E9431E280E090E0A0E2B1E489879A879E
:10158000AB87BC879E01215C3F4F44E050E0BE0129
:10159000675F7F4FCE018F5B9F4F0E9431E22B969A
:1015A0001FAE2B9719821A821B821C8283E02C9615
:1015B0008FAF2C972D968FAF2D979E01215C3F4FBB
:1015C00041E050E0BE01665B7F4FCE018F5B9F4FD5
:1015D0000E9431E29E01215C3F4F44E050E0BE0199
:1015E0006F5F7F4FCE018F5B9F4F0E9431E29E0164
:1015F000215C3F4F41E050E0BE01655B7F4FCE0173
:101600008F5B9F4F0E9431E29E01215C3F4F41E082
:1016100050E0BE01645B7F4FCE018F5B9F4F0E9405
:1016200031E21AE0115071F09E01215C3F4F44E01D
:1016300050E0BE016F5F7F4FCE018F5B9F4F0E94D6
:1016400031E2F0CF1D861E861F86188A9E01215C1E
:101650003F4F44E050E0BE01635F7F4FCE018F5BA0
:101660009F4F0E9431E219821A821B821C821AE06B
:10167000115071F09E01215C3F4F44E050E0BE01EB
:101680006F5F7F4FCE018F5B9F4F0E9431E2F0CFA3
:1016900083E02E968FAF2E972F968FAF2F97198AB4
:1016A0001A8A1B8A1C8A1D8A1E8A1F8A188E198212
:1016B0001A821B821C829E01215C3F4F41E050E058
:1016C000BE01635B7F4FCE018F5B9F4F0E9431E273
:1016D0009E01215C3F4F41E050E0BE01625B7F4FC5
:1016E000CE018F5B9F4F0E9431E29E01215C3F4FF4
:1016F00044E050E0BE016B5E7F4FCE018F5B9F4F99
:101700000E9431E29E01215C3F4F44E050E0BE0167
:101710006F5E7F4FCE018F5B9F4F0E9431E20AE0E8
:1017200010E00150110971F09E01215C3F4F44E02F
:1017300050E0BE016F5F7F4FCE018F5B9F4F0E94D5
:1017400031E2EFCF60961FAE609719821A821B823A
:101750001C828FEF61968FAF61979E01215C3F4F96
:1017600041E050E0BE01615B7F4FCE018F5B9F4F38
:101770000E9431E29E01215C3F4F44E050E0BE01F7
:101780006F5F7F4FCE018F5B9F4F0E9431E29E01C2
:10179000215C3F4F41E050E0BE01605B7F4FCE01D6
:1017A0008F5B9F4F0E9431E219821A821B821C823A
:1017B0001DE011509E01215C3F4F44E050E0112399
:1017C00049F0BE016F5F7F4FCE018F5B9F4F0E943C
:1017D00031E2EFCF69EC7FE0CE018F5B9F4F0E943B
:1017E00031E29E01215C3F4F44E050E065EC7FE038
:1017F000CE018F5B9F4F0E9431E29E01215C3F4FE3
:1018000044E050E06DEC7FE0CE018F5B9F4F0E9483
:1018100031E210E0C12C80E8D82E8BE3E82E85E47D
:10182000F82E812C912C90E8A92E9FE3B92E11114E
:1018300036C09E01215C3F4F44E050E069EA7DE004
:10184000CE018F5B9F4F0E9431E29E01215C3F4F92
:1018500044E050E065EA7DE0CE018F5B9F4F0E943F
:1018600031E29E01215C3F4F44E050E06DEA7DE0B3
:10187000CE018F5B9F4F0E9431E289829A82AB82B8
:10188000BC829E01215C3F4F44E050E0BE016F5F8F
:101890007F4FCE018F5B9F4F0E9431E226C0C982ED
:1018A000DA82EB82FC829E01215C3F4F44E050E0F3
:1018B000BE016F5F7F4FCE018F5B9F4F0E9431E271
:1018C00019821A821B821C8204E0015071F09E0171
:1018D000215C3F4F44E050E0BE016F5F7F4FCE017F
:1018E0008F5B9F4F0E9431E2F0CF1F5F153009F0F0
:1018F0009ECF84E190E025969FAF8EAF25979E0105
:10190000215C3F4F42E050E0BE016D5B7F4FCE0156
:101910008F5B9F4F0E9431E29E01215C3F4F44E06C
:1019200050E061EA7DE0CE018F5B9F4F0E9431E283
:101930009E01215C3F4F44E050E06DE97DE0CE0127
:101940008F5B9F4F0E9431E29E01215C3F4F44E03C
:1019500050E069E97DE0CE018F5B9F4F0E9431E24C
:1019600080E290E027969FAF8EAF27979E01215C83
:101970003F4F42E050E0BE016B5B7F4FCE018F5B7B
:101980009F4F0E9431E262961FAE629780E090E026
:10199000A0E4B0E4898F9A8FAB8FBC8F80E090E099
:1019A000A4E3B2E48D8F9E8FAF8FB8A319A21AA2C1
:1019B0001BA21CA21DA21EA21FA218A619A61AA62F
:1019C0001BA61CA680E090E0A0E5B1E48DA79EA731
:1019D000AFA7B8AB19AA1AAA1BAA1CAA80E090E06C
:1019E000A0E0B1E48DAB9EABAFABB8AF9E01215C84
:1019F0003F4F41E050E0BE016F5A7F4FCE018F5BF9
:101A00009F4F0E9431E29E01215C3F4F44E050E035
:101A1000BE01675E7F4FCE018F5B9F4F0E9431E218
:101A20009E01215C3F4F44E050E0BE01635E7F4F6A
:101A3000CE018F5B9F4F0E9431E29E01215C3F4FA0
:101A400044E050E0BE016F5D7F4FCE018F5B9F4F42
:101A50000E9431E29E01215C3F4F44E050E0BE0114
:101A60006B5D7F4FCE018F5B9F4F0E9431E29E01E5
:101A7000215C3F4F44E050E0BE01675D7F4FCE01E7
:101A80008F5B9F4F0E9431E29E01215C3F4F44E0FB
:101A900050E0BE01635D7F4FCE018F5B9F4F0E9480
:101AA00031E29E01215C3F4F44E050E0BE016F5C9B
:101AB0007F4FCE018F5B9F4F0E9431E29E01215CE0
:101AC0003F4F44E050E0BE016B5C7F4FCE018F5B27
:101AD0009F4F0E9431E29E01215C3F4F41E050E068
:101AE0006EE576E0CE018F5B9F4F0E9431E210E001
:101AF00011110CC080915A0690915B06A0915C0672
:101B0000B0915D0689839A83AB83BC839E01215C7F
:101B10003F4F44E050E0BE016F5F7F4FCE018F5BCF
:101B20009F4F0E9431E21F5F153011F729961FAEBB
:101B30001EAE29971CE0115071F09E01215C3F4FB1
:101B400042E050E0BE01695B7F4FCE018F5B9F4F4B
:101B50000E9431E2F0CF19821A821B821C829E0100
:101B6000215C3F4F44E050E0BE016F5F7F4FCE01EC
:101B70008F5B9F4F0E9431E29E01215C3F4F44E00A
:101B800050E0BE016F5F7F4FCE018F5B9F4F0E9481
:101B900031E219AE1AAE1BAE1CAE14E0115071F05A
:101BA0009E01215C3F4F44E050E0BE01675C7F4FE7
:101BB000CE018F5B9F4F0E9431E2F0CF8091C30F27
:101BC000811150C02396EEACFFAC239721968EADC9
:101BD0009FAD21979EAF8DAF84E690E023969FAF97
:101BE0008EAF23979E01215C3F4F44E050E063EEAF
:101BF00072E0CE018F5B9F4F0E9431E29E01215C1B
:101C00003F4F42E050E0BE01635C7F4FCE018F5BEF
